:200000000C94ED0A0C94180B0C94180B0C94180B0C94180B0C94180B0C94180B0C94180BF4
:200020000C94180B0C94180B0C949F8F0C94198E0C94180B0C94180B0C94180B0C94180B19
:200040000C94180B0C94736E0C94180B0C94180B0C94180B0C94180B0C944B760C94E28CE1
:200060000C94180B0C94180B0C94180B0C94180B0C94180B0C94180B0C94180B0C94180B68
:200080000C94180B0C94180B0C94180B0C94180B0C94180B0C94180B084AD73B3BCE016EF2
:2000A00084BCBFFDC12F3D6C74319ABD56833DDA3D00C77F11BED9E4BB4C3E916BAAAABE5D
:2000C000000000803F05A84CCDB2D44EB93836A9020C50B9918688083CA6AAAA2ABE00001B
:2000E00000803F4D3834205820592045006563686F3A0043616E6E6F7420656E7465722098
:200100007375626469723A20004D3234004D3233202573006175746F25692E6700457272DA
:200120006F723A006572726F722077726974696E6720746F2066696C65004E6F74205344AB
:20014000207072696E74696E67002F005344207072696E74696E67206279746520002E00A1
:2001600044656C6574696F6E206661696C65642C2046696C653A200046696C652064656CCB
:20018000657465643A002E006F70656E206661696C65642C2046696C653A20005772697452
:2001A000696E6720746F2066696C653A20002E006F70656E206661696C65642C2046696C18
:2001C000653A20002E006F70656E206661696C65642C2046696C653A200046696C652073C2
:2001E000656C6563746564002053697A653A200046696C65206F70656E65643A20002E0071
:200200006F70656E206661696C65642C2046696C653A200053442063617264206F6B006FC7
:2002200070656E526F6F74206661696C656400766F6C756D652E696E6974206661696C65B7
:200240006400534420696E6974206661696C006563686F3A0048617264636F646564204458
:20026000656661756C742053657474696E6773204C6F616465640053746F726564207365BA
:200280007474696E67732072657472696576656400205A0020590020204D3938205800482A
:2002A00079737465726573697320286D6D293A002044002049002020204D33303120500050
:2002C0005049442073657474696E67733A00205A0020590020204D323036205800486F6DC2
:2002E00065206F666673657420286D6D293A00204500205A00205800204200205400202000
:200300004D323035205300416476616E636564207661726961626C65733A20533D4D696E89
:2003200020666565647261746520286D6D2F73292C20543D4D696E2074726176656C20663B
:200340006565647261746520286D6D2F73292C20423D6D696E696D756D207365676D656E70
:20036000742074696D6520286D73292C20583D6D6178696D756D205859206A65726B202825
:200380006D6D2F73292C20205A3D6D6178696D756D205A206A65726B20286D6D2F73292C58
:2003A0002020453D6D6178696D756D2045206A65726B20286D6D2F73290020540020204D5E
:2003C000323034205300416363656C65726174696F6E3A20533D616363656C657261746953
:2003E0006F6E2C20543D7265747261637420616363656C65726174696F6E00204500205A65
:200400000020590020204D3230312058004D6178696D756D20416363656C65726174696F71
:200420006E20286D6D2F7332293A00204500205A0020590020204D3230332058004D6178DD
:20044000696D756D2066656564726174657320286D6D2F73293A00204500205A0020590092
:2004600020204D393220580053746570732070657220756E69743A0053657474696E67732B
:200480002053746F7265640020653D00207A3D0020793D00205348494654533A783D00205C
:2004A0004500205A00205900483D58006563686F3A004572726F723A005072696E74657226
:2004C0002073746F707065642064756520746F206572726F72732E204669782074686520E9
:2004E0006572726F7220616E6420757365204D39393920746F20726573746172742E20285C
:2005000054656D70657261747572652069732072657365742E20536574206974206166743C
:2005200065722072657374617274696E6729005072696E7465722068616C7465642E206B29
:20054000696C6C28292063616C6C656421006F6B00526573656E643A20002200556E6B6E10
:200560006F776E20636F6D6D616E643A2022007A5F6D696E3A2000795F6D61783A20007845
:200580005F6D696E3A20005A3A00593A0020436F756E7420583A2000453A005A3A00593A96
:2005A00000583A004D616368696E652D547970653A20506978696520382C204669726D7723
:2005C0006172652D56657273696F6E3A20312E302E3134303731346120202020416C6C206E
:2005E0005269676874732052657365727665642C20506F6C6172203344204C4C430A002024
:20060000423A0020453A00543A0020573A0020453A00543A002042403A0020403A00202F8E
:200620000020423A00202F006F6B20543A002569206D696E2C2025692073656300456E6409
:200640002066696C65206C69737400426567696E2066696C65206C697374000000C8420073
:2006600000B44300001643000020410000000000002041FF00FF000000000000B443000073
:2006800000000000000000000000000000000000C8420000B44300001643256920686F7506
:2006A0007273202569206D696E7574657300446F6E65207072696E74696E672066696C65B1
:2006C000005072696E7465722073746F707065642064756520746F206572726F72732E20AB
:2006E00046697820746865206572726F7220616E6420757365204D39393920746F20726556
:2007000073746172742E202854656D70657261747572652069732072657365742E20536562
:20072000742069742061667465722072657374617274696E6729006F6B004E6F204C696EB0
:2007400065204E756D626572207769746820636865636B73756D2C204C617374204C696E39
:20076000653A20004E6F20436865636B73756D2077697468206C696E65206E756D6265725D
:200780002C204C617374204C696E653A2000636865636B73756D206D69736D617463682C82
:2007A000204C617374204C696E653A20004C696E65204E756D626572206973206E6F7420E5
:2007C0004C617374204C696E65204E756D6265722B312C204C617374204C696E653A200016
:2007E0004D31313000446F6E6520736176696E672066696C652E006F6B004D32390020202C
:20080000506C616E6E657242756666657242797465733A20002046726565204D656D6F728B
:20082000793A2000417567203131203230313400436F6D70696C65643A20007069786965B9
:200840007072696E746572736C6C6300207C20417574686F723A200041756720313120326C
:200860003031342031363A34383A323900204C61737420557064617465643A2000312E308D
:200880002E30004D61726C696E200020536F6674776172652052657365740020576174633A
:2008A00068646F67205265736574002042726F776E206F757420526573657400204578745F
:2008C00065726E616C20526573657400506F7765725570007374617274002200656E717508
:2008E00065696E672022002200656E717565696E672022007C3C3E5E2B3D3F2F5B5D3B2C0A
:200900002A225C0045313A200045303A20005A3A2000593A2000583A20004D53312C4D53DA
:20092000322050696E730A0024F404D9201BC40C5C0E9804C4095F0265077101F405F900BD
:20094000FB04B30048048700C10369005803550003034500BE023A008402310053022A00BA
:200960002902250004022000E4011C00C8011900AF01170098011400840113007101100090
:200980006101100051010E0043010D0036010B002B010B0020010B00150109000C0109005A
:2009A00003010800FB000800F3000800EB000700E4000600DE000600D8000600D2000600B7
:2009C000CC000500C7000500C2000500BD000400B9000400B5000400B1000400AD00040016
:2009E000A9000400A5000300A20003009F0004009B000300980003009500020093000300F4
:200A0000900003008D0002008B000300880002008600020084000300810002007F00020089
:200A20007D0002007B000200790002007700010076000200740002007200010071000200F3
:200A40006F0002006D0001006C0002006A000100690002006700010066000100650001003E
:200A6000640002006200010061000100600001005F0002005D0001005C0001005B00010072
:200A80005A000100590001005800010057000100560001005500010054000100530000009B
:200AA000530001005200010051000100500001004F0001004E0000004E0001004D000100B1
:200AC0004C0001004B0000004B0001004A00010049000100480000004800010047000100C4
:200AE0004600000046000100450000004500010044000100430000004300010042000000D0
:200B0000420001004100000041000100400001003F0000003F0001003E0000003E000100D2
:200B20003D0000003D0001003C0000003C0000003C0001003B0000003B0001003A000000D4
:200B40003A00010039000000390001003800000038000000380001003700000037000100CF
:200B60003600000036000000360001003500000035000000350001003400000034000000CA
:200B80003400010033000000330000003300010032000000320000003200010031000000BE
:200BA00031000000310001003000000030000000300001002F0000002F0000002F000000B4
:200BC0002F0001002E0000002E0000002E0001002D0000002D0000002D0000002D000100A5
:200BE0002C0000002C0000002C0000002C0001002B0000002B0000002B0000002B00010097
:200C00002A0000002A0000002A0000002A0001002900000029000000290000002900000087
:200C2000290001002800000028000000280000002800000028000100270000002700000073
:200C400027000000270000002700010026000000260000002600000026000000260001005F
:200C600025000000250000002500000025000000250000002500010024000000240000004D
:200C8000240000002400000024000100230000002300000023000000230000002300000038
:200CA000230000002300010022000000220000002200000022000000220000002200010020
:200CC00021000000210000002100000021000000210000002100000021000100200000000C
:200CE000200000002000000020000000200000002000000020000000200001001F000000F4
:200D00001F0000001F0000001F0000001F0000001F0000001F0001001E0000001E000000DC
:200D20001E0000001E00000024F4D43050C38E20C2A24017828B7011127A910D816CD90A57
:200D4000A861E108C7586607615143061E4B5D05C145A7041A411104093D9803713931036F
:200D60004036DB0265339102D4305402802E1D02632CEE01752AC501B028A00110278101B9
:200D80008F2564012B244B01E0223401AC211F018D200D01801FFC00841EED00971DDF0003
:200DA000B81CD200E61BC600201BBC00641AB200B219A8000A19A0006A189900D1179100D5
:200DC00040178B00B516840031167E00B31579003A157300C7146F0058146A00EE13660093
:200DE0008813630025135E00C7125B006C12570015125400C111510070114F0021114B006B
:200E0000D61049008D1047004610440002104200C00F4000800F3E00420F3C00060F3B0018
:200E2000CB0E3800930E37005C0E3500270E3400F30D3200C10D3100900D3000600D2E0028
:200E4000320D2D00050D2C00D90C2B00AE0C2900850C29005C0C2700350C27000E0C260004
:200E6000E80B2400C40B2400A00B23007D0B23005A0B2100390B2100180B2000F80A1F00A0
:200E8000D90A1E00BB0A1E009D0A1D00800A1D00630A1C00470A1B002C0A1B00110A1A0088
:200EA000F7091A00DD091900C4091900AB091900920917007B091800630917004C0916002A
:200EC00036091600200916000A091500F5081500E0081400CC081400B8081400A4081400CC
:200EE000900813007D0812006B0813005808120046081200340811002308110012081100A4
:200F000001081100F0071000E0071000D0071000C0071000B0070F00A107100091070E00D7
:200F200083070F0074070F0065070E0057070E0049070E003B070D002E070E0020070D0084
:200F400013070D0006070D00F9060C00ED060D00E0060C00D4060C00C8060C00BC060C00C5
:200F6000B0060C00A4060B0099060C008D060B0082060B0077060B006C060B0061060A00A8
:200F800057060B004C060A0042060A0038060A002E060A0024060A001A060A001006090038
:200FA00007060A00FD050900F4050900EB050900E2050900D9050900D0050900C70509008A
:200FC000BE050900B5050800AD050800A50509009C050800940508008C05080084050800A2
:200FE0007C050800740508006C050700650508005D050700560508004E0507004705070084
:201000004005080038050700310507002A050700230507001C050600160507000F05070039
:201020000805060002050700FB040600F5040700EE040600E8040600E2040700DB040600CE
:20104000D5040600CF040600C9040600C3040600BD040600B7040600B1040500AC04060040
:20106000A6040600A00405009B04060095040500900406008A04050085040500800406008F
:201080007A04050075040500700405006B04050066040500610405005C04050057040500C4
:2010A000520405004D04050048040500430405003E0404003A0405003504050030040400E3
:2010C0002C04050027040400230405001E0404001A04040016040500110404000D040400EB
:2010E000090405000404040000040400FC030400F8030400F4030400F0030400EC030400E3
:20110000E8030400E4030400E0030400DC030400D8030400D4030400D0030400CC030400C7
:20112000C8030300C50303006563686F3A00205A3A0020593A0020583A00656E6473746F97
:201140007073206869743A20004572726F723A0054656D7065726174757265206865617459
:20116000656420626564207377697463686564206F66662E204D415854454D5020747269AC
:20118000676765726564202121003A204578747275646572207377697463686564206F6662
:2011A000662E204D494E54454D50207472696767657265642021003A204578747275646508
:2011C00072207377697463686564206F66662E204D415854454D50207472696767657265E4
:2011E00064202100202D20496E76616C6964206578747275646572206E756D626572202199
:2012000000504944204175746F74756E652066696E6973686564202120506C616365207438
:201220006865204B702C204B6920616E64204B6420636F6E7374616E747320696E207468F4
:201240006520636F6E66696775726174696F6E2E6800504944204175746F74756E65206623
:2012600061696C6564212074696D656F75740020403A006F6B20543A006F6B20423A00503F
:201280004944204175746F74756E65206661696C6564212054656D706572617475726520D8
:2012A000746F206869676800204B643A2000204B693A2000204B703A200020436C617369F3
:2012C000632050494420002054753A2000204B753A2000206D61783A2000206D696E3A2093
:2012E0000020643A200020626961733A200070012C0190012701B0012201C0011D01F001FC
:2013000018011002130130020E016002090190020401C002FF000003FA004003F5008003D1
:20132000F000D003EB002004E6007004E100E004DC004005D700C005D2004006CD00D00644
:20134000C8008007C3003008BE00F008B900C009B400B00AAF00B00BAA00D00CA500000EFA
:20136000A000500F9B00C01096005012910000148C00C0158700B0178200B0197D00D01B04
:201380007800001E730040206E0090226900F024640040275F0090295A00E02B5500102E6C
:2013A000500020304B0010324600E033410090353C001037370070383200A0392D00B03A1D
:2013C0002800A03B2300603C1E00103D1900903D1400103E0F00703E0A00C03E0500003F8F
:2013E00000002000204163743A2000526F643A2000205761726E696E672120496E636F6E8E
:2014000073697374656E7420706172616D657465727321002070756C732000207065726979
:201420006F642028572920002070686173652028502920005A576F62626C6520416D7020CC
:201440002841292000437573746F6D20776F62626C652066756E6374696F6E0001290229E9
:20146000042908291029202940298029012C022C01260226042608261026202640268026F0
:20148000402C802C012302230423082310232023402380230120022004200820102020201E
:2014A00040208020102C202C012F022F042F082F102F202F402F802F7EFE7EFD7EFB7EF748
:2014C0007EEF7EDF7EBF7E7F00010000FC1412000200000E15430003000051150401030903
:2014E00004551518020309046F15160303090487150C0001C10201803601813612010002B7
:2015000002000020C016830400010102030109024300020100C032090400000102020100EE
:20152000052400100105240100010424020605240600010705820308004009040100020AF3
:2015400000000007050302400000070584024000000403090418035400650065006E00733A
:201560000079006400750069006E006F00000016035500530042002000530065007200691D
:201580000061006C0000000C03310032003300340035000000494E46494E4954594E414E29
:2015A000CDCCCC3D0AD7233C17B7D13877CC2B329595E6241FB14F0A000020410000C8420A
:2015C00000401C4620BCBE4CCA1B0E5AAEC59D74B826B72888860C93B22811241FBECFEF9E
:2015E000D0E2DEBFCDBF13E0A0E0B1E0E2EFF1E301E00BBF02C007900D92A234B107D9F766
:201600001BBE10E1A2E4B3E001C01D92A333B107E1F715E1C8EDD5E104C02297FE010E9492
:201620009F98C03DD107C9F70E941D900C94ED980C940000A0E0B0E0E0E2FBE00C94BC9829
:20164000EC015B016115710519F0FB0191838083F9908F2D90E00E94A398892BC9F7FDE254
:20166000FF1621F4F990EE24E39405C02BE2F21609F4F990EE248E0101501040C80165E975
:2016800075E143E050E069D2892BF9F48E010E5F1F4FC80168E975E145E050E05ED2892BB2
:2016A00019F48E01095F1F4FA114B10419F0F50111830083E0FC04C070E090E080E813C09D
:2016C00070E090E080E86FEF07C1C8016DE975E143E050E042D2892B69F4A114B10429F448
:2016E00070E090E080EC6FE7F7C02296F501D183C083F6CF8824992440E050E060E070E05E
:20170000EF2DE053EA30A0F5F2E0EF2A8E2D90E09C0128703070E2FE06C0232B79F50894E2
:20172000811C911C2BC0232B19F0089481089108DB01CA0112E0880F991FAA1FBB1F1A9525
:20174000D1F7480F591F6A1F7B1F440F551F661F771F4E0F511D611D711D483929E952072A
:2017600029E9620729E1720748F084E0E82A06C0EE3F31F4E3FC39C098E0E92AF990C0CF2A
:20178000E53311F0E53189F529912D3219F4E0E1EE2A05C02B3219F081E090E003C0299124
:2017A00082E090E0E22FE053EA3018F0C81BD90B1CC020E030E0FCE020383F075CF4C901AA
:2017C000880F991F880F991F280F391F220F331F2E0F311DE991E053EA3068F3E4FE03C007
:2017E000309521953F4F820E931ECE2CDD24E1FE07C0A114B10421F02197F501D183C0833E
:20180000CB01BA010E9408957B018C01F3E0CF22DD2423E0C216D10421F417FB109517F9A8
:20182000109557016801C801B70120E030E040E050E00E946894882309F44AC097FE0DC0AF
:2018400024EBE22E25E1F22E9094819491089394C0E2D0E000E010E012C09CECE92E95E141
:20186000F92EF6CFF7012591359145915491C601B5010E9448975B016C018C1A9D0A8C1697
:201880009D0684F7D595C7950F5F1F4F0630110529F08CEF9FEFE80EF91EF1CFC501D601B0
:2018A0007C018D018C2D880F8D2D881F8F3F51F0C601B50120E030E040E050E00E946894E2
:2018C000882331F482E290E090933210809331107E2D9F2D802F612F272F392F482F562F3B
:2018E000B901CA01CDB7DEB7ECE00C94D8982F923F925F926F927F928F929F92AF92BF92F5
:20190000CF92DF92EF92FF920F931F93CF93DF938C011B01EA016115710519F0FB01918322
:201920008083209749F0CE010297839728F020E030E040E050E0F6C0F801A1908F018A2D93
:2019400090E00E94A398892BB9F7FDE2AF1631F4F801A1908F015524539407C0FBE2AF168A
:2019600019F4F801A1908F015524209719F0C031D105C1F4F0E3AF1679F4F801808188372D
:2019800011F0883549F4F801A1800E5F1F4FF2E05F2AC0E1D0E006C0209721F480E3A816F8
:2019A000E9F427C0C830D10531F1C930D10524F4C230D10531F50CC0CA30D10589F0C03198
:2019C000D105F9F4C12CD12CE12CB8E0FB2E28C0C12CD12CE12CA0E4FA2E22C0CAE0D0E0C5
:2019E000FCECCF2EFCECDF2EFCECEF2EFCE0FF2E17C0C8E0D0E0C12CD12CE12CE0E1FE2EEC
:201A00000FC09E01442737FD4095542F60E070E080E090E80E944C98C901DA016C017D01E3
:201A200020E030E040E050E060E03E01882477FC8094982C70EDB72EBA0CE9E0EB1570F49B
:201A40008A2D81548A3118F499ECB92E06C08A2D81568A3150F589EAB82EBA0C8B2D90E02C
:201A60008C179D0714F56F3FE1F0C216D306E406F506B0F0CA01B901A40193010E941A984F
:201A80009B01AC012B0D311D411D511D2130F0E03F07F0E04F07F0E85F0710F461E001C0DA
:201AA0006FEFF801A1908F01C5CF2114310481F0662331F001501040F1011183008308C083
:201AC00051FE1AC002501040F1011183008314C067FF12C050FC05C02FEF3FEF4FEF5FE745
:201AE00004C020E030E040E050E882E290E0909332108093311016C050FE08C05095409587
:201B0000309521953F4F4F4F5F4F0CC057FF0AC082E290E090933210809331102FEF3FEFAB
:201B20004FEF5FE7B901CA01DF91CF911F910F91FF90EF90DF90CF90BF90AF909F908F90C4
:201B40007F906F905F903F902F900895FB01DC0105900D920020E1F70895FB01DC01415051
:201B6000504088F08D9181341CF08B350CF4805E659161341CF06B350CF4605E861B6111D8
:201B800071F3990B0895881BFCCFFB0155915523A9F0BF01DC014D9145174111E1F759F4F1
:201BA000CD010590002049F04D9140154111C9F3FB014111EFCF81E090E001970895FB011A
:201BC000DC0104C08D910190801921F441505040C8F7881B990B0895FB01DC0102C0019017
:201BE0000D9241505040D8F70895FB01DC010D900020E9F7119701900D920020E1F70895D6
:201C0000FC018191861721F08823D9F7992708953197CF010895FB01DC0101900D920020D1
:201C2000E1F70895FB01DC014150504030F08D910190801919F40020B9F7881B990B08950C
:201C4000FB01DC014150504048F001900D920020C9F701C01D9241505040E0F70895AEE0AF
:201C6000B0E0E5E3FEE00C94C4980D891E898EE08C831A8309838FEF9FE79E838D839E017B
:201C8000275E3F4FCE0101966F89788DA9010AD02F813885020F131FF80110822E96E4E087
:201CA0000C94E098ABE0B0E0E8E5FEE00C94B6983C012B015A01FC0117821682838181FDE4
:201CC00003C06FEF7FEFB9C19AE0892E1E010894211C311CF3012381F20123FD859123FFA2
:201CE00081912F01882309F4A5C1853239F423FD859123FF81912F01853221F490E0B30126
:201D0000B7D1E8CF982FFF24EE249924FFE1FF15D0F09B3269F09C3228F4903259F0933237
:201D200091F40EC09D3249F0903369F441E024C052E0F52A84E0F82A28C098E0F92A25C0E4
:201D4000E0E1FE2A22C0F7FC29C0892F80538A3070F4F6FE05C0989C902C1124980E15C0DA
:201D6000E89CE02C1124E80EF0E2FF2A0EC09E3229F4F6FC5FC140E4F42A07C09C3619F4F8
:201D800050E8F52A02C0983649F4F20123FD959123FF91912F01992309F0B8CF892F8554A5
:201DA000833018F08052833038F444E050E0A40EB51E5FE359830FC0933631F0933779F0D4
:201DC000933509F052C01FC0F5018081898342E050E0A40EB51E610101E010E011C0F5017D
:201DE000C080D180F6FC03C06FEF7FEF02C0692D70E042E050E0A40EB51EC6012ED18C01FF
:201E00005FE7F52213C0F501C080D180F6FC03C06FEF7FEF02C0692D70E042E050E0A40EDE
:201E2000B51EC6010FD18C0150E8F52AF3FE06C018C080E290E0B3011BD1EA948E2D90E09A
:201E400008171907B0F30DC0F601F7FC8591F7FE81916F0190E0B3010BD1E110EA9401509C
:201E600010400115110581F7E2C0943611F0993661F5F7FE08C0F50120813181428153813F
:201E800084E090E00AC0F501808191819C01442737FD4095542F82E090E0A80EB91E9FE623
:201EA000F92257FF09C050954095309521953F4F4F4F5F4FE0E8FE2ACA01B901A1012AE0B8
:201EC00030E002D1D82ED2183FC0953729F41F2D1F7E2AE030E01DC01F2D197F9F3661F05D
:201EE000903720F4983509F0A5C00FC0903739F0983709F09FC004C028E030E00AC01061DF
:201F000014FD146020E130E004C014FD166020E132E017FF08C0F50160817181828193810F
:201F200044E050E008C0F50180819181BC0180E090E042E050E0A40EB51EA101C5D0D82EDB
:201F4000D2188FE7F82EF122F6FE0BC05EEFF522D91438F4F4FE07C0F2FC05C08FEEF822A9
:201F600002C01D2D01C0192DF4FE0DC0FE01ED0DF11D8081803319F499EEF92208C01F5FDF
:201F8000F2FE05C003C08F2D867809F01F5F0F2DF3FC13C0F0FE0EC01E1510F09D2C0AC018
:201FA0009D2C9E0C911A1E2D05C080E290E0B3015FD01F5F1E15C8F304C01E1510F4E11ADC
:201FC00001C0EE2404FF0EC080E390E0B30150D002FF1BC001FD03C088E790E00EC088E5FF
:201FE00090E00BC0802F867881F001FF02C08BE201C080E2F7FC8DE290E0B30139D005C0E2
:2020000080E390E0B30134D09A94D914C8F3DA94F101ED0DF11D808190E0B30129D0DD20DC
:20202000B1F705C080E290E0B30122D0EA94EE20C9F750CEF30166817781CB012B96E2E12E
:202040000C94D298FC010590615070400110D8F7809590958E0F9F1F0895FC016150704013
:2020600001900110D8F7809590958E0F9F1F08950F931F93CF93DF938C01EB018B8181FF90
:202080001BC082FF0DC02E813F818C819D812817390764F4E881F9810193F983E88306C082
:2020A000E885F985802F0995892B31F48E819F8101969F838E8302C00FEF1FEFC801DF910F
:2020C000CF911F910F910895FA01AA27283051F1203181F1E8946F936E7F6E5F7F4F8F4FA6
:2020E0009F4FAF4FB1E03ED0B4E03CD0670F781F891F9A1FA11D680F791F8A1F911DA11D65
:202100006A0F711D811D911DA11D20D009F468943F912AE0269F11243019305D3193DEF683
:20212000CF010895462F4770405D4193B3E00FD0C9F7F6CF462F4F70405D4A3318F0495DA2
:2021400031FD4052419302D0A9F7EACFB4E0A6959795879577956795BA95C9F70097610595
:20216000710508959B01AC010A2E06945795479537952795BA95C9F7620F731F841F951F78
:20218000A01D0895DF93CF930F92CDB7DEB7FC016983A081B18114962D913C911597BE017B
:2021A0006F5F7F4F41E050E0F90109950F90CF91DF910895FC0111AA14AA27E233E030AB21
:2021C00027A7E05BFF4F1082339610823597318320837F9610823396108235973183208373
:2021E0007F961082339610823597318320837E9689E18083339610827896108239961082DD
:20220000339610823597318320837D96108211821282138238961082118212821382ED5E78
:20222000F0401282138210821182EF50FF4F81E08083E15FF04016A615A60FB6F8948091E6
:202240001F1090912010A0912110B09122100FBEE751FF4F88579C4EAF4FBF4F80839183EA
:20226000A283B3830895FC01128213820895FC018381882311F081E082830895FC018281F3
:20228000811112820895FC0187E293E0918380838581882321F0CF0102960C94F7600895CD
:2022A0000F931F93CF93DF938C010E94616E0E943E6EC80186539F4F0E94F760F801128294
:2022C00083EE90E00E943D468091E006882301F11092E00680919A04C82FD0E0CC0FDD1FAF
:2022E000C05ED14F68817981882777FD8095982F0E940A9520918C0230918D0240918E028D
:2023000050918F020E947696181614F419821882DF91CF911F910F910895EF92FF920F93C1
:202320001F938C013AECE32EF12CE80EF91EC7010E94A960C7010E94F760F80110821182AB
:202340001F910F91FF90EF900895CF92DF92EF92FF920F931F93CF93DF937C016B01DB01B1
:202360000D900020E9F78D0101501040061B170BEAECF0E0EE0EFF1ED7011C92E6E3FFEF52
:20238000EE0EFF1ECB016EE470E03ADCEC01009731F4F8013197EC0DFD1D86010CC060E28E
:2023A00070E02EDC8C010F5F1F4FCE016AE270E027DCFC0131978DE081838AE082831382B2
:2023C000C70188539F4FB8010E94C2688AEC90E0E80EF91ED7018C918823F1F0EDE1F1E0D4
:2023E0006491EF0106C088E290E1CCDE2196FE0164916623C1F7E4E2F1E06491EF0106C07F
:2024000088E290E1BFDE2196FE0164916623C1F788E290E16AE0B6DEDF91CF911F910F917F
:20242000FF90EF90DF90CF900895EF92FF920F93CF93DF937C01FC018381882309F43DC078
:20244000ECE4F1E06491EF0106C088E290E19ADE2196FE0164916623C1F78DEE90E0E80E10
:20246000F91EF701408151816281738183E19FEFE80EF91E88E290E12AE000E00E945E908F
:20248000EAE4F1E06491EF0106C088E290E17ADE2196FE0164916623C1F785EE90E0E80EFA
:2024A000F91EF701408151816281738188E290E12AE000E00E945E900DC0EAE3F1E06491EE
:2024C000EF0106C088E290E15DDE2196FE0164916623C1F788E290E16AE054DEDF91CF911D
:2024E0000F91FF90EF9008952F923F924F925F926F927F928F929F92AF92BF92CF92DF9265
:20250000EF92FF920F931F93DF93CF93CDB7DEB7AB970FB6F894DEBF0FBECDBF5C014B0136
:202520004BA7FC018381882309F4C9C15AEC452E512C4A0C5B1CC2010E94F760F50112822D
:20254000188A1B8A87E293E09F878E874CE4C42ED12CCA0CDB1C2FE230E0A20EB31EF60198
:20256000B182A08221ED3FEFA20EB31EF40180818F3209F083C0C4016FE270E041DB7C0157
:202580000894E11CF11C3E010894611C711C160170C0C7016FE270E033DB6C01009709F4F1
:2025A0007BC0E816F90608F077C08C010E191F09C301B701A80144DB060D171DF8011082C2
:2025C000E0912810F09129100280F381E02D88E290E1B301099588E290E16AE0D3DDF101A1
:2025E000608171816115710519F460E070E002C06E5F7F4FCE014096A30121E00E94C96706
:20260000882361F5E0E0F2E064917F0108C088E290E1B8DD0894E11CF11CF701649166235E
:20262000B1F7E0912810F09129100280F381E02D88E290E1BE016F5F7F4F0995EEEFF1E00A
:2026400064917F0108C088E290E19CDD0894E11CF11CF70164916623B1F72AC12EE030E01C
:202660002C0F3D1FF1013183208376010894E11CF11CE114F10409F08CCF0BC08EE490E072
:20268000A80EB91EF601B182A08222EB3FEFA20EB31E082DD92C02C00E2DDF2CF501E45B2E
:2026A000FF4F3BA5332309F4A9C0608171816115710519F460E070E002C06E5F7F4FC201B4
:2026C000402F5D2D21E00E94C967882309F46BC0A5014B515F4F8BED90E0A80EB91EF50100
:2026E00080819181A281B38125E23FEFA20EB31EFA0180839183A283B383E0EFF1E06491B8
:202700007F0108C088E290E13DDD0894E11CF11CF70164916623B1F7E0912810F091291055
:202720000280F381E02D88E290E1602F7D2D0995E8EEF1E064917F0108C088E290E122DD26
:202740000894E11CF11CF70164916623B1F725EE30E0A20EB31EF5014081518162817381B1
:2027600088E290E12AE000E00E945E9088E290E16AE008DD28E030E0A20EB31EF5011082D9
:20278000118212821382EAEDF1E064917F0108C088E290E1F7DC0894E11CF11CF701649157
:2027A0006623B1F785C0E6ECF1E064917F0108C088E290E1E7DC0894E11CF11CF701649192
:2027C0006623B1F7E0912810F09129100280F381E02D88E290E1602F7D2D0995E4ECF1E00F
:2027E00064917F0108C088E290E1CCDC0894E11CF11CF70164916623B1F75AC06081718168
:202800006115710519F460E070E002C06E5F7F4FC201402F5D2D26E50E94C967882359F540
:20282000E0EBF1E064917F0108C088E290E1AADC0894E11CF11CF70164916623B1F7E09129
:202840002810F09129100280F381E02D88E290E1602F7D2D0995EEEAF1E064917F0108C0EB
:2028600088E290E18FDC0894E11CF11CF70164916623B1F71DC081E0F5018083ECE9F1E071
:2028800064917F0108C088E290E17CDC0894E11CF11CF70164916623B1F7E0912810F091DA
:2028A00029100280F381E02D88E290E1B401099588E290E16AE066DCCE010E96E4DCAB96D3
:2028C0000FB6F894DEBF0FBECDBFCF91DF911F910F91FF90EF90DF90CF90BF90AF909F90F8
:2028E0008F907F906F905F904F903F902F900895FC0181E08183CF0140E0F6CD2F923F920B
:202900004F925F926F927F928F929F92AF92BF92CF92DF92EF92FF920F931F93DF93CF93E3
:20292000CDB7DEB7AA970FB6F894DEBF0FBECDBF5C014B01FC018381882309F426C1C501F7
:2029400086539F4F0E94F760F5011282188A1B8A87E293E09F878E877CE4C72ED12CCA0CA7
:20296000DB1C2FE230E0A20EB31EF601B182A08221ED3FEFA20EB31EF40180818F3209F005
:2029800087C0C4016FE270E03BD97C010894E11CF11C3E010894611C711C260160E1262EB2
:2029A000312C2C0E3D1E6FC0C7016FE270E028D96C01009709F47AC0E816F90608F076C026
:2029C0008C010E191F09C301B701A80139D9060D171DF8011082E0912810F091291002802D
:2029E000F381E02D88E290E1B301099588E290E16AE0C8DBF201608171816115710519F4A2
:202A000060E070E002C06E5F7F4FC101A30121E00E94C967882361F5E8E8F1E064917F0179
:202A200008C088E290E1AEDB0894E11CF11CF70164916623B1F7E0912810F09129100280C1
:202A4000F381E02D88E290E1BE016F5F7F4F0995E6E8F1E064917F0108C088E290E192DBFD
:202A60000894E11CF11CF70164916623B1F786C02EE030E02C0F3D1FF201318320837601D6
:202A80000894E11CF11CE114F10409F08DCF0BC08EE490E0A80EB91EF601B182A08222EBBE
:202AA0003FEFA20EB31ED82C092D02C0DE2C0F2D8CE490E0A80EB91EF5018081918124EBA0
:202AC0003FEFA20EB31E009719F480E090E001C002966D2D702F0E949568882329F1E8E70E
:202AE000F1E064917F0108C088E290E14BDB0894E11CF11CF70164916623B1F7E09128105A
:202B0000F09129100280F381E02D88E290E16D2D702F09952DEE30E0A20EB31EF501108212
:202B20001182128213822EC0E0E6F1E064917F0108C088E290E126DB0894E11CF11CF7019D
:202B400064916623B1F7E0912810F09129100280F381E02D88E290E16D2D702F0995EEE564
:202B6000F1E064917F0108C088E290E10BDB0894E11CF11CF70164916623B1F788E290E1E7
:202B80006AE000DBCE010E967EDBAA960FB6F894DEBF0FBECDBFCF91DF911F910F91FF900E
:202BA000EF90DF90CF90BF90AF909F908F907F906F905F904F903F902F900895EF92FF92D3
:202BC0000F931F93CF93DF937C01FC01138284A9882321F0C701C1960E94F76087010B55D5
:202BE0001F4FC80160E048E00E94C15E8823D9F4EDEEF0E06491EF0106C088E290E1C2DA30
:202C00002196FE0164916623C1F7E2E4F2E06491EF0106C088E290E1B5DA2196FE01649170
:202C20006623C1F76BC0E701C655DF4FCE01B80141E00E945369882311F5CE01B80140E097
:202C40000E9453698823D9F4EDE1F1E06491EF0106C088E290E196DA2196FE0164916623D5
:202C6000C1F7EFE2F2E06491EF0106C088E290E189DA2196FE0164916623C1F73FC0C7015D
:202C8000C196BE010E94CE638823D9F4EDE1F1E06491EF0106C088E290E174DA2196FE01AA
:202CA00064916623C1F7EFE1F2E06491EF0106C088E290E167DA2196FE0164916623C1F789
:202CC0001DC081E0F7018383EDEEF0E06491EF0106C088E290E156DA2196FE016491662323
:202CE000C1F7E4E1F2E06491EF0106C088E290E149DA2196FE0164916623C1F788E290E115
:202D00006AE040DAD701A05BBF4FF701F1968BE101900D928150E1F7C7018F962CE430E09D
:202D2000E20EF31EF70191838083DF91CF911F910F91FF90EF9008952F923F924F925F9254
:202D40006F927F929F92AF92BF92CF92DF92EF92FF920F931F93DF93CF93CDB7DEB7CC5558
:202D6000D0400FB6F894DEBF0FBECDBF8C01662319F50F501F4FD8018C91015F10408823BA
:202D800009F4E6C00FB6F89420911F103091201040912110509122100FBE07511F4FF801CD
:202DA00080819181A281B381095E104082179307A407B50708F4CCC00F501F4FD8011C927C
:202DC000015F1040F8018381882341F4C801F6DED80113968C91882309F4BAC000D000D068
:202DE00000D0EDB7FEB731966E010894C11CD11CADB7BEB71296DC92CE92119784E191E041
:202E000093838283D8019D968D919C919E97958384830E942F0E7601EDB7FEB736960FB6AC
:202E2000F894FEBF0FBEEDBF56010AC0D7018C91992787FD90950E94AB98F70181937F01E0
:202E4000F50101900020E9F73197EA19FB098E2D8C198E175CF3B1E3AB2EB12CA00EB11E01
:202E6000C50140E050E060E070E00E94DF5F9924ADE3CA2ED12CCC0EDD1E2E010894411C8D
:202E8000511CFFE16F2E712C6C0E7D1EEDE02E2EE1E03E2E43C0D7018C9190E00E94AB98F3
:202EA000F70181937F01D6010D900020E9F71197AC19BD098E2D8C198A176CF327968FAD86
:202EC00027978E3759F1C601B20145E050E00E94120E009719F500D000D000D0EDB7FEB726
:202EE0003196ADB7BEB712967C926E92119733822282558244820E942F0EEDB7FEB73696DA
:202F00000FB6F894FEBF0FBEEDBFC3010E94B44689E091E00E943D4699249394C501B6016A
:202F200040E050E00E94ED62181614F47601BBCF992041F48FEF9FEFD8019E969C938E93C2
:202F40009D9706C0F80185A596A5019696A785A7C45ADF4F0FB6F894DEBF0FBECDBFCF9126
:202F6000DF911F910F91FF90EF90DF90CF90BF90AF909F907F906F905F904F903F902F908E
:202F800008952F923F924F925F926F927F928F929F92AF92BF92CF92DF92EF92FF920F93B4
:202FA0001F93DF93CF93CDB7DEB7CB58D0400FB6F894DEBF0FBECDBF7C012B015A0182E092
:202FC00090E0A80EB91EF7017196CB57DF4FF983E883C558D040C7010496CE57DF4F9983C0
:202FE0008883C258D040CC57DF4F1882C458D04092E6C92ED12CCC0EDD1EF6013B96C9575C
:20300000DF4FF983E883C758D04082EF682E712C6E0C7F1C04EF802E912C8E0C9F1C1EE002
:20302000212E312C2C0E3D1E85E490E08C0F9D1F0296C757DF4F99838883C958D040EDEE08
:20304000F0E09491C557DF4F9883CB58D0403EC1F6018385482F50E0BA0168717070603139
:20306000710509F041C1F301208131812130310509F43AC12230310509F436C1F601DE01C7
:2030800011969081903239F08E2F8C19883011F48EE28D939D933196C957DF4F8881998176
:2030A000C758D040E817F90761F71C921E86F2018081882329F4C10160E071E00E94F50D85
:2030C000C101B2010E94F50DC101BE016F5F7F4F0E94F50DC10160E071E00E94F50D1AA65F
:2030E0001DA687E293E099A788A7CE018A96B501AE014F5F5F4F21E00E94C9678823B9F5E6
:20310000F30180819181892B91F5C557DF4F6881CB58D0400DEE10E007C088E290E132D871
:203120000F5F1F4FF80164916623B9F7E0912810F09129100280F381E02D88E290E162E009
:2031400071E0099588E290E16AE01CD8E0912810F09129100280F381E02D88E290E1BE0167
:203160006F5F7F4F099588E290E16AE00BD8C757DF4FA881B981C958D040FE01BA968BE172
:2031800001900D928150E1F787E293E027969FAF8EAF2797C701B101AE014B5B5F4FF1DE28
:2031A000CE018B5B9F4F6FD8CE0188966CD88EC0953E09F48BC09E3209F488C09F3509F4A5
:2031C00085C0F7019189992331F09E3209F47EC09F3509F47BC043FD79C080E060317105C4
:2031E00009F481E0F70184A7882349F4F6018085873409F06BC081858E3709F467C0CE5777
:20320000DF4FA881B981C258D040F6018081803241F08E2F8C19883011F48EE28D93808168
:203220008D933196C957DF4F88819981C758D040E817F90759F71C92F3018081918100976C
:2032400009F5E0912810F09129100280F381E02D88E290E1B2010995E0912810F09129107B
:203260000280F381E02D88E290E1CE57DF4F68817981C258D040099588E290E16AE00E94AB
:20328000C21024C08130910539F4F401808191810196918380831AC00297C1F4CC57DF4FD5
:2032A000F881C458D0402F2F30E0F4018081918128173907F1F0CC57DF4FF881C458D0409D
:2032C000FF5FCC57DF4FF883C458D040C501B601CB57DF4F48815981C558D0400E94ED620A
:2032E00018160CF4B5CE05C0F6019081992309F05FCFC557DF4F0FB6F894DEBF0FBECDBFDC
:20330000CF91DF911F910F91FF90EF90DF90CF90BF90AF909F908F907F906F905F904F90F9
:203320003F902F900895EF92FF920F931F93DF93CF93CDB7DEB76D970FB6F894DEBF0FBE50
:20334000CDBF7C0182EF90E0E80EF91EF701118210828EE09FEFE80EF91E87010F5C1F4FEF
:20336000C80140E050E060E070E00E94DF5FDE011396F8018BE101900D928150E1F787E295
:2033800093E09A838983C70165E171E08E010F5F1F4FA801F6DDC8010E9443116D960FB6C4
:2033A000F894DEBF0FBECDBFCF91DF911F910F91FF90EF9008950F931F93DF93CF93CDB714
:2033C000DEB7E0970FB6F894DEBF0FBECDBFDE011196E7EDF2E080E101900D928150E1F734
:2033E000DE015196E7ECF2E080E101900D928150E1F7DE019196E7EBF2E080E101900D92ED
:203400008150E1F789819A81AB81BC818093840690938506A0938606B093870689899A8966
:20342000AB89BC898093740690937506A0937606B093770689A19AA1ABA1BCA180939406BE
:2034400090939506A0939606B09397068D819E81AF81B8858093880690938906A0938A064F
:20346000B0938B068D899E89AF89B88D8093780690937906A0937A06B0937B068DA19EA1A7
:20348000AFA1B8A58093980690939906A0939A06B0939B0689859A85AB85BC8580938C0612
:2034A00090938D06A0938E06B0938F06898D9A8DAB8DBC8D80937C0690937D06A0937E0607
:2034C000B0937F0689A59AA5ABA5BCA580939C0690939D06A0939E06B0939F068D859E8597
:2034E000AF85B8898093900690939106A0939206B09393068D8D9E8DAF8DB8A180938006DA
:2035000090938106A0938206B09383068DA59EA5AFA5B8A98093A0069093A106A093A206F2
:20352000B093A3060E942B4C80E090E0AAE7B4E48093A8069093A906A093AA06B093AB0623
:2035400080E090E8ABE3B5E48093AC069093AD06A093AE06B093AF0620E030E040E050E092
:203560002093A4063093A5064093A6065093A70680E29EE4A0E0B0E080937006909371065A
:20358000A0937206B09373062093BC063093BD064093BE065093BF0680E090E0A0E2B1E4A3
:2035A0008093B0069093B106A093B206B093B3068DEC9CECACECBEE38093B4069093B5069C
:2035C000A093B606B093B70680E090E0A0EAB0E48093B8069093B906A093BA06B093BB0664
:2035E00020938A0430938B0440938C0450938D042093860430938704409388045093890407
:20360000209382043093830440938404509385048AE999E9A1EBB1E48093990290939A02DD
:20362000A0939B02B0939C0261E77DE38AE89FE30E94B57560939D0270939E0280939F0288
:203640009093A00260E070E084EE92E40E94C1756093A1027093A2028093A3029093A40297
:2036600082E493E060E070E020E030E040E050E00E94962482E493E061E070E020E030E0AB
:2036800040E050E00E94962482E493E062E070E020E030E040E050E00E9496240E948475BC
:2036A00080E090E0A0E8BFE38093A5029093A602A093A702B093A802EFE4F2E064918F0198
:2036C00008C088E290E10E94C2100F5F1F4FF80164916623B1F7E5E5F2E064918F0108C0EF
:2036E00088E290E10E94C2100F5F1F4FF80164916623B1F788E290E16AE00E94C210E09671
:203700000FB6F894DEBF0FBECDBFCF91DF911F910F9108950F931F93CF93DF930FE412E098
:20372000F8016491E80107C088E290E10E94C2102196FE0164916623B9F7E8E6F4E0649121
:20374000EF0107C088E290E10E94C2102196FE0164916623B9F788E290E16AE00E94C210E6
:20376000F8016491CFE4D2E007C088E290E10E94C2102196FE0164916623B9F740918406A1
:2037800050918506609186067091870680E694E00E94582E409188065091890660918A0660
:2037A00070918B068DE594E00E94582E40918C0650918D0660918E0670918F068AE594E094
:2037C0000E94582E4091900650919106609192067091930687E594E00E94582EE09128100E
:2037E000F09129100280F381E02D88E290E166E171E0099588E290E16AE00E94C210F80169
:203800006491CFE4D2E007C088E290E10E94C2102196FE0164916623B9F7EDE3F4E06491BB
:20382000EF0107C088E290E10E94C2102196FE0164916623B9F788E290E16AE00E94C21005
:20384000F8016491CFE4D2E007C088E290E10E94C2102196FE0164916623B9F740917406D0
:2038600050917506609176067091770684E394E00E94582E409178065091790660917A06DE
:2038800070917B0681E394E00E94582E40917C0650917D0660917E0670917F068EE294E010
:2038A0000E94582E409180065091810660918206709183068BE294E00E94582EE09128106C
:2038C000F09129100280F381E02D88E290E166E171E0099588E290E16AE00E94C210F80188
:2038E0006491CFE4D2E007C088E290E10E94C2102196FE0164916623B9F7EDE0F4E06491DE
:20390000EF0107C088E290E10E94C2102196FE0164916623B9F788E290E16AE00E94C21024
:20392000F8016491CFE4D2E007C088E290E10E94C2102196FE0164916623B9F740919406CF
:2039400050919506609196067091970684E094E00E94342E409198065091990660919A0664
:2039600070919B0681E094E00E94342E40919C0650919D0660919E0670919F068EEF93E0AA
:203980000E94342E4091A0065091A1066091A2067091A3068BEF93E00E94342EE091281047
:2039A000F09129100280F381E02D88E290E166E171E0099588E290E16AE00E94C210F801A7
:2039C0006491CFE4D2E007C088E290E10E94C2102196FE0164916623B9F7E6ECF3E06491F9
:2039E000EF0107C088E290E10E94C2102196FE0164916623B9F788E290E16AE00E94C21044
:203A0000F8016491CFE4D2E007C088E290E10E94C2102196FE0164916623B9F74091A806DA
:203A20005091A9066091AA067091AB068DEB93E00E94582E4091AC065091AD066091AE06D4
:203A40007091AF068AEB93E00E94582EE0912810F09129100280F381E02D88E290E166E118
:203A600071E0099588E290E16AE00E94C210F8016491CFE4D2E007C088E290E10E94C21055
:203A80002196FE0164916623B9F7E7E0F3E06491EF0107C088E290E10E94C2102196FE01F7
:203AA00064916623B9F788E290E16AE00E94C210F8016491CFE4D2E007C088E290E10E94A8
:203AC000C2102196FE0164916623B9F74091A4065091A5066091A6067091A7068EEF92E0EF
:203AE0000E94582E4091BC065091BD066091BE067091BF068BEF92E00E94582E4091700691
:203B000050917106609172067091730688EF92E00E94342E4091B0065091B1066091B206B5
:203B20007091B30685EF92E00E94582E4091B4065091B5066091B6067091B70682EF92E048
:203B40000E94582E4091B8065091B9066091BA067091BB068FEE92E00E94582EE0912810DB
:203B6000F09129100280F381E02D88E290E166E171E0099588E290E16AE00E94C210F801E5
:203B80006491CFE4D2E007C088E290E10E94C2102196FE0164916623B9F7EDEDF2E0649130
:203BA000EF0107C088E290E10E94C2102196FE0164916623B9F788E290E16AE00E94C21082
:203BC000F8016491CFE4D2E007C088E290E10E94C2102196FE0164916623B9F74091820441
:203BE00050918304609184047091850484ED92E00E94582E4091860450918704609188040B
:203C00007091890481ED92E00E94582E40918A0450918B0460918C0470918D048EEC92E040
:203C20000E94582EE0912810F09129100280F381E02D88E290E166E171E0099588E290E10A
:203C40006AE00E94C210F8016491CFE4D2E007C088E290E10E94C2102196FE016491662309
:203C6000B9F7E0ECF2E06491EF0107C088E290E10E94C2102196FE0164916623B9F788E2AD
:203C800090E16AE00E94C210F8016491CFE4D2E007C088E290E10E94C2102196FE016491E1
:203CA0006623B9F74091990250919A0260919B0270919C0286EB92E00E94582E60919D021A
:203CC00070919E0280919F029091A0020E94BB75AB01BC0183EB92E00E94582E6091A102F7
:203CE0007091A2028091A3029091A4020E94C775AB01BC0180EB92E00E94582EE0912810AD
:203D0000F09129100280F381E02D88E290E166E171E0099588E290E16AE00E94C210F80143
:203D20006491CFE4D2E007C088E290E10E94C2102196FE0164916623B9F7EFE9F2E0649190
:203D4000EF0107C088E290E10E94C2102196FE0164916623B9F788E290E16AE00E94C210E0
:203D6000F8016491CFE4D2E007C088E290E10E94C2102196FE0164916623B9F782E493E01D
:203D800060E070E0C5D5AB01BC0187E992E00E94582E82E493E061E070E0BAD5AB01BC0124
:203DA00084E992E00E94582E82E493E062E070E0AFD5AB01BC0181E992E00E94582EE0912F
:203DC0002810F09129100280F381E02D88E290E166E171E0099588E290E16AE00E94C21044
:203DE000DF91CF911F910F9108950F931F93DF93CF93CDB7DEB7A0970FB6F894DEBF0FBED3
:203E0000CDBF8091170190911801A0911901B0911A01898B9A8BAB8BBC8BFE013D9604E69A
:203E200010E0F999FECF12BD01BDF89A80B580830F5F1F4F0836110511F03196F2CFCE0154
:203E40004196BE01635F7F4F43E050E00E94120E009709F0C1C1E4E8F6E0F999FECF12BD45
:203E600001BDF89A80B580830F5F1F4F0837110511F03196F2CFE4E7F6E0F999FECF12BD31
:203E800001BDF89A80B580830F5F1F4F0838110511F03196F2CFE4E9F6E0F999FECF12BD0E
:203EA00001BDF89A80B580830F5F1F4F0839110511F03196F2CF0E942B4CE8EAF6E0F9996B
:203EC000FECF12BD01BDF89A80B580830F5F1F4F0C39110511F03196F2CFECEAF6E0F999C0
:203EE000FECF12BD01BDF89A80B580830F5F1F4F003A110511F03196F2CFE4EAF6E0F999B3
:203F0000FECF12BD01BDF89A80B580830F5F1F4F043A110511F03196F2CFECEBF6E0F99985
:203F2000FECF12BD01BDF89A80B580830F5F1F4F083A110511F03196F2CFE0E7F6E0F99971
:203F4000FECF12BD01BDF89A80B580830F5F1F4F0C3A110511F03196F2CFE0EBF6E0F99949
:203F6000FECF12BD01BDF89A80B580830F5F1F4F003B110511F03196F2CFE4EBF6E0F99930
:203F8000FECF12BD01BDF89A80B580830F5F1F4F043B110511F03196F2CFE8EBF6E0F99908
:203FA000FECF12BD01BDF89A80B580830F5F1F4F083B110511F03196F2CFE2E8F4E0F999EF
:203FC000FECF12BD01BDF89A80B580830F5F1F4F043C110511F03196F2CFFE013196F999AA
:203FE000FECF12BD01BDF89A80B580830F5F1F4F063C110599F7FE013396F999FECF12BDE3
:2040000001BDF89A80B580830F5F1F4F083C110511F03196F2CFFE013596F999FECF12BD61
:2040200001BDF89A80B580830F5F1F4F0A3C110511F03196F2CFFE013796F999FECF12BD3D
:2040400001BDF89A80B580830F5F1F4F0C3C110511F03196F2CFFE013996F999FECF12BD19
:2040600001BDF89A80B580830F5F1F4F0E3C110511F03196F2CFFE013B96F999FECF12BDF5
:2040800001BDF89A80B580830F5F1F4F003D110511F03196F2CFE9E9F2E0F999FECF12BD0E
:2040A00001BDF89A80B580830F5F1F4F043D110511F03196F2CFEDE9F2E0F999FECF12BDE6
:2040C00001BDF89A80B580830F5F1F4F083D110511F03196F2CFE1EAF2E0F999FECF12BDCD
:2040E00001BDF89A80B580830F5F1F4F0C3D110511F03196F2CF0E948475FE017596F9993D
:20410000FECF12BD01BDF89A80B580830F5F1F4F003E110511F03196F2CFFE017996F99922
:20412000FECF12BD01BDF89A80B580830F5F1F4F043E110511F03196F2CFFE017D96F999FA
:20414000FECF12BD01BDF89A80B58083073E110521F00F5F1F4F3196F2CF2D893E894F8916
:20416000588D82E493E060E070E0E0D3298D3A8D4B8D5C8D82E493E061E070E0D7D32D8D32
:204180003E8D4F8D58A182E493E062E070E0CED3EFE4F2E064918F0108C088E290E10E9404
:2041A000C2100F5F1F4FF80164916623B1F7E7E7F2E064918F0108C088E290E10E94C210F6
:2041C0000F5F1F4FF80164916623B1F788E290E16AE00E94C21001C0EED89CDAA0960FB653
:2041E000F894DEBF0FBECDBFCF91DF911F910F9108950F931F93DF93CF93CDB7DEB7A09708
:204200000FB6F894DEBF0FBECDBF80911B0190911C01A0911D01B0911E018D879E87AF87CE
:20422000B88BFE013D9604E610E08081F999FECF1FBA12BD01BD80BD0FB6F894FA9AF99A14
:204240000FBE0F5F1F4F0836110511F03196EDCFE4E8F6E08081F999FECF1FBA12BD01BD75
:2042600080BD0FB6F894FA9AF99A0FBE0F5F1F4F0837110511F03196EDCFE4E7F6E0808165
:20428000F999FECF1FBA12BD01BD80BD0FB6F894FA9AF99A0FBE0F5F1F4F0838110511F0A4
:2042A0003196EDCFE4E9F6E08081F999FECF1FBA12BD01BD80BD0FB6F894FA9AF99A0FBE90
:2042C0000F5F1F4F0839110511F03196EDCFE8EAF6E08081F999FECF1FBA12BD01BD80BD7C
:2042E0000FB6F894FA9AF99A0FBE0F5F1F4F0C39110511F03196EDCFECEAF6E08081F9997F
:20430000FECF1FBA12BD01BD80BD0FB6F894FA9AF99A0FBE0F5F1F4F003A110511F03196F4
:20432000EDCFE4EAF6E08081F999FECF1FBA12BD01BD80BD0FB6F894FA9AF99A0FBE0F5F67
:204340001F4F043A110511F03196EDCFECEBF6E08081F999FECF1FBA12BD01BD80BD0FB6A2
:20436000F894FA9AF99A0FBE0F5F1F4F083A110511F03196EDCFE0E7F6E08081F999FECF08
:204380001FBA12BD01BD80BD0FB6F894FA9AF99A0FBE0F5F1F4F0C3A110511F03196EDCF79
:2043A000E0EBF6E08081F999FECF1FBA12BD01BD80BD0FB6F894FA9AF99A0FBE0F5F1F4F38
:2043C000003B110511F03196EDCFE4EBF6E08081F999FECF1FBA12BD01BD80BD0FB6F8940F
:2043E000FA9AF99A0FBE0F5F1F4F043B110511F03196EDCFE8EBF6E08081F999FECF1FBA32
:2044000012BD01BD80BD0FB6F894FA9AF99A0FBE0F5F1F4F083B110511F03196EDCFE2E80A
:20442000F4E08081F999FECF1FBA12BD01BD80BD0FB6F894FA9AF99A0FBE0F5F1F4F043C44
:20444000110511F03196EDCF80EA90E09A83898386E490E09C838B832FEF30E03E832D8319
:204460008EEB90E098878F838AE590E09A8789873C872B87FE0131968081F999FECF1FBA9E
:2044800012BD01BD80BD0FB6F894FA9AF99A0FBE0F5F1F4F063C110571F7FE0133968081A8
:2044A000F999FECF1FBA12BD01BD80BD0FB6F894FA9AF99A0FBE0F5F1F4F083C110511F07E
:2044C0003196EDCFFE0135968081F999FECF1FBA12BD01BD80BD0FB6F894FA9AF99A0FBE47
:2044E0000F5F1F4F0A3C110511F03196EDCFFE0137968081F999FECF1FBA12BD01BD80BD31
:204500000FB6F894FA9AF99A0FBE0F5F1F4F0C3C110511F03196EDCFFE0139968081F99937
:20452000FECF1FBA12BD01BD80BD0FB6F894FA9AF99A0FBE0F5F1F4F0E3C110511F03196C2
:20454000EDCFFE013B968081F999FECF1FBA12BD01BD80BD0FB6F894FA9AF99A0FBE0F5F19
:204560001F4F003D110511F03196EDCFE9E9F2E08081F999FECF1FBA12BD01BD80BD0FB68A
:20458000F894FA9AF99A0FBE0F5F1F4F043D110511F03196EDCFEDE9F2E08081F999FECFDC
:2045A0001FBA12BD01BD80BD0FB6F894FA9AF99A0FBE0F5F1F4F083D110511F03196EDCF58
:2045C000E1EAF2E08081F999FECF1FBA12BD01BD80BD0FB6F894FA9AF99A0FBE0F5F1F4F1A
:2045E0000C3D110511F03196EDCF82E493E060E070E08ED1698B7A8B8B8B9C8B82E493E001
:2046000061E070E085D16D8B7E8B8F8B988F82E493E062E070E07CD1698F7A8F8B8F9C8F73
:20462000FE0171968081F999FECF1FBA12BD01BD80BD0FB6F894FA9AF99A0FBE0F5F1F4F50
:20464000003E110511F03196EDCFFE0175968081F999FECF1FBA12BD01BD80BD0FB6F89424
:20466000FA9AF99A0FBE0F5F1F4F043E110511F03196EDCFFE0179968081F999FECF1FBA47
:2046800012BD01BD80BD0FB6F894FA9AF99A0FBE073E110521F00F5F1F4F3196EDCF80912F
:2046A000170190911801A0911901B0911A018D8F9E8FAF8FB8A3FE017D9684E690E0208192
:2046C000F999FECF1FBA92BD81BD20BD0FB6F894FA9AF99A0FBE8736910519F00196319639
:2046E000EECFEFE4F2E064918F0108C088E290E10E94C2100F5F1F4FF80164916623B1F7C1
:20470000E8E7F4E064918F0108C088E290E10E94C2100F5F1F4FF80164916623B1F788E2F5
:2047200090E16AE00E94C210A0960FB6F894DEBF0FBECDBFCF91DF911F910F9108952F924F
:204740003F924F925F926F927F928F929F92AF92BF92CF92DF92EF92FF920F931F93DF9316
:20476000CF93CDB7DEB73C011A012B01C901B801F30120823182428253820483158326830D
:204780003783C086D186E286F38684869586A686B78620E030E040E050E00E9468948823AA
:2047A00011F410E001C012E0F301608571858285938520E030E040E050E00E9468948823BA
:2047C00011F4EE2402C094E0E92EC501B40120E030E040E050E00E946894882311F4FF2429
:2047E00002C088E0F82E00E0C201B10120E030E040E050E00E946894811101E0102B1E2921
:204800001F29F30111A36081718182819381209184063091850640918606509187060E94CA
:2048200048970E94D794F301608B718B828B938B64817581868197812091880630918906FD
:2048400040918A0650918B060E9448970E94D794F301648B758B868B978B608571858285FF
:20486000938520918C0630918D0640918E0650918F060E9448970E94D794F301608F718F3D
:20488000828F938F6485758586859785209190063091910640919206509193060E944897D8
:2048A0000E94D794F301648F758F868F978FCF91DF911F910F91FF90EF90DF90CF90BF907A
:2048C000AF909F908F907F906F905F904F903F902F9008958F929F92AF92BF92CF92DF928E
:2048E000EF92FF920F931F93DF93CF93CDB7DEB7FC0110A224DFCF91DF911F910F91FF9004
:20490000EF90DF90CF90BF90AF909F908F900895FB01EE0FFF1FEE0FFF1FE80FF91F2081EF
:20492000318142815381B901CA0108950F931F93CF93DF93EC018B01FB01EE0FFF1FEE0F57
:20494000FF1FE80FF91F2083318342835383CA01B90120E030E040E050E00E94689429A1EB
:20496000882309F45EC081E090E002C0880F991F0A95E2F7282B29A3688179818A819B81EE
:20498000209184063091850640918606509187060E9448970E94D794688B798B8A8B9B8B05
:2049A0006C817D818E819F81209188063091890640918A0650918B060E9448970E94D794ED
:2049C0006C8B7D8B8E8B9F8B688579858A859B8520918C0630918D0640918E0650918F0609
:2049E0000E9448970E94D794688F798F8A8F9B8F6C857D858E859F8520919006309191061E
:204A000040919206509193060E9448970E94D7946C8F7D8F8E8F9F8FDF91CF911F910F91B3
:204A2000089581E090E002C0880F991F0A95E2F780952823A0CFCF93DF93EC01FB0160E0B3
:204A4000208131814281538188819981AA81BB81281739074A075B070CF461E02481358114
:204A6000468157818C819D81AE81BF81281739074A075B070CF4626020853185428553850F
:204A800088859985AA85BB85281739074A075B070CF4646024853585468557858C859D8549
:204AA000AE85BF85281739074A075B070CF46860862FDF91CF910895CF93DF93EC01FB01A6
:204AC00060E0208131814281538188819981AA81BB81281739074A075B0709F061E0248111
:204AE0003581468157818C819D81AE81BF81281739074A075B0709F06260208531854285B8
:204B0000538588859985AA85BB85281739074A075B0709F0646024853585468557858C8519
:204B20009D85AE85BF85281739074A075B0709F06860862FDF91CF9108952F923F924F9254
:204B40005F926F927F928F929F92AF92BF92CF92DF92EF92FF920F931F93DF93CF93CDB7DE
:204B6000DEB765970FB6F894DEBF0FBECDBF1C01FB017A01690158018E010F5F1F4F80E13A
:204B8000D8011D928A95E9F760817181828193812091840630918506409186065091870652
:204BA0000E9448970E94D79469837A838B839C83F70160817181828193812091880630916F
:204BC000890640918A0650918B060E9448970E94D7946D837E838F839887D6016D917D91E0
:204BE0008D919C9120918C0630918D0640918E0650918F060E9448970E94D79469877A8779
:204C00008B879C87F5016081718182819381209190063091910640919206509193060E945B
:204C200048970E94D7946D877E878F87988B80ED96E0B80100DF482E80ED96E0B8013CDFAE
:204C4000582ED1019096BC91B98B8B2F84258521282F30E0F10181A190E082239323892B42
:204C600009F465C0E0ED8E2EE6E09E2E74E6A72E73E0B72E3101CC24DD243B8B2A8B842D41
:204C800090E09D8B8C8B8A899B890C2C02C0959587950A94E2F780FF3AC08C899D890C2C8B
:204CA00002C0959587950A94E2F7D3015096ED90FD900D911C91539780FF08C02227332792
:204CC000A9012E193F09400B510B02C0A8019701F40180819181A281B381821B930BA40BA8
:204CE000B50B80839183A283B383CA01B9010E940A959B01AC01D5016D917D918D919C9146
:204D00000E948F93F50160837183828393830894C11CD11C84E090E0880E991EA80EB91ED3
:204D2000680E791E94E0C916D10409F0ACCF852D8095A9898A2354208529F10180A36596F2
:204D40000FB6F894DEBF0FBECDBFCF91DF911F910F91FF90EF90DF90CF90BF90AF909F9053
:204D60008F907F906F905F904F903F902F9008958F929F92AF92BF92CF92DF92EF92FF9245
:204D80000F931F9382E493E040E050E060E070E08A019B016A017B014A015B019BDD1F9129
:204DA0000F91FF90EF90DF90CF90BF90AF909F908F900895CF92DF92EF92FF920F931F93C6
:204DC000DF93CF930F92CDB7DEB77C01E8EAF4E084918F016E010894C11CD11C0CC08983D0
:204DE00088E290E1B60141E050E00E9428920F5F1F4FF8018491882391F7F70140815181CC
:204E00006281738188E290E122E00E94FA90E5EAF4E084918F016E010894C11CD11C0CC0C9
:204E2000898388E290E1B60141E050E00E9428920F5F1F4FF8018491882391F7F70144814D
:204E400055816681778188E290E122E00E94FA90E2EAF4E084918F016E010894C11CD11C7A
:204E60000CC0898388E290E1B60141E050E00E9428920F5F1F4FF8018491882391F7F70106
:204E8000408551856285738588E290E122E00E94FA90EFE9F4E084918F016E010894C11C56
:204EA000D11C0CC0898388E290E1B60141E050E00E9428920F5F1F4FF8018491882391F7D1
:204EC000F701448555856685778588E290E122E00E94FA90E4E9F4E084918F017E010894E6
:204EE000E11CF11C0CC0898388E290E1B70141E050E00E9428920F5F1F4FF80184918823FB
:204F000091F74091640350916503609166037091670388E290E122E00E94FA90E0E9F4E01D
:204F200084918F017E010894E11CF11C0CC0898388E290E1B70141E050E00E9428920F5F21
:204F40001F4FF8018491882391F7409168035091690360916A0370916B0388E290E122E06F
:204F60000E94FA90ECE8F4E084918F017E010894E11CF11C0CC0898388E290E1B70141E007
:204F800050E00E9428920F5F1F4FF8018491882391F740916C0350916D0360916E03709174
:204FA0006F0388E290E122E00E94FA90E8E8F4E084918F017E010894E11CF11C0CC0898330
:204FC00088E290E1B70141E050E00E9428920F5F1F4FF8018491882391F74091700350914F
:204FE0007103609172037091730388E290E122E00E94FA90E0912810F09129100280F381FE
:20500000E02D88E290E16FE171E009958AE0898388E290E1B70141E050E00E9428920F9014
:20502000CF91DF911F910F91FF90EF90DF90CF900895DC01ED91FC910280F381E02D09954E
:205040000895CF93DF930FB6F89480911F1090912010A0912110B09122100FBE8093AF0495
:205060009093B004A093B104B093B204E091D804F091D904E652FB4F8081882399F4EEE440
:20508000F5E06491EF0107C088E290E10E94C2102196FE0164916623B9F788E290E16AE037
:2050A0000E94C210DF91CF91089508958091A50408958130910541F46F5F7F4F09F051C0F9
:2050C00084E793E00C94DA10892B09F04AC06F5F7F4F09F046C087E293E090933D048093C3
:2050E0003C0480914104882321F08EE394E00E94F76087E293E09093FD038093FC0380915E
:205100000104882321F08EEF93E00E94F76087E293E09093E0038093DF038091E40388236B
:2051200021F081EE93E00E94F76087E293E09093C3038093C2038091C703882321F084ECDF
:2051400093E00E94F76087E293E09093A4038093A3038091A803882321F085EA93E00C948A
:20516000F760089580E090E06FEF7FEFA2CF81E090E06FEF7FEF9DCFCF93DF930E94A77593
:205180008091A504882309F034C081E08093A5048091A7049091A804A091A904B091AA044A
:2051A0008093AB049093AC04A093AD04B093AE04E2EBF4E06491EF0107C088E290E10E94B7
:2051C000C2102196FE0164916623B9F7E9EBF4E06491EF0107C088E290E10E94C2102196BF
:2051E000FE0164916623B9F788E290E16AE00E94C210DF91CF910895CF93DF93F8940E947A
:20520000A775779A769A479A439AE2EBF4E06491EF0107C088E290E10E94C2102196FE0141
:2052200064916623B9F7EFE2F5E06491EF0107C088E290E10E94C2102196FE01649166236B
:20524000B9F788E290E16AE00E94C210FFCFEF92FF920F931F930FB6F89480911F1090911F
:205260002010A0912110B09122100FBEE090B304F090B4040091B5041091B6042091AF04F4
:205280003091B0044091B1045091B204821B930BA40BB50BE816F9060A071B0730F4E11489
:2052A000F1040105110509F0A7DFE0907F02F09080020091810210918202E114F104010542
:2052C000110531F10FB6F89480911F1090912010A0912110B09122100FBE2091AF043091ED
:2052E000B0044091B1045091B204821B930BA40BB50BE816F9060A071B0750F49091B10BE2
:205300008091B20B981721F4779A769A479A439A0E94C64B1F910F91FF90EF9008956F926D
:205320007F928F929F92AF92BF92CF92DF92EF92FF920F931F93F82E6091B7047091B804B1
:205340008091B9049091BA042091BB043091BC044091BD045091BE040E9483963B014C0136
:2053600000D000D000D00DB71EB70F5F1F4F60916F0270917002882777FD8095982F0E94D2
:205380000A95209183023091840240918502509186020E94489720E030E040E752E40E94A0
:2053A0006F9420E030E048EC52E40E946F945B016C01F8016082718282829382F482809194
:2053C0009A04858382E794E063EC74E047EB54E020E001E032E0E32E0E942B478091C30451
:2053E0009091C404A091C504B091C6048093720490937304A0937404B09375048091C70459
:205400009091C804A091C904B091CA048093760490937704A0937804B09379048091CB0418
:205420009091CC04A091CD04B091CE0480937A0490937B04A0937C04B0937D048091CF04D8
:205440009091D004A091D104B091D20480937E0490937F04A0938004B09381040FB6F8942F
:2054600080911F1090912010A0912110B09122100FBE8093AF049093B004A093B104B09331
:20548000B2048DB79EB706960FB6F8949EBF0FBE8DBF1F910F91FF90EF90DF90CF90BF90DF
:2054A000AF909F908F907F906F900895CF92DF92EF92FF920F931F930FB6F89480911F10EB
:2054C00090912010A0912110B09122100FBE8093AF049093B004A093B104B093B20460916A
:2054E00072047091730480917404909175042091C3043091C4044091C5045091C6040E94B3
:205500006894882309F07AC0609176047091770480917804909179042091C7043091C80496
:205520004091C9045091CA040E946894882309F065C0609183027091840280918502909101
:20554000860220E030E040E752E40E946F947B018C0183EC94E067EC74E04BEC54E02FEC98
:2055600034E0EAE9CE2EE4E0DE2E0E945A518091C3049091C404A091C504B091C604809352
:20558000720490937304A0937404B09375048091C7049091C804A091C904B091CA048093AB
:2055A000760490937704A0937804B09379048091CB049091CC04A091CD04B091CE0480936B
:2055C0007A0490937B04A0937C04B0937D048091CF049091D004A091D104B091D20480932B
:2055E0007E0490937F04A0938004B09381041F910F91FF90EF90DF90CF90089560916F02D9
:2056000070917002882777FD8095982F0E940A952091830230918402409185025091860299
:205620000E94489720E030E040E752E40E946F9420E030E048EC52E488CFCF93DF9388E2C8
:2056400090E10E941092E1E5F5E06491EF0107C088E290E10E94C2102196FE0164916623CB
:20566000B9F74091A7045091A8046091A9047091AA044F5F5F4F6F4F7F4F88E290E10E94BF
:20568000E99088E290E16AE00E94C210DADCDF91CF9108952F923F924F925F926F927F925F
:2056A0008F929F92AF92BF92CF92DF92EF92FF920F931F93DF93CF9300D000D000D0CDB706
:2056C000DEB72C0163991AC1609172047091730480917404909175040E94D7944B015C0179
:2056E00080915F0290916002A0916102B09162028093830290938402A0938502B0938602B6
:2057000080E090E0A0E0B0E08093720490937304A0937404B093750482E794E066E774E0A1
:205720004AE754E02EE734E00E94734CE7E6F6E0E590F59005911491F3E76F2EF6E07F2EA8
:20574000F301649117FB109517F91095772767FD7095872F972F0E940A959B01AC01C8011E
:20576000B7010E9448976093C3047093C4048093C5049093C6046091830270918402809194
:2057800085029091860220E030E040E752E40E946F947B018C0183EC94E067EC74E04BECFD
:2057A00054E02FEC34E0EAE9CE2EE4E0DE2E0E945A510E94616EB401882777FD8095982F75
:2057C0000E940A95609372047093730480937404909375046093C3047093C4048093C5041D
:2057E0009093C60463998AC060917A0470917B0480917C0490917D040E94D7944B015C019E
:205800008091670290916802A0916902B0916A028093830290938402A0938502B093860274
:2058200080E090E0A0E0B0E080937A0490937B04A0937C04B0937D0482E794E066E774E060
:205840004AE754E02EE734E00E94734CEFE6F6E0E590F59005911491A2E0B0E06A0E7B1E56
:20586000F301649117FB109517F91095772767FD7095872F972F0E940A959B01AC01C801FD
:20588000B7010E9448976093CB047093CC048093CD049093CE046091830270918402809153
:2058A00085029091860220E030E040E752E40E946F947B018C0183EC94E067EC74E04BECDC
:2058C00054E02FEC34E00E945A510E94616EB401882777FD8095982F0E940A9560937A0441
:2058E00070937B0480937C0490937D046093CB047093CC048093CD049093CE0441145104D7
:2059000029F0F2E04F16510409F074C13201660C771C660C771C93012E583B4F3A8329836A
:2059200080E090E0A0E0B0E0F90180839183A283B38382E794E066E774E04AE754E02EE723
:2059400034E00E94734CF301E55AF94F659175918591949123E736E0420E531EF201E490D8
:2059600093012D533B4F3E832D8320E030E040EC5FE30E9448975B016C01FF24E7FCF094C6
:205980000F2D1F2DC801B7010E940A951B012C01C601B501A20191010E944897AD81BE81D4
:2059A0006D937D938D939C931397F301E15AFD4FFC83EB8360817181828193816093830214
:2059C00070938402809385029093860220E030E040E752E40E946F947B018C0183EC94E0FB
:2059E00067EC74E04BEC54E02FEC34E0AAE9CA2EA4E0DA2E0E945A510E94616E80E090E0C1
:205A0000A0E0B0E0E981FA8180839183A283B38382E794E066E774E04AE754E02EE734E013
:205A20000E94734CF301E959F94F85909590A590B490C501B4019058A20191010E944897BB
:205A4000AD81BE816D937D938D939C9313976091830270918402809185029091860220E092
:205A600030E040E752E40E946F947B018C0183EC94E067EC74E04BEC54E02FEC34E00E9445
:205A80005A510E94616EC501B401A50194010E948F93A20191010E944897ED81FE816083EA
:205AA000718382839383AB81BC816D917D918D919C9120E030E040E05FE30E944897609331
:205AC000830270938402809385029093860220E030E040E752E40E946F947B018C0183ECE9
:205AE00094E067EC74E04BEC54E02FEC34E00E945A510E94616E83010E571B4FF301EE57A7
:205B0000F94F6591759185919491FEE8EF2EF4E0FF2EE60CF71CF80120813181428153811A
:205B20000E948F93D7016D937D938D939C931397F301E257F94F6591759185919491E3E74A
:205B4000F2E06E0E7F1ED8012D913D914D915C910E948F93F3016083718382839383F80187
:205B600080819181A281B381E981FA8180839183A283B383ED81FE8180839183A283B38305
:205B800080E090E0A0E0B0E08093830290938402A0938502B09386020E94856D82E794E0EE
:205BA00066E774E04AE754E02EE734E00E94734CAB81BC816D917D918D919C91609383021D
:205BC00070938402809385029093860220E030E040E752E40E946F947B018C0183EC94E0F9
:205BE00067EC74E04BEC54E02FEC34E00E945A510E94616E26960FB6F894DEBF0FBECDBFA3
:205C0000CF91DF911F910F91FF90EF90DF90CF90BF90AF909F908F907F906F905F904F90D0
:205C20003F902F9008954091D8045091D90420E630E0B901469F9001479F300D569F300D33
:205C40001124682F772767FD7095C9018C519B4F0E94000E9C019093E3048093E20480E030
:205C6000232B09F081E00895EF92FF920F931F93CF93DF93EC017A018B01FC01649107C0F8
:205C800088E290E10E94C2102196FE0164916623B9F788E290E1B801A7012AE000E00E9409
:205CA0005E90DF91CF911F910F91FF90EF900895EF92FF920F931F93CF93DF93EC017A0189
:205CC0008B01FC01649107C088E290E10E94C2102196FE0164916623B9F788E290E1B801B8
:205CE000A70122E00E94FA90DF91CF911F910F91FF90EF900895F8946AE070E080E090E00D
:205D00000E94228D81E08093E00080E28093D80064E670E080E090E00E94228D1DBA10925D
:205D200068001CBC10BE1FBA10927A0010926E0010926F0010927000109271001092C900AF
:205D40001092BC0011B814B817B81AB81DB810BA12B815B818B81BB81EB811BA0C9400F89D
:205D6000FFCF8091E2049091E304019660E070E04AE050E00C94770C8091E2049091E304B3
:205D8000019660E070E00C941A0B0F931F93CF93DF938C0180919A048093A60484E543DF6B
:205DA000882309F44EC0E8DF0E94DC946093A604662309F446C0ECEAF4E06491EF0107C0D5
:205DC00088E290E10E94C2102196FE0164916623B9F70936110599F00A36110524F4083606
:205DE0001105E1F407C00D36110571F00A3D1105A9F40FC088E290E160E271E00EC088E2C8
:205E000090E167E371E009C088E290E16EE471E004C088E290E165E671E00BD9E091281067
:205E2000F09129100190F081E02D88E290E16091A604099588E290E16AE00E94C21081E08B
:205E400001C080E0DF91CF911F910F910895AF92BF92CF92DF92EF92FF920F931F93CF9338
:205E6000DF93A2E7EA2EA4E0FA2EC3ECD4E000E010E0F801E951FD4F8081D5DE882331F130
:205E80007BDF5B016C01F801E459FB4F8081882311F061E002C06091D30470E0882777FD74
:205EA0008095982F0E940A95F70120813181428153810E9448979B01AC01C601B5010E94FA
:205EC0008F93688379838A839B8309C0F70180819181A281B38188839983AA83BB830F5F63
:205EE0001F4F84E090E0E80EF91E24960430110509F0BFCF86E497DE8823D9F03DDF7B01DD
:205F00008C016093D4047093D5048093D6049093D70420E030E040E050E00E947696181626
:205F200044F4E0928302F09284020093850210938602DF91CF911F910F91FF90EF90DF9048
:205F4000CF90BF90AF90089582DF89E46CDE882351F012DF6093B7047093B8048093B90485
:205F60009093BA040CC080E090E0A0E0B0E08093B7049093B804A093B904B093BA048AE488
:205F800052DE882351F0F8DE6093BB047093BC048093BD049093BE04089580E090E0A0E0F4
:205FA000B0E08093BB049093BC04A093BD04B093BE0408952F923F924F925F926F927F9290
:205FC0008F929F92AF92BF92CF92DF92EF92FF920F931F93DF93CF93CDB7DEB76E970FB6EE
:205FE000F894DEBF0FBECDBF87E41DDE882309F429C2C2DE0E94D7946430710509F43CC076
:206000006530710554F46230710531F16330710554F57723CCF40C94D43F6A35710509F492
:20602000C0C16B35710534F46C31710511F00C94D43F78C06B35710509F4B7C16C35710500
:2060400011F00C94D43FB6C18091A504882321F4FEDE2CDA0C9407408091A504882319F460
:2060600073DF81E006C08091A504882329F46CDF80E055D90C94074080E5D5DD882321F48E
:20608000AA24BB24650105C077DE0E94DC945B016C0183E5C8DD882359F06EDE20E030E09B
:2060A0004AE754E40E9448970E94DC945B016C010E94616E0FB6F894E0901F10F09020100A
:2060C00000912110109122100FBEEA0CFB1C0C1D1D1D0FB6F89480911F1090912010A091DB
:2060E0002110B09122100FBE8093AF049093B004A093B104B093B20403C00E94FF78A7D856
:206100000FB6F89480911F1090912010A0912110B09122100FBE8E159F05A007B10768F3FA
:206120000C94D43F8091830290918402A0918502B09186028093DE049093DF04A093E004DC
:20614000B093E10480916F0290917002909371048093700484E690E09093700280936F02F0
:206160000FB6F89480911F1090912010A0912110B09122100FBE8093AF049093B004A093CB
:20618000B104B093B20481E00E948C6D8091720490917304A0917404B09175048093C304F9
:2061A0009093C404A093C504B093C6048091760490917704A0917804B09179048093C7047B
:2061C0009093C804A093C904B093CA0480917A0490917B04A0917C04B0917D048093CB043B
:2061E0009093CC04A093CD04B093CE0480917E0490917F04A0918004B09181048093CF04FB
:206200009093D004A093D104B093D20480E090E0A0E0B0E08093830290938402A09385028B
:20622000B093860288E5FFDC882351F489E5FBDC882331F48AE5F7DC882311F481E001C032
:2062400080E080938702882321F488E5ECDC882319F080E090E01EDA80918702882321F477
:2062600089E5E1DC882361F080E090E0A0E0B0E08093760490937704A0937804B09379047D
:2062800080918702882321F48AE5CDDC882319F082E090E0FFD988E5C6DC8823B1F061DD95
:2062A000611571058105910581F08091820490918304A0918404B0918504809372049093F7
:2062C0007304A0937404B093750489E5ACDC882391F047DD611571058105910561F080E0E1
:2062E00090E0A0E0B0E08093760490937704A0937804B09379048AE596DC8823B1F031DD49
:20630000611571058105910581F080918A0490918B04A0918C04B0918D0480937A0490936E
:206320007B04A0937C04B0937D0482E794E066E774E04AE754E02EE734E00E94734C80E09A
:206340000E948C6D8091DE049091DF04A091E004B091E1048093830290938402A093850275
:20636000B093860280917004909171049093700280936F020FB6F89480911F10909120103C
:20638000A0912110B09122100FBE8093AF049093B004A093B104B093B2040E94856D0C94A9
:2063A000D43F1092D3040C94D43F81E08093D3040C94D43F85E437DC882311F40E94616E03
:2063C000B2E7EB2EB4E0FB2EA2E8CA2EA4E0DA2E00E010E0F801E951FD4F808124DC882345
:2063E00021F1033059F4C8DCF70160837183828393838EE794E00E94564C17C0BDDCF601E9
:2064000020813181428153810E948F93F701608371838283938382E794E066E774E04AE735
:2064200054E02EE734E00E94734C0F5F1F4F44E050E0E40EF51EC40ED51E0430110551F613
:206440000C94D43F8DE4EFDB882311F40C940D3F93DC0E94D7946B36710511F40C948C3AB4
:206460006C3671050CF092C06F31710509F48AC3603271050CF042C06731710509F469C21A
:2064800068317105E4F46431710509F428C2653171055CF46131710509F41BC262317105DC
:2064A00011F00C94D43F0C949A3A6531710509F444C26631710511F00C94D43F44C26A3143
:2064C000710509F480C26B31710554F46831710509F45AC26931710511F00C94D43F6DC292
:2064E0006C31710509F492C26C3171050CF488C26E31710511F00C94D43FC4C26036710580
:2065000009F4F8C06136710514F56335710511F40C94963A6435710554F46A32710509F4C7
:20652000DEC36235710511F00C94D43FFCC76535710511F40C94E33A653571050CF4FAC793
:206540006C35710511F00C94D43F0C94F93A6336710509F486C16436710554F461367105E5
:2065600009F4CEC06236710511F00C94D43F73C16936710509F424C46A3671050CF09BC72C
:206580006836710511F00C94D43FEAC36E3C710511F40C94B83D6F3C71050CF04FC0693700
:2065A000710511F40C948D3C6A37710524F56337710511F40C947E3B643771055CF46D3655
:2065C000710509F4CDC46237710511F00C94D43F0C949E3B6737710511F40C94913C683756
:2065E000710514F00C94893C6537710511F00C94D43F0C948E3B693C710511F40C94FA3C97
:206600006A3C710554F46C38710509F4C8C36E3B710511F00C94D43F7CC66C3C710511F43C
:206620000C943A3D6D3C710514F00C945A3D6B3C710511F00C94D43F0C941C3D51E0643F4B
:20664000750711F40C94E33E81E0653F78074CF591E06D32790711F40C94F43DE1E06E326C
:206660007E0764F46C3D710511F40C94D63D6D3D710511F00C94D43F0C94E53DF1E06F325E
:206680007F0711F40C94A03E21E06F32720714F40C949C3E6059714011F00C94D43F0C9496
:2066A000E03E51E0673F750711F40C94EC3E81E0683F78076CF491E0653F790711F40C9479
:2066C000E63E665F714011F00C94D43F0C94E93EF3E0603A7F0709F41AC223E0673E7207B8
:2066E00011F40C94F83E6455734011F00C94D43F0C94EF3E8FE69EE00E94A0860C94D43F64
:2067000081E491DA882339F037DBAB01BC018FE69EE00E942B8687E586DA882339F02CDB6D
:20672000AB01BC018FE69EE00E94038680E57BDA882339F021DBAB01BC018FE69EE00E944A
:2067400082818AE570DA882359F40F2EF0E04F2EF0E05F2EF0E86F2EFFEB7F2EF02D03C0B2
:206760000BDB2B013C0188E45EDA882359F40F2EF0E08F2EF0E09F2EF0E8AF2EFFEBBF2E3B
:20678000F02D03C0F9DA4B015C018CE44CDA882359F40F2EF0E0CF2EF0E0DF2EF0E8EF2E33
:2067A000FFEBFF2EF02D03C0E7DA6B017C01C301B20120E030E040E050E00E947696882308
:2067C00024F1C501B40120E030E040E050E00E947696882344F08FE69EE0B301A20195015C
:2067E00084010E94D088C701B60120E030E040E050E00E947696882344F08FE69EE0B30107
:20680000A201970186010E942B89C701B60120E030E040E050E00E947696181614F00C9401
:20682000D43FC501B40120E030E040E050E00E947696181614F00C94D43FC501B401A701B4
:2068400096010E946F94AB01BC018FE69EE00E94AC7F0C94D43F82E493E00E94DA260C9405
:20686000D43F88E5E0D9882349F086DA9B01AC0182E493E060E070E00E94962489E5D3D973
:20688000882349F079DA9B01AC0182E493E061E070E00E9496248AE5C6D9882349F06CDA7A
:2068A0009B01AC0182E493E062E070E00E94962485E4B9D9882311F40C94D43F5DDA9B0197
:2068C000AC0182E493E063E070E00E9496240C94D43F77987698479843980C94D43FEBE437
:2068E000F6E064918F0108C088E290E10E94C2100F5F1F4FF80164916623B1F788E290E150
:206900006AE00E94C21084E793E00E949319EDE3F6E064918F0108C088E290E10E94C2104B
:206920000F5F1F4FF80164916623B1F788E290E16AE00E94C2100C94D43F84E793E00E9490
:20694000DE150C94D43F84E793E00E9433110C94D43F8091E2049091E30404966AE270E0E5
:206960000E94000EFC01009711F0319710826091E2047091E3046C5F7F4F84E793E041E021
:206980000E9474120C94D43F84E793E00E9437110FB6F89480911F1090912010A091211010
:2069A000B09122100FBE80939D0490939E04A0939F04B093A0040C94D43F84E793E00E942E
:2069C0003E110C94D43F80917703882311F40C94D43F83E528D9882311F40C94D43FC1D961
:2069E000AB01BC01409361045093620480936304709364048EE394E00E94DF5F0C94D43F50
:206A000084E793E00E9415120C94D43F8091E2049091E30404966AE270E00E94000E8C01AA
:206A2000009719F12091D8043091D90480E690E0AC01249FC001259F900D349F900D11247D
:206A40008C519B4F6EE470E00E94000E60E270E00E94000E9C012F5F3F4F3093E3042093C5
:206A6000E20401501040F80110826091E2047091E3046C5F7F4F84E793E040E00E94741286
:206A80000C94D43F80917703882311F40C94D43F84E793E00E948D118091E2049091E30438
:206AA00004966AE270E00E94000E8C01009719F12091D8043091D90480E690E0AC01249F51
:206AC000C001259F900D349F900D11248C519B4F6EE470E00E94000E60E270E00E94000E94
:206AE0009C012F5F3F4F3093E3042093E20401501040F80110826091E2047091E3046C5FE4
:206B00007F4F84E793E00E947E140C94D43F8091E2049091E30405966AE270E00E94000EFC
:206B20008C01009719F12091D8043091D90480E690E0AC01249FC001259F900D349F900D24
:206B400011248C519B4F6EE470E00E94000E60E270E00E94000E9C012F5F3F4F3093E30442
:206B60002093E20401501040F80110826091E2047091E3046B5F7F4F84E793E00E947814ED
:206B80000C94D43F0FB6F89460911F107091201080912110909122100FBE6093A1047093A3
:206BA000A2048093A3049093A40420919D0430919E0440919F045091A004621B730B840B72
:206BC000950B28EE33E040E050E00E944C98F22EE32ED42EC52E4DB75EB7485050400FB6EA
:206BE000F8945EBF0FBE4DBF0DB71EB70F5F1F4FCE010196EDB7FEB7928381838EE296E0E0
:206C0000F801938382836F2D7E2D8D2D9C2D2CE330E040E050E00E944C98F8013583248349
:206C20006F2D7E2D8D2D9C2D2CE330E040E050E00E944C98F801778366830E942F0EECEA04
:206C4000F4E064918F014DB75EB7485F5F4F0FB6F8945EBF0FBE4DBF08C088E290E10E94E1
:206C6000C2100F5F1F4FF80164916623B1F788E290E1BE016F5F7F4F0E94192888E290E153
:206C80006AE00E94C2108091E006882311F40C94D43F1092E00680919A04082F10E0000F6F
:206CA000111F005E114FF80160817181882777FD8095982F0E940A9520918C0230918D024B
:206CC00040918E0250918F020E947696181614F00C94D43FF801118210820C94D43F83E515
:206CE0000E94132E882311F40C94D43F45D80E94D7947B018C016B0180E50E94132E8823BC
:206D000061F0F7FC0AC0FFEFEF16F10409F02CF433D80E94D7947B0103C0EE24EA94FE2C53
:206D2000EBEEF2E0808191818E159F0511F40C94D43F329623E0EB35F207A1F7F7FE02C063
:206D40000C94D43F8E2D0E94988BEE2DF0E00C2C0E94A98B8E2DB6010E94538D0C94D43F60
:206D600088E690E012D8882311F00C94D43F83E50E94132E882379F00E94BC2E2091A604A6
:206D8000022F10E0000F111F005E114F0E94D794F801718360830E94A6750C94D43F83E520
:206DA0000E94132E882311F40C94D43F0E94BC2E0E94D7947093230E6093220E0C94D43FEA
:206DC00089E690E00E94C52E882311F00C94D43FE8E2F6E064918F0108C088E290E10E9476
:206DE000C2100F5F1F4FF80164916623B1F7E091A604F0E0EE0FFF1FEE0FFF1FEA5DF14F1E
:206E0000408151816281738188E290E121E00E94FA90E5E2F6E064918F0108C088E290E13B
:206E20000E94C2100F5F1F4FF80164916623B1F7E091A604F0E0EE0FFF1FE05EF14F60817E
:206E40007181882777FD8095982F0E940A95AB01BC0188E290E121E00E94FA90E1E2F6E0F6
:206E600064918F0108C088E290E10E94C2100F5F1F4FF80164916623B1F740912C0E50918F
:206E80002D0E60912E0E70912F0E88E290E121E00E94FA90EEE1F6E064918F0108C088E2E8
:206EA00090E10E94C2100F5F1F4FF80164916623B1F76091220E7091230E882777FD809567
:206EC000982F0E940A95AB01BC0188E290E121E00E94FA90EAE1F6E064918F0108C088E2E1
:206EE00090E10E94C2100F5F1F4FF80164916623B1F78091A60490E00E949B75AC0166279B
:206F000057FD6095762F88E290E10E94E990E5E1F6E064918F0108C088E290E10E94C21055
:206F20000F5F1F4FF80164916623B1F78FEF9FEF0E949B75AC01662757FD6095762F88E206
:206F400090E10E94E99088E290E16CE771E00E94192888E290E16AE00E94C2100C940740C3
:206F60008DE690E00E94C52E882311F00C94D43F1092E00683E50E94132E882379F00E94B1
:206F8000BC2E2091A604022F10E0000F111F005E114F0E94D794F8017183608383E50E94A7
:206FA000132E882351F00E94BC2E60938C0270938D0280938E0290938F0282E40E94132E65
:206FC000882351F00E94BC2E609388027093890280938A0290938B0286E40E94132E8823E7
:206FE00069F00E94BC2E6093900270939102809392029093930281E08093E0060E94A6751B
:207000000FB6F89480901F1090902010A0902110B09022100FBE2091A604022F10E07724D9
:20702000000F111FF801E05EF14F60817181882777FD8095982F0E940A95000F111F0A5DE1
:20704000114FF80120813181428153810E947696181614F477247394CC24CA94DC2C76019A
:20706000E2E1F6E04490EEE0F6E05490EAE0F6E0649039C1642D02E116E008C088E290E180
:207080000E94C2100F5F1F4FF80164916623B1F7E091A604F0E0EE0FFF1FEE0FFF1FEA5D19
:2070A000F14F408151816281738188E290E121E00E94FA90652D0EE016E008C088E290E105
:2070C0000E94C2100F5F1F4FF80164916623B1F74091A60450E0662757FD6095762F88E2B1
:2070E00090E10E94E990662D0AE016E008C088E290E10E94C2100F5F1F4FF8016491662327
:20710000B1F7F7FC24C00FB6F89420911F103091201040912110509122100FBEC701B6016D
:2071200068577C4E8F4F9F4F621B730B840B950B28EE33E040E050E00E944C9888E290E1F6
:20714000BA01A9012AE000E00E945E9006C088E290E16DE771E00E94192888E290E16AE002
:207160000E94C2100FB6F89480901F1090902010A0902110B09022100FBE0E94FF780E9460
:207180002729FFEFCF16FFEFDF06FFEFEF06FFEFFF0609F050C0E091A604772031F1F0E076
:2071A0008F01000F111F000F111F0A5D114FEE0FFF1FE05EF14F60817181882777FD809556
:2071C000982F0E940A9520E030E040E85FE30E948E939B01AC01F80160817181828193813E
:2071E0000E94769687FF58C062C0F0E08F01000F111F000F111F0A5D114FEE0FFF1FE05E23
:20720000F14F60817181882777FD8095982F0E940A9520E030E040E85FE30E948F939B0141
:20722000AC01F80160817181828193810E946894181694F53CC0F7FC3AC0E091A604F0E095
:207240008F01000F111F000F111F0A5D114FEE0FFF1FE05EF14F60817181882777FD8095B5
:20726000982F0E940A959B01AC01F80160817181828193810E948E930E94D79497FF07C0AD
:2072800090958095709561957F4F8F4F9F4F64307105810591055CF00FB6F894C0901F10DD
:2072A000D0902010E0902110F09022100FBEFFEFCF16FFEFDF06FFEFEF06FFEFFF0699F019
:2072C000F7FC75C60FB6F89480911F1090912010A0912110B09122100FBE8C199D098858D1
:2072E000934108F064C60FB6F89480911F1090912010A0912110B09122100FBE88199909D1
:20730000AA09BB09895E9340A040B04008F0B2CE34CF83E50E94132E882341F00E94BC2E3E
:207320000E94D7947093230E6093220E0FB6F894E0901F10F09020100091211010912210B4
:207340000FBEE7E0F6E09490E3E0F6E0A490EFEFF5E0B49085C00FB6F89480911F109091E4
:207360002010A0912110B09122100FBE8E199F09A00BB10B895E9340A040B04008F46CC0D3
:20738000E0919A04F0E0EE0FFF1FEE0FFF1FEA5DF14FC080D180E280F380692D07E016E078
:2073A00008C088E290E10E94C2100F5F1F4FF80164916623B1F788E290E1B701A60122E07F
:2073C0000E94FA906A2D03E016E008C088E290E10E94C2100F5F1F4FF80164916623B1F7FF
:2073E00040919A0450E0662757FD6095762F88E290E10E94E9906B2D0FEF15E008C088E2C0
:2074000090E10E94C2100F5F1F4FF80164916623B1F740912C0E50912D0E60912E0E709137
:207420002F0E88E290E121E00E94FA9088E290E16CE771E00E94192888E290E16AE00E94DE
:20744000C2100FB6F894E0901F10F090201000912110109122100FBE0E94FF780E9427294D
:207460006091220E7091230E882777FD8095982F0E940A9520912C0E30912D0E40912E0E85
:2074800050912F0E0E94769618160CF464CF0FB6F89480911F1090912010A0912110B0913A
:2074A00022100FBE8093AF049093B004A093B104B093B20479C53C9A449A83E50E94132E12
:2074C000882319F10E94BC2E20E030E040E050E00E94689488231CF460E070E011C00E94AF
:2074E000BC2E20E030E04FE753E40E94769618161CF46FEF70E004C00E94BC2E0E94D7942E
:2075000070939C0460939B044FC58FEF90E090939C0480939B0448C510929C0410929B042F
:207520003C9A449841C510926F043EC581E080936F043AC583E50E94132E882399F00E9474
:20754000BC2E20E030E04AE754E40E9448970E94DC9460937F027093800280938102909383
:20756000820222C588E50E94132E882309F046C589E50E94132E882309F040C58AE50E9496
:20758000132E882309F03AC585E40E94132E882309F034C50E94616E439A0E946D6E04C58A
:2075A000779A89E50E94132E8111769A8AE50E94132E8111479A85E40E94132E882309F40E
:2075C000F3C4439AF1C483E50E94132E0E94BC2E20E030E04AE754E40E9448970E94DC947F
:2075E0006093B3047093B4048093B5049093B604DBC444E8642E46E0742E34E7232E36E0D6
:20760000332E20EC422E26E0522E88249924F401E951FD4F80810E94132E882309F45DC07A
:20762000F3E08F1609F052C00E94BC2E5B016C0120E030E040EA51E40E94689488230CF0BE
:207640003FC0F3016081718182819381A60195010E946F947B018C016091B8067091B906F3
:207660008091BA069091BB06A80197010E9448976093B8067093B9068093BA069093BB066B
:20768000F1016081718182819381A80197010E944897F1016083718382839383F201608194
:2076A0007181828193810E940895A80197010E9448970E94DC94F2016083718382839383C9
:2076C000F301A082B182C282D38207C00E94BC2EF30160837183828393830894811C911CA9
:2076E00044E050E0640E751E240E351E440E551E54E08516910409F08ACF56C4E4EAF5E074
:2077000064918F0108C088E290E10E94C2100F5F1F4FF80164916623B1F746C48091E204D1
:207720009091E30405966AE270E00E94000EFC01009709F439C43197108236C4E1EAF5E0D8
:2077400064918F0108C088E290E10E94C2100F5F1F4FF80164916623B1F74091720450916A
:207760007304609174047091750488E290E122E00E94FA90EEE9F5E064918F0108C088E243
:2077800090E10E94C2100F5F1F4FF80164916623B1F74091760450917704609178047091F4
:2077A000790488E290E122E00E94FA90EBE9F5E064918F0108C088E290E10E94C2100F5F90
:2077C0001F4FF80164916623B1F740917A0450917B0460917C0470917D0488E290E122E09D
:2077E0000E94FA90E8E9F5E064918F0108C088E290E10E94C2100F5F1F4FF80164916623C8
:20780000B1F740917E0450917F04609180047091810488E290E122E00E94FA90EDE8F5E05B
:2078200064918F0108C088E290E10E94C2100F5F1F4FF80164916623B1F780E00E942C6E15
:207840000E940A95209184063091850640918606509187060E946F94AB01BC0188E290E1AC
:2078600022E00E94FA90EAE8F5E064918F0108C088E290E10E94C2100F5F1F4FF8016491CD
:207880006623B1F781E00E942C6E0E940A95209188063091890640918A0650918B060E94D5
:2078A0006F94AB01BC0188E290E122E00E94FA90E7E8F5E064918F0108C088E290E10E94E5
:2078C000C2100F5F1F4FF80164916623B1F782E00E942C6E0E940A9520918C0630918D0665
:2078E00040918E0650918F060E946F94AB01BC0188E290E122E00E94FA9088E290E16CE768
:2079000071E00E94192888E290E16AE00E94C2104BC380E00E948C6D47C381E00E948C6D8B
:2079200043C388E290E16FE771E00E94192888E290E16AE00E94C210EFE7F5E064918F0113
:2079400008C088E290E10E94C2100F5F1F4FF80164916623B1F7639B03C068E971E002C0F0
:207960006DE971E088E290E10E94192888E290E16AE00E94C210E7E7F5E064918F0108C019
:2079800088E290E10E94C2100F5F1F4FF80164916623B1F7639B03C068E971E002C06DE922
:2079A00071E088E290E10E94192888E290E16AE00E94C210EFE6F5E064918F0108C088E2BE
:2079C00090E10E94C2100F5F1F4FF80164916623B1F7639B03C068E971E002C06DE971E0FB
:2079E00088E290E10E94192888E290E16AE00E94C210DAC207EE12E094E9E92E96E0F92E7C
:207A0000F80180810E94132E882349F00E94BC2E0E94DC94F70160837183828393830F5FAF
:207A20001F4F44E050E0E40EF51E52E00B3E150739F70E942B4CB8C207EE12E084E7E82EBD
:207A400086E0F82EF80180810E94132E882339F00E94BC2EF70160837183828393830F5F05
:207A60001F4F44E050E0E40EF51E52E00B3E150749F79AC283E50E94132E882351F00E9433
:207A8000BC2E6093A8067093A9068093AA069093AB0684E50E94132E882309F485C20E9435
:207AA000BC2E6093AC067093AD068093AE069093AF067AC283E50E94132E882351F00E94CD
:207AC000BC2E6093A4067093A5068093A6069093A70684E50E94132E882351F00E94BC2E1E
:207AE0006093BC067093BD068093BE069093BF0682E40E94132E882361F00E94BC2E0E94D9
:207B0000DC946093700670937106809372069093730688E50E94132E882351F00E94BC2E23
:207B20006093B0067093B1068093B2069093B3068AE50E94132E882351F00E94BC2E60937E
:207B4000B4067093B5068093B6069093B70685E40E94132E882309F427C20E94BC2E6093A2
:207B6000B8067093B9068093BA069093BB061CC207EE12E0B2E8EB2EB4E0FB2EF80180819F
:207B80000E94132E882339F00E94BC2EF70160837183828393830F5F1F4F44E050E0E40E96
:207BA000F51E52E00A3E150749F7FEC183E50E94132E882309F4F8C10E94BC2E0E94D794D8
:207BC0007093700260936F02EFC183E50E94132E882309F4E9C10E94BC2E0E94D7947093E3
:207BE000720260937102E0C180E50E94132E882351F00E94BC2E6093990270939A0280930A
:207C00009B0290939C0289E40E94132E882361F00E94BC2E0E94B57560939D0270939E022D
:207C200080939F029093A00284E40E94132E882361F00E94BC2E0E94C1756093A102709387
:207C4000A2028093A3029093A40283E40E94132E882351F00E94BC2E6093A5027093A602F8
:207C60008093A7029093A8020E94847588E290E167EA71E00E94192888E290E16AEA71E000
:207C80000E9419284091990250919A0260919B0270919C0288E290E122E00E94FA9088E278
:207CA00090E16EEA71E00E94192860919D0270919E0280919F029091A0020E94BB75AB01A3
:207CC000BC0188E290E122E00E94FA9088E290E162EB71E00E9419286091A1027091A20249
:207CE0008091A3029091A4020E94C775AB01BC0188E290E122E00E94FA9088E290E166EB8B
:207D000071E00E9419284091A5025091A6026091A7027091A80288E290E122E00E94FA90E0
:207D200088E290E16CE771E00E94192888E290E16AE00E94C21038C181E00E942A4C34C1E1
:207D400085E40E94132E882319F4CC24DD2412C00E94BC2E0E94D7946B0177FF0BC00F2ED9
:207D6000F0E0EF2EF0E0FF2EFCE80F2FF2E41F2FF02D0AC00F2EF0E0EF2EF0E0FF2EF6E1EE
:207D80000F2FF3E41F2FF02D83E50E94132E882321F00E94BC2E7B018C0183E40E94132E7D
:207DA000882319F425E030E005C00E94BC2E0E94D7949B01C801B701A6010E94C47AF4C040
:207DC0000E94616EF1C00E94F920EEC00E94F51EEBC00E94DB19E8C00E948A1BE5C086E424
:207DE0000E94132E882309F4DFC00E947B2EDCC01092A5048091AB049091AC04A091AD04B4
:207E0000B091AE048093A7049093A804A093A904B093AA040E941D2BC7C084E50E94132E54
:207E2000882309F47CC00E94BC2E0E94DC946093A604662369F1ECEAF4E064918F0108C049
:207E400088E290E10E94C2100F5F1F4FF80164916623B1F788E290E16AEB71E00E94192874
:207E6000E0912810F09129100190F081E02D88E290E16091A604099588E290E16CEB71E0F9
:207E80000E94192888E290E16AE00E94C2108CC086E40E94132E8823E1F00E94BC2E7B0149
:207EA0008C016093D4047093D5048093D6049093D70420E030E040E050E00E947696181667
:207EC00044F4E0928302F09284020093850210938602ECEAF4E064918F0108C088E290E154
:207EE0000E94C2100F5F1F4FF80164916623B1F788E290E16DEC71E00E94192840919A043C
:207F000050E0662757FD6095762F88E290E10E94E99088E290E16AE00E94C21045C0ECEA4C
:207F2000F4E064918F0108C088E290E10E94C2100F5F1F4FF80164916623B1F7ECE5F5E030
:207F400064918F0108C088E290E10E94C2100F5F1F4FF80164916623B1F72091D80430913C
:207F6000D90480E690E0289FB001299F700D389F700D11246C517B4F88E290E10E941928C3
:207F8000EAE5F5E064918F0108C088E290E10E94C2100F5F1F4FF80164916623B1F788E23C
:207FA00090E16AE00E94C2100E94212830C00FB6F89480911F1090912010A0912110B09132
:207FC00022100FBE80939D0490939E04A0939F04B093A0040FB6F89480911F10909120108A
:207FE000A0912110B09122100FBE8093AF049093B004A093B104B093B204D6CF0E94616E4B
:208000000895889A0895899A08958A9A08958B9A08958C9A08958D9A08958E9A08958F9A4C
:20802000089558985AC0599874C05A9808955B9808955C9808955D9808955E9808955F98A8
:20804000089570980895719808954098089541980895429808954398089544986CC0459879
:2080600064C046985CC047980895769808957798089528980895299808952A9808952B9832
:2080800008952C9840C02D982CC02E9830C02F9834C01098089511980895129808951398E0
:2080A0000895149808951598089516980895179808957498089575980895889808958998C8
:2080C00008958A9808958B9808958C9808958D9808958E9808958F980895E4B5EF7DE4BDD4
:2080E0000895E0918000EF77E09380000895E0918000EF7DE09380000895E0918000E77FB8
:20810000E09380000895E091B000EF77E093B0000895E091B000EF7DE093B0000895E091CA
:208120009000EF77E09390000895E0919000EF7DE09390000895E0919000E77FE093900032
:208140000895EE3258F4EE0FEE0FFF27EC3718F4EE54FF430994EC54FF430994EE270895D5
:20816000E1E00895E9B1E170D9F70895E9B1E270B9F70895E9B1E47099F70895E9B1E87003
:2081800079F70895E9B1E07159F70895E9B1E07239F70895E9B1E07419F70895E9B1E078B4
:2081A000F9F60895ECB1E170D9F60895ECB1E270B9F60895E6B1E17099F60895E6B1E270A1
:2081C00079F60895E6B1E47059F60895E6B1E87039F60895E6B1E07119F60895E6B1E07284
:2081E000E9F50895E6B1E074C9F50895E6B1E078A9F50895ECB1E07489F50895ECB1E07893
:2082000069F50895E3B1E17049F50895E3B1E27029F50895E3B1E47009F50895E3B1E87093
:20822000E9F40895E3B1E071C9F40895E3B1E072A9F40895E3B1E07489F40895E3B1E07877
:2082400069F40895E0B1E17049F40895E0B1E27029F40895E0B1E47009F40895E1E00895EE
:20826000E0B1E870D9F70895E0B1E071B9F70895E0B1E07299F70895E0B1E07479F7089577
:20828000E0B1E07859F70895ECB1E07139F70895ECB1E07219F70895EFB1E170F9F6089534
:2082A000EFB1E270D9F60895EFB1E470B9F60895EFB1E87099F60895EFB1E07179F60895FF
:2082C000EFB1E07259F60895EFB1E07439F60895EFB1E07819F608951DBA109268001CBCA3
:2082E00010BE1FBA10927A0010926E0010926F0010927000109271001092C9001092BC00AC
:2083000011B814B817B81AB81DB810BA12B815B818B81BB81EB811BA0895F89480E29EE4A0
:208320000197F1F781E08093E00080E28093D80080E69AEE0197F1F7CFDF0C9400FEFFCF94
:20834000F894CADF80E69AEE0197F1F70C940000FFCF8F938FB78F9380915B118D5F8D3755
:20836000D0F480935B11809157118F5F80935711D8F0809158118F4F80935811A8F0809193
:2083800059118F4F8093591178F080915A118F4F80935A1109C08D5780935B118091571133
:2083A0008E5F8093571128F7809153118C5F8093531158F0809154118F4F8093541128F033
:2083C000809155118F4F809355118F918FBF8F9118959B01AC0114D0FB010CC011D06E1B35
:2083E0007F0B685E7340D0F32150304040405040E851FC4F211531054105510579F708952D
:208400000FB6F89466B515B27091531180915411909155110FBE10FE05C06F3F19F07C5F95
:208420008F4F9F4F11240024660F001C660F001C702908951F93CF93DF93182FEB014CDDDD
:20844000103109F44FC0113160F4113009F442C01130A8F01E3009F455C01F3009F05CC05C
:2084600049C01931B9F01A3120F4183109F054C02BC01A31B9F01B3109F04EC01DC0209785
:2084800021F4589884B58F7D03C0C8BD84B5806284BD4AC0D0938900C0938800809180008C
:2084A000806807C0D0938B00C0938A008091800080628093800038C0D0938D00C0938C0075
:2084C000809180008860F5CFC093B3008091B000806805C0C093B4008091B000806280932E
:2084E000B00022C0D0939900C09398008091900080680FC0D0939B00C0939A00809190001F
:20850000806207C0D0939D00C0939C008091900088608093900008C0E12FF0E0C038D10521
:2085200014F41CDD01C014DDDF91CF911F910895F894E1E6F0E020E82083108283E084BD67
:2085400085BDEEE6F0E080818160808391E09093800082E0809381009093B0008093B100AF
:20856000909390008093910086E880937A0020937B0010927E0002D0789408958091D800F7
:2085800087FF02C085FF1BC081E88093D70080EA8093D80086E189BD09B400FEFDCF80E9EF
:2085A0008093D8001092E00010926B1110926C1110925F111092E1008DE08093E20008957D
:2085C0001F920F920FB60F920BB60F9211242F933F934F935F936F937F938F939F93AF933A
:2085E000BF93EF93FF931092E9008091E80083FF57C12091F1009091F1004091F1005091A0
:20860000F1006091F1007091F100A091F100B091F10082EF8093E800963009F044C0E8EE3C
:20862000F9E120E0859195918417950711F0359617C0859195918617970711F0339610C039
:20864000259135914491CD01AF3FB10519F010F08FEF90E0841708F4482FF9015EEF04C047
:208660002F5F2630F9F61CC18091E800282F30E0C90185709070892BB9F322FD14C1242F84
:20868000413208F020E2922F04C085918093F10091509923D1F7421B5093E800442321F7C2
:2086A000203211F300C1953061F48EEF8093E8008091E80080FFFCCF842F80688093E3003D
:2086C000F2C0993009F5222309F0EAC040936B1110925F1110925C118EEF8093E800E2E18E
:2086E000FAE191E09093E90085918093EB00882331F085918093EC0085918093ED009F5F19
:20870000953081F78EE1C7C0983061F4203809F0C7C08091E80080FFFCCF80916B1180934E
:20872000F10096C09132A9F4213A09F0B9C08091E80080FFFCCF20E030E0F901E153FD4FF8
:2087400080818093F1002F5F3F4F27303105A9F77FC0903209F04BC0213209F0A1C0809108
:20876000E80082FFFCCF20E030E0F901E153FD4F8091F10080832F5F3F4F27303105A9F7ED
:208780008BEF8093E8008EEF8093E8008091CF029091D002A091D102B091D20286389105AA
:2087A000A105B10519F48FE080935D118091CF029091D002A091D102B091D202863991051D
:2087C000A105B10509F06FC084E08093E9002FEF06C02093E8008091E80082FDFCCF8091E2
:2087E000EE0090E083709070892B99F7A9DD923251F4213209F054C040935F118091E800B9
:2088000080FFFCCF25C0933241F4213209F048C08091E80080FFFCCF1BC09923E9F4809113
:20882000E80080FFFCCF223811F080E00DC06093E9008091EB0090E025E0969587952A952B
:20884000E1F781701092E9008093F1001092F1008EEF8093E80027C0913011F0933001F553
:208860002230F1F4452BE1F4262F2F77822F81508630B0F48EEF8093E8002093E9009330CE
:2088800079F089E18093EB0081E090E002C0880F991F2A95E2F78093EA001092EA0003C041
:2088A00081E28093EB00FF91EF91BF91AF919F918F917F916F915F914F913F912F910F9058
:2088C0000BBE0F900FBE0F901F9018951F920F920FB60F920BB60F9211242F933F934F93A3
:2088E0005F936F937F938F939F93AF93BF93EF93FF938091E1001092E100982F83FF11C0E7
:208900001092E90081E08093EB001092EC0082E28093ED0088E08093F00010926B11109250
:208920005F1192FF1DC080916B118823C9F080915C11882359F0815080935C11882331F4D5
:2089400084E08093E9008AE38093E80080915D11882331F0815080935D11882309F4DDDC51
:2089600090FF0CC080E18093E20010926B1181E080936C1180EA8093D80019BC80916C117F
:20898000882379F094FF0DC086E189BD09B400FEFDCF80E98093D8008DE08093E2001092D7
:2089A0006C11FF91EF91BF91AF919F918F917F916F915F914F913F912F910F900BBE0F90D3
:2089C0000FBE0F901F901895B3DD0E9480440E94FC43FDCFEF92FF920F931F93CF93DF93F2
:2089E0008C017B01EA010CC0D7016D917D01D801ED91FC910190F081E02DC8010995219751
:208A0000209791F7DF91CF911F910F91FF90EF900895DF93CF9300D0CDB7DEB7DC018DE045
:208A200089838AE08A83ED91FC9111970480F581E02DCD01BE016F5F7F4F42E050E00995E0
:208A40000F900F90CF91DF9108954F925F926F927F928F929F92AF92BF92CF92DF92EF9250
:208A6000FF920F931F93DF93CF93CDB7DEB7A1970FB6F894DEBF0FBECDBF3C016A017B0181
:208A8000222349F4DC01ED91FC910190F081E02D642F099550C0213009F42AE0C114D1041A
:208AA000E104F10421F480E389A310E229C010E2822E9924AA24BB242E010894411C511CBC
:208AC000C701B601A50194010E9482CD6A3010F4605D01C0695CF201E10FF11D6083C7016E
:208AE000B601A50194010E9482CDC901DA016C017D01C114D104E104F10411F01150E0CF6E
:208B0000002331F01150FE01E10FF11D8DE28183812F90E0D301ED91FC91BE016F5F7F4FE6
:208B2000680F791F41E250E0481B590B0480F581E02DC3010995A1960FB6F894DEBF0FBEB1
:208B4000CDBFCF91DF911F910F91FF90EF90DF90CF90BF90AF909F908F907F906F905F90B4
:208B60004F9008950F9377FD02C000E008C070956095509541955F4F6F4F7F4F0DE22AE011
:208B800064DF0F9108954F925F926F927F928F929F92AF92BF92CF92DF92EF92FF920F9307
:208BA0001F93DF93CF93CDB7DEB728970FB6F894DEBF0FBECDBF3C017A018B01522ECB0180
:208BC000BA0120E030E040E050E05FD387FD02C0442406C017FB109517F910954424439429
:208BE00020E030E040E05FE3DD240AC0CA01B9012DEC3CEC4CEC5DE36DD69B01AC01D39407
:208C0000D514A0F3C801B70167D24B015C01B1D36B017C01C301B701A6012AE0042D15DFB6
:208C2000552009F447C0C701B601CFD39B01AC01C501B40150D29B01AC018EE28983D52CEE
:208C400087E0851510F487E0D82EBD2CCC24C3944E010894811C911C1FC0CA01B90120E0D9
:208C600030E040E251E436D67B018C0182D3F401EC0DF11D605D60836053C39470E088277E
:208C800077FD8095982FA3D39B01AC01C801B70122D29B01AC01BA94BB20F9F6D301ED919D
:208CA000FC91D3940480F581E02DC301B4014D2D50E0099528960FB6F894DEBF0FBECDBFF3
:208CC000CF91DF911F910F91FF90EF90DF90CF90BF90AF909F908F907F906F905F904F90E0
:208CE0000895CF93DF93DB010D900020E9F71197A61BB70BEC01E881F9810480F581E02D88
:208D0000AD010995DF91CF910895FC019FB7F89480916B11882311F420E010C083E0809338
:208D2000E9002091F200222349F48091E80082FF05C085FD03C08BE68093E8009FBF8781CF
:208D4000908597FD03C02F3F09F02F5F822F90E00895CF93DF93EC018F81988597FF09C0A7
:208D6000E881F9810084F185E02DCE01099598878F838F819885DF91CF910895FC0127812C
:208D8000308537FD05C08FEF9FEF9087878322C02FB7F89480916B11882369F083E080939D
:208DA000E9009BE68091E80085FD09C082FF03C09093E800F7CF2FBF2FEF3FEF0CC09091C9
:208DC000F1008091E80085FD03C08BE68093E8002FBF292F30E0C9010895FC0180916B11B1
:208DE000882371F09FB7F89483E08093E9002BE602C02093E8008091E80085FDFACF9FBF16
:208E00008FEF9FEF9087878308950F931F93CF93DF93EB0180916B11882309F4D5C03FB7B4
:208E2000F89484E08093E90080915E11882309F4C0C08091E80085FFC6C010925E11B9C011
:208E40009091E400915F8091E80085FD13C03FBF8091E400891721F481E080935E11B4C0D0
:208E600080916B11882309F4AFC03FB7F8940093E900E9CF8091F200212F281B822F90E0E1
:208E80004817590708F4242FE0E4E21BE03428F4EE0FFF27E25BF843099480C089918C9322
:208EA00089918C9389918C9389918C9389918C9389918C9389918C9389918C9389918C93EA
:208EC00089918C9389918C9389918C9389918C9389918C9389918C9389918C9389918C93CA
:208EE00089918C9389918C9389918C9389918C9389918C9389918C9389918C9389918C93AA
:208F000089918C9389918C9389918C9389918C9389918C9389918C9389918C9389918C9389
:208F200089918C9389918C9389918C9389918C9389918C9389918C9389918C9389918C9369
:208F400089918C9389918C9389918C9389918C9389918C9389918C9389918C9389918C9349
:208F600089918C9389918C9389918C9389918C9389918C9389918C9389918C9389918C9329
:208F800089918C9389918C9389918C9389918C9389918C9389918C9389918C938091E80049
:208FA00085FD02C07093E800421B510960935C1106C004E010E4A1EFB0E07AE363E04115B7
:208FC000510509F03DCF3FBFDF91CF911F910F910895E0E6F1E189E0DF011D928A95E9F7EC
:208FE00088EE93E0A0E0B0E08093621190936311A0936411B09365111092661182EA93E002
:2090000090936111809360110895CF93DF93DB010D900020E9F71197A61BB70BEC01E881CC
:20902000F9810480F581E02DAD010995DF91CF9108952FEF3FEFFC01308727839FDA0FB60E
:20904000F8948091571190915811A0915911B0915A110FBEAC0180916B11882329F068EC1B
:2090600070E080E090E0B5C980916C11882309F10FB6F8948091571190915811A091591130
:20908000B0915A110FBE9C0110C00FB6F8948091571190915811A0915911B0915A110FBE82
:2090A000821B930B8B3F9105A8F480916C11882361F70FB6F8948091571190915811A09163
:2090C0005911B0915A110FBE841B950B855C994008F4C1CF08955058BB27AA270ED081C20F
:2090E00041D230F046D220F031F49F3F11F41EF411C20EF4E095E7FBDCC1E92F94D280F341
:20910000BA17620773078407950718F071F49EF5C3C20EF4E0950B2EBA2FA02D0B01B901C3
:2091200090010C01CA01A0011124FF27591B99F0593F50F4503E68F11A16F040A22F232F87
:20914000342F4427585FF3CF469537952795A795F0405395C9F77EF41F16BA0B620B730BFA
:20916000840BBAF09150A1F0FF0FBB1F661F771F881FC2F70EC0BA0F621F731F841F48F458
:20918000879577956795B795F7959E3F08F0B3CF9395880F08F09927EE0F97958795089523
:2091A000E1D158F080E891E009F49EEFE2D128F040E851E059F45EEF09C0ACC16DC2E92F17
:2091C000E07831D268F3092E052AC1F3261737074807590738F00E2E07F8E02569F0E025CF
:2091E000E0640AC0EF6307F8009407FADB01B9019D01DC01CA01AD01EF935DD0F2D10AD0A5
:209200005F91552331F02BED3FE049E450FD49EC63CF0895DF93DD27B92FBF7740E85FE312
:209220001616170648075B0710F4D92FA1D29F938F937F936F9305D4E8E9F0E06ED1D1D1F2
:209240002F913F914F915F9151D3DD2349F09058A2EA2AED3FE049EC5FE3D0785D274DDF38
:20926000DF91BFC102D280F09F3740F491110EF414C260E070E080E89FE3089526F01B16D8
:20928000611D711D811D1BC135C1EFD008F481E0089577D1E395B6C10CD0A3C16AD140F0B7
:2092A00061D130F021F45F3F19F003C15111F5C131C1B9D198F39923C9F35523B1F3951B79
:2092C000550BBB27AA2762177307840738F09F5F5F4F220F331F441FAA1FA9F333D00E2E9F
:2092E0003AF0E0E830D091505040E695001CCAF729D0FE2F27D0660F771F881FBB1F2617CD
:2093000037074807AB07B0E809F0BB0B802DBF01FF2793585F4F2AF09E3F510568F0C9C05D
:20932000BCC15F3FECF3983EDCF3869577956795B795F7959F5FC9F7880F911D9695879549
:2093400097F90895E1E0660F771F881FBB1F621773078407BA0720F0621B730B840BBA0BF5
:20936000EE1F88F7E095089504D06894B11195C1089561D188F09F5790F0B92F9927B751FA
:20938000A0F0D1F0660F771F881F991F1AF0BA95C9F712C0B13081F07FD1B1E008957CC11A
:2093A000672F782F8827B85F39F0B93FCCF3869577956795B395D9F73EF49095809570951E
:2093C00061957F4F8F4F9F4F0895E89409C097FB3EF490958095709561957F4F8F4F9F4F88
:2093E0009923A9F0F92F96E9BB279395F695879577956795B795F111F8CFFAF4BB0F11F4E6
:2094000060FF1BC06F5F7F4F8F4F9F4F16C0882311F096E911C0772321F09EE8872F762F4C
:2094200005C0662371F096E8862F70E060E02AF09A95660F771F881FDAF7880F9695879510
:2094400097F9089512D180F09F3740F491110EF024C160E070E080E89FEB089526F41B1693
:20946000611D711D811D2BC045C0990F0008550FAA0BE0E8FEEF16161706E807F907C0F0EC
:2094800012161306E407F50798F0621B730B840B950B39F40A2661F0232B242B252B21F442
:2094A00008950A2609F4A140A6958FEF811D811D089597F99F6780E870E060E00895882399
:2094C00071F4772321F09850872B762F07C0662311F499270DC09051862B70E060E02AF01F
:2094E0009A95660F771F881FDAF7880F9695879597F908959F3F49F0915028F48695779574
:209500006795B7959F5F80389F4F880F9695879597F908959FEF80EC0895DF93CF931F9337
:209520000F93FF92EF92DF927B018C01689405C0DA2EEF01DBD1FE01E894A591259135916B
:2095400045915591AEF3EF01D8DDFE019701A801DA9479F7DF90EF90FF900F911F91CF91BE
:20956000DF91089500240A941616170618060906089500240A941216130614060506089544
:20958000C9CF59D0E8F3E894EFEFBB273FE048EC5FE76B3D73078407950708F1FF279F57FC
:2095A000B25A6A4D7F40894CF04032F4BE556542704F8643FF4F0894EE1F915030F0BB0FFA
:2095C000661F771F881FFF1FEBCF9EE7882332F0BB0F661F771F881F9A95C1F79395E0958F
:2095E00089CF092E0394000C11F4882352F0BB0F40F4BF2B11F460FF04C06F5F7F4F8F4FBD
:209600009F4F0895EF93E0FF06C0A2EA2AED3FE049EC5FEB72DDE5DF0F90039401FC905829
:20962000E5ECF0E018C257FD9058440F551F59F05F3F71F04795880F97FB991F61F09F3F78
:2096400079F087950895121613061406551FF2CF4695F1DF08C0161617061806991FF1CF06
:2096600086957105610508940895E5DFA0F0BEE7B91788F4BB279F3860F41616B11D672FD8
:20968000782F8827985FF7CF869577956795B11D93959639C8F30895E894BB2766277727EE
:2096A000CB0197F90895E1DE08F48FEF08955ADF19F05FDF09F02ECFFCCEB901CA011ACF2D
:2096C0009F775F77B0DF98F39923B9F35523B9F3FF27951758F4E52FE91BED3070F75E3BA5
:2096E00010F0F1E41CC09034E0F40AC0E92FE51BED3028F79E3B10F0F1E411C0503488F484
:20970000F9EA88232AF09A95660F771F881FDAF744232AF05A95220F331F441FDAF79F1B0E
:209720005F1BFF931F930F93FF92EF9279018A01BB27AB2F9B01AC01DBD09701A801BF936F
:209740007B018C01AA27BA2FB901CA01D1D0AF919701A801EF90FF900F911F91CEDC41DF77
:2097600026D14F9140FF0895552747FD509509C09B01AC0160E070E080E89FE38DCD99CE44
:20978000B9CE59DFE8F39923D9F3940F511DBBF39150504094F059F0882332F0660F771FD2
:2097A000881F91505040C1F79E3F510544F7880F911D9695879597F908955F3FACF0983EA2
:2097C0009CF0BB27869577956795B79508F4B1609395C1F7BB0F58F711F460FFE8CF6F5FBD
:2097E0007F4F8F4F9F4FE3CF58CF0EF083CE92CE68945FCE20DFC8F39923D1F3C6F3DF93B9
:20980000CF931F930F93FF92C92FDD2788232AF02197660F771F881FDAF720E030E040E8CD
:209820005FEB9FE3883920F0803E30F021968F7753DCE3EEF0E003C04FDCE0E1F1E06DDE55
:209840008B01BE01EC01FB2E6F5771097595771F880B990BBCDD28E132E741E35FE346D059
:20986000AF2D9801AE01FF900F911F91CF91DF9144DCB7CEE0DE58F19E5758F19851A0F0B2
:20988000E9F0983020F5092E9927660F771F881F991F0A94D1F712C0062E672F782F882759
:2098A000985F11F4000C07C0993FB4F38695779567959395D9F7611D711D811D3EF490953E
:2098C0008095709561957F4F8F4F9F4F08956894E4CEE2CE0BD085CE45DE28F04ADE18F04A
:2098E000952309F0E6CD16CE1124D7CE9CDEA0F3959FD1F3950F50E0551F629FF001729FF6
:20990000BB27F00DB11D639FAA27F00DB11DAA1F649F6627B00DA11D661F829F2227B00D7C
:20992000A11D621F739FB00DA11D621F839FA00D611D221F749F3327A00D611D231F849F4F
:20994000600D211D822F762F6A2F11249F5750408AF0E1F088234AF0EE0FFF1FBB1F661F08
:20996000771F881F91505040A9F79E3F510570F0A0CD93CE5F3FECF3983EDCF386957795EF
:209980006795B795F795E7959F5FC1F7FE2B880F911D9695879597F908959F93F2DD0F903F
:2099A00007FCEE5F2FCE11F40EF4B4CDA3CD43DED0F39923D9F3CEF39F57550B87FF44D045
:2099C00056959795B0E020F4660F771F881FBB1F1F930F9300249001A0018001F001A0E89C
:2099E0000E0F1F1F0A1E511D601B710B8009B50B48F4600F711F801DB51F0E1B1F0B0A0A23
:209A0000510907C02E0F3F1F4A1F0E0F1F1F0A1E511D660F771F881FBB1FA695F795E79561
:209A2000F8F60617170708065B07211D311D411D0F911F91B901842F9158880F969587951F
:209A400008959B01AC0146CF91505040660F771F881FD2F708959F938F937F936F93FF9388
:209A6000EF939B01AC0136DFEF91FF9156DD2F913F914F915F912ECF629FD001739FF00191
:209A8000829FE00DF11D649FE00DF11D929FF00D839FF00D749FF00D659FF00D9927729F7D
:209AA000B00DE11DF91F639FB00DE11DF91FBD01CF0111240895AA1BBB1B51E107C0AA1F41
:209AC000BB1FA617B70710F0A61BB70B881F991F5A95A9F780959095BC01CD01089597FBCC
:209AE000092E07260AD077FD04D0E5DF06D000201AF4709561957F4F0895F6F7909581958A
:209B00009F4F0895A1E21A2EAA1BBB1BFD010DC0AA1FBB1FEE1FFF1FA217B307E407F50761
:209B200020F0A21BB30BE40BF50B661F771F881F991F1A9469F760957095809590959B0153
:209B4000AC01BD01CF01089597FB092E05260ED057FD04D0D7DF0AD0001C38F450954095A1
:209B6000309521953F4F4F4F5F4F0895F6F790958095709561957F4F8F4F9F4F0895EE0F9D
:209B8000FF1F0590F491E02D099491110EC0803219F089508550D0F7089591110895815492
:209BA0008A5108F4805E855A08959927882708952F923F924F925F926F927F928F929F92A0
:209BC000AF92BF92CF92DF92EF92FF920F931F93CF93DF93CDB7DEB7CA1BDB0B0FB6F894B2
:209BE000DEBF0FBECDBF09942A88398848885F846E847D848C849B84AA84B984C884DF8074
:209C0000EE80FD800C811B81AA81B981CE0FD11D0FB6F894DEBF0FBECDBFED0108951AE133
:209C2000C8EFDAE103C0FE01ACDF2296CA3FD107D1F7F894FFCF2F0043616E6E6F74206F89
:209C400070656E207375626469720000004D31303420496E76616C69642065787472756493
:209C6000657220004D31303520496E76616C696420657874727564657220004D3130392069
:209C8000496E76616C696420657874727564657220004D32313820496E76616C69642065F6
:209CA000787472756465722000003F005265706F7274696E6720656E6473746F7020737459
:209CC00061747573006F70656E00545249474745524544004D32303020496E76616C6964B2
:209CE00020657874727564657220006F6B0020703A0020693A0020643A0020633A0054007B
:209D0000496E76616C6964206578747275646572004163746976652045787472756465721A
:209D20003A2000537465707261746520746F6F20686967683A200000504944204175746F5F
:209D400074756E65206661696C65642E20426164206578747275646572206E756D62657231
:209D60002E00504944204175746F74756E65207374617274000000FA440000FA4400002079
:209D80004200000000640064000000803F00004D4300004D43000039430101983A0000008A
:209DA00080BB440100007A4300005243CDCCCC3D000020410101010101C40F5C12FB4F0737
:209DC0003EC40F5C12FB4F073E0000B0411EE1343EFF082B440000803F0000204120F0402D
:209DE0003BFF1E1545FF3F0108FF3F5261706964426F74332072656164792E000000000081
:209E00006E8A026D1100E10000000008282300002823000064000000102700000000FA4373
:209E20000000FA4300004040000034420000A0420000A042004085445AE4B54258595A459D
:209E4000000001000000010027002300FFFF0200030026002500FFFF040005001700240026
:209E6000FFFFFFFF140010000600070013001500DBFFD9FFD9FFDAFF00000000A4699A691A
:209E8000EAC4000E1315110E00001C10181705060500001C1F11111F00000006191803138B
:209EA0000C00040E1F041C000000040A0A0A0A11110E0C12120C00000000001F1511151F34
:209EC000000000000000BBBD71C6EAC4000040001400540000000000721305C805C785C614
:209EE000BEC6A9C6EDC6FFFFFFFFFFFFFFFFFFFFFFFFFFFFFFFFFFFFFFFFFFFFFFFFFFFFD6
:209F0000FFFFFFFFFFFFFFFFFFFFFFFFFFFFFFFFFFFFFFFFFFFFFFFFFFFFFFFFFFFFFFFF61
:209F2000FFFFFFFFFFFFFFFFFFFFFFFFFFFFFFFFFFFFFFFFFFFFFFFFFFFFFFFFFFFFFFFF41
:209F4000FFFFFFFFFFFFFFFFFFFFFFFFFFFFFFFFFFFFFFFFFFFFFFFFFFFFFFFFFFFFFFFF21
:209F6000FFFFFFFFFFFFFFFFFFFFFFFFFFFFFFFFFFFFFFFFFFFFFFFFFFFFFFFFFFFFFFFF01
:20F000004BC0000066C0000064C0000062C0000060C000005EC000005CC000005AC0000005
:20F0200058C0000056C00000B9C4000052C0000050C000004EC000004CC000004AC00000DF
:20F0400048C0000046C0000044C0000042C0000041C000003EC000003CC000003AC00000A7
:20F0600038C0000036C0000034C0000032C0000030C000002EC000002CC000002AC0000008
:20F0800028C0000026C0000024C0000022C0000020C000001EC0000011241FBECFEFD0E29C
:20F0A000DEBFCDBF11E0A0E0B1E0EEEAFEEF01E00BBF02C007900D92AC38B107D9F711E060
:20F0C000ACE8B1E001C01D92AA39B107E1F778D0ECC696CF1F920F920FB60F9211240F903D
:20F0E0000FBE0F901F90189584E08093E9000DC08091E8008B778093E80003C08EB3882376
:20F1000051F08091E80082FFF9CF8091E80085FFEFCF8091F1000895982F83E08093E9006C
:20F120008091E80085FD0DC08091E8008E778093E80003C08EB3882331F08091E80080FF46
:20F14000F9CF9093F100089590919201892F8F77813249F5809193018032A1F0813219F52A
:20F16000913A09F58091E800877F8093E80088E091E067E070E0C7D48091E8008B778093B3
:20F18000E8000895913279F48091E800877F8093E80088E091E067E070E011D58091E80071
:20F1A0008E778093E800089582E061EC42E06AD383E061E842E166D384E060E842E162C3A8
:20F1C0002F923F924F925F926F927F928F929F92AF92BF92CF92DF92EF92FF920F931F939D
:20F1E000DF93CF9300D000D0CDB7DEB784B7877F84BF88E10FB6F8948093600010926000CF
:20F200000FBE80E090E020E80FB6F89420936100809361000FBE11E015BF82E085BFA8D3BD
:20F2200010936F0083E080938100789479E0672E8FC224E02093E9008091E80082FF87C217
:20F2400053DF182F853419F410920F0103C0843519F44ADF8DE051C28C34E1F38035D1F37E
:20F26000843711F484E49AC0813611F489E545C28134F1F439DF382E330C222471010027A5
:20F28000F7FC0095102FE0928C01F0928D0100938E0110938F0128DF90E0880F991FAA27AC
:20F2A00097FDA095BA2F8E299F29A02BB12BF6C1803711F483E521C2833559F400E011E0E2
:20F2C000D8018D918D0128DFB1E007301B07C1F715C2863521F481E31FDF80E30EC283370A
:20F2E00031F482E819DF87E917DF8EE106C2853629F580E090E0A0E0B0E023E0FC01A093FE
:20F300005B0020935700E89507B600FCFDCF35E0FC01A0935B0030935700E89507B600FC96
:20F32000FDCF80509F4FAF4FBF4F803060EF960761E0A60760E0B60701F78CCF8C3649F45E
:20F34000D3DE8095E1E0F0E0082E60925700E89581CF823731F4E1E0F0E06092570084913D
:20F36000CCC1863431F4E0E0F0E0609257008491C4C18E3431F4E3E0F0E0609257008491D6
:20F38000BCC1813531F4E2E0F0E0609257008491B4C1823631F489E5BFDE81E0BDDE80E06C
:20F3A000ACC1823419F0873609F0F5C09DDE082F9BDEF82E99DE882E8554823008F09CC158
:20F3C0000A8319822F2D30E089819A81282B392B3C832B83173609F055C091E19093570009
:20F3E000E895DD2449C0E0908C01F0908D0100918E0110918F01A6E48A1609F58D2D90E0D8
:20F40000A0E0B0E08E299F29A02BB12BABBFFC01879182DEDD2081F082E090E0A0E0B0E087
:20F42000E80EF91E0A1F1B1FE0928C01F0928D0100938E0110938F0191E0D92618C0D801D7
:20F44000C701B695A7959795879519D565DE82E090E0A0E0B0E0E80EF91E0A1F1B1FE09220
:20F460008C01F0928D0100938E0110938F01AB81BC811197BC83AB83EB81FC81EF2B09F020
:20F48000B2CF3CC1A0908C01B0908D01C0908E01D0908F01F6E48F1609F067C023E0F501FC
:20F4A000C0925B0020935700E89507B600FCFDCF5CC036E4831681F5992049F1E0908C015E
:20F4C000F0908D0100918E0110918F010DDE582E4424872D90E08429952961E00C01F7011F
:20F4E00000935B0060935700E895112482E090E0A0E0B0E0E80EF91E0A1F1B1FE0928C01D1
:20F50000F0928D0100938E0110938F0102C0ECDD782E91E0992623C0E0908C01F0908D0137
:20F5200000918E0110918F0116950795F794E794DBDD682FC701ABD480918C0190918D014A
:20F54000A0918E01B0918F010296A11DB11D80938C0190938D01A0938E01B0938F01AB81E4
:20F56000BC811197BC83AB8302C077249924EB81FC81EF2B09F09DCFF6E48F1609F06ACE07
:20F5800025E0F501C0925B0020935700E89507B600FCFDCF5FCE8334A1F4E0908C01F090C1
:20F5A0008D0100918E0110918F019EDD90E031E00C01F70100935B0030935700E8951124B1
:20F5C00049CE833639F5E0908C01F0908D0100918E0110918F0188DDA8019701216090E03A
:20F5E00061E00C01F90140935B0060935700E895112482E090E0A0E0B0E0E80EF91E0A1F81
:20F600001B1FE0928C01F0928D0100938E0110938F0120CE8D3699F480918C0190918D01C1
:20F62000A0918E01B0918F0125E0FC01A0935B0020935700E89507B600FCFDCF0BCE82350D
:20F6400081F4E0908C01F0908D0100918E0110918F010BBFF701E790F6908F2D5DDD8E2D69
:20F660004CC0843421F5E0908C01F0908D0100918E0110918F0116950795F794E79434DDF6
:20F68000682FC70104D480918C0190918D01A0918E01B0918F010296A11DB11D80938C0191
:20F6A00090938D01A0938E01B0938F01D3CD843609F5E0908C01F0908D0100918E011091E0
:20F6C0008F01D801C701B695A79597958795D7D323DD82E090E0A0E0B0E0E80EF91E0A1F68
:20F6E0001B1FE0928C01F0928D0100938E0110938F0104C08B3111F08FE30EDD93E09093F8
:20F70000E9009091E8008091E8008E778093E80095FF04C010C08EB38823C9F08091E80038
:20F7200080FFF9CF8091E8008E778093E80003C08EB3882361F08091E80080FFF9CFA4E0C5
:20F74000A093E9008091E8008B778093E80085D380910F01882309F06CCD8091E00081606F
:20F760008093E0002CE088E190E00FB6F894A895809360000FBE20936000FFCF9B01AC01B9
:20F7800007B600FCFDCFF999FECF83E0F90140935B0080935700E89581E180935700E895CA
:20F7A00008959B01AC0107B600FCFDCFF999FECF85E0F90140935B0080935700E89581E1A9
:20F7C00080935700E89508950F931F938B019C0107B600FCFDCFF999FECF81E00A01F801DF
:20F7E00020935B0080935700E89511241F910F91089521E2FC01209357002491822F0895E5
:20F8000029E0FC01209357002491822F0895E1E0F0E089E08093570084910895982F07B63B
:20F8200000FCFDCFF999FECF909589E0E1E0F0E0092E80935700E8950895FA01923071F0A9
:20F84000933089F0913029F480E191E022E130E015C080E090E020E030E010C082E291E04F
:20F860002EE330E00BC0882329F480E691E024E030E004C084E691E026E230E0918380831B
:20F88000C90108958093E9008091EB0081608093EB001092ED006093EC004093ED008091EB
:20F8A000EE00881F8827881F08958091920188238CF403C08EB38823B1F08091E80082FF27
:20F8C000F9CF8091E8008B778093E80008958EB3882349F08091E80080FFF9CF8091E8006F
:20F8E0008E778093E8000895EF92FF920F931F9348D04FD008ED10E0F80180818F778083E6
:20F9000080818068808380818F7D8083E7EDF0E080818068808319BC1EBA1092900180EE0D
:20F92000E82EF12CF70180818B7F8083F80180818160808380E060E042E0A4DFE1EEF0E0CC
:20F9400080818E7F8083E2EEF0E0808181608083808188608083F70180818E7F8083F80123
:20F960008081806180831F910F91FF90EF900895E7EDF0E080818160808381E08093910118
:20F98000B3CFE8EDF0E080818C7F80831092E20008951092DA001092E10008951F920F9222
:20F9A0000FB60F920BB60F9211242F933F934F935F936F937F938F939F93AF93BF93EF9364
:20F9C000FF938091DA0080FF1BC08091D80080FF17C08091DA008E7F8093DA008091D90042
:20F9E00080FF0BC084E189BD86E189BD09B400FEFDCF81E08EBB30D203C019BC1EBA2CD2C4
:20FA00008091E10080FF17C08091E20080FF13C08091E2008E7F8093E2008091E200806190
:20FA20008093E2008091D80080628093D80019BC85E08EBB11D28091E10084FF2CC0809143
:20FA4000E20084FF28C084E189BD86E189BD09B400FEFDCF8091D8008F7D8093D800809189
:20FA6000E1008F7E8093E1008091E2008F7E8093E2008091E20081608093E2008091900144
:20FA8000882331F48091E30087FD02C081E001C084E08EBBE1D18091E10083FF21C0809175
:20FAA000E20083FF1DC08091E100877F8093E10082E08EBB109290018091E1008E7F809329
:20FAC000E1008091E2008E7F8093E2008091E20080618093E20080E060E042E0D3DEBCD187
:20FAE000FF91EF91BF91AF919F918F917F916F915F914F913F912F910F900BBE0F900FBED2
:20FB00000F901F9018959C0140919801509199014617570718F4F90190E03CC0611571054F
:20FB200011F0AB01F8CF8091E8008E778093E80040E050E0F0CF8EB38823E9F18530E9F1F4
:20FB40008091E80083FF02C081E008958091E80082FD2BC08091E80080FF1CC02091F20010
:20FB60003091F30007C081918093F100415050402F5F3F4F4115510519F02830310598F3E9
:20FB800090E02830310509F491E08091E8008E778093E8004115510571F6992361F605C015
:20FBA0008EB3882341F0853041F08091E80082FFF7CF80E0089582E0089583E008959C0169
:20FBC0006115710529F48091E8008B778093E800F90121C08EB3882369F1853069F18091E5
:20FBE000E80083FF02C081E008958091E80082FFF1CF06C08091F10081936150704031F043
:20FC00008091F2009091F300892BA1F78091E8008B778093E80061157105E1F605C08EB3C2
:20FC2000882341F0853041F08091E80080FFF7CF80E0089582E0089583E008950F931F9374
:20FC4000DF93CF9300D0CDB7DEB7E2E9F1E08091F100819381E0EA39F807C9F775DA809192
:20FC6000E80083FFE4C08091920190919301953009F46DC0963040F4913081F1913070F0E0
:20FC8000933009F0D4C02AC0983009F4A3C0993009F4B2C0963009F0CAC07CC0803809F490
:20FCA000C6C0823809F0C3C0809196018F708093E9008091EB001092E9002091E800277F1F
:20FCC0002093E80090E025E0969587952A95E1F781708093F1001092F10087C0882319F0B3
:20FCE000823009F0A4C08F71823009F0A0C080919401882331F5209196012F7009F497C038
:20FD00002093E9008091EB0080FF1BC0933021F48091EB00806213C08091EB008061809378
:20FD2000EB0081E090E002C0880F991F2A95E2F78093EA001092EA008091EB0088608093DE
:20FD4000EB001092E9008091E800877F51C0882309F06DC0109194011F770FB7F89480911D
:20FD6000E800877F8093E800A0DD8091E80080FFFCCF8091E3008078812B8093E300806864
:20FD80008093E300112311F482E001C083E08EBB0FBF4DC08058823008F049C08091940159
:20FDA0009091950160919601AE014F5F5F4F45DDBC01009709F43BC08091E800877F809379
:20FDC000E80089819A819FDE8091E8008B778093E8002DC0803859F58091E800877F80939E
:20FDE000E800809190018093F1008091E8008E778093E8005ADD1BC08823C9F4909194014C
:20FE00009230A8F48091E800877F8093E800909390014BDD80919001882331F48091E30048
:20FE200087FD02C081E001C084E08EBBBDD98091E80083FF0AC08091EB0080628093EB00F6
:20FE40008091E800877F8093E8000F900F90CF91DF911F910F91089508951F938EB3882372
:20FE600061F01091E9001092E9008091E80083FF01C0E4DE1F701093E9001F910895F99924
:20FE8000FECF92BD81BDF89A992780B50895262FF999FECF1FBA92BD81BD20BD0FB6F8949C
:20FEA000FA9AF99A0FBE01960895F894FFCF4C5546414344430000000000000008011201B2
:20FEC000100102000008EB034A2000010001000109023E000201008032090400000102029C
:20FEE00001000524001001042402060524060001070582030800FF09040100020A000000B5
:20FF000007050402100001070583021000010403090426034100560052002000430044004F
:20FF20004300200042006F006F0074006C006F0061006400650072000000FFFFFFFFFFFF59
:20FF4000FFFFFFFFFFFFFFFFFFFFFFFFFFFFFFFFFFFFFFFFFFFFFFFFFFFFFFFFFFFFFFFFC1
:20FF6000FFFFFFFFFFFFFFFFFFFFFFFFFFFFFFFFFFFFFFFFFFFFFFFFFFFFFFFFFFFFFFFFA1
:20FF8000FFFFFFFFFFFFFFFFFFFFFFFFFFFFFFFFFFFFFFFFFFFFFFFFFFFFFFFFFFFFFFFF81
:20FFA000FFFFFFFFFFFFFFFFFFFFFFFFFFFFFFFFFFFFFFFFFFFFFFFFFFFFFFFFFFFFFFFF61
:20FFC000FFFFFFFFFFFFFFFFFFFFFFFFFFFFFFFFFFFFFFFFFFFFFFFFFFFFFFFFFFFFFFFF41
:20FFE000CDCBDFCBF1CB05CC0BCC11CC17CC00000000000000000000000000000000FBDCC4
:020000040001F9
:200000000C94ED0A0C94180B0C94180B0C94180B0C94180B0C94180B0C94180B0C94180BF4
:200020000C94180B0C94180B0C949F8F0C94198E0C94180B0C94180B0C94180B0C94180B19
:200040000C94180B0C94736E0C94180B0C94180B0C94180B0C94180B0C944B760C94E28CE1
:200060000C94180B0C94180B0C94180B0C94180B0C94180B0C94180B0C94180B0C94180B68
:200080000C94180B0C94180B0C94180B0C94180B0C94180B0C94180B084AD73B3BCE016EF2
:2000A00084BCBFFDC12F3D6C74319ABD56833DDA3D00C77F11BED9E4BB4C3E916BAAAABE5D
:2000C000000000803F05A84CCDB2D44EB93836A9020C50B9918688083CA6AAAA2ABE00001B
:2000E00000803F4D3834205820592045006563686F3A0043616E6E6F7420656E7465722098
:200100007375626469723A20004D3234004D3233202573006175746F25692E6700457272DA
:200120006F723A006572726F722077726974696E6720746F2066696C65004E6F74205344AB
:20014000207072696E74696E67002F005344207072696E74696E67206279746520002E00A1
:2001600044656C6574696F6E206661696C65642C2046696C653A200046696C652064656CCB
:20018000657465643A002E006F70656E206661696C65642C2046696C653A20005772697452
:2001A000696E6720746F2066696C653A20002E006F70656E206661696C65642C2046696C18
:2001C000653A20002E006F70656E206661696C65642C2046696C653A200046696C652073C2
:2001E000656C6563746564002053697A653A200046696C65206F70656E65643A20002E0071
:200200006F70656E206661696C65642C2046696C653A200053442063617264206F6B006FC7
:2002200070656E526F6F74206661696C656400766F6C756D652E696E6974206661696C65B7
:200240006400534420696E6974206661696C006563686F3A0048617264636F646564204458
:20026000656661756C742053657474696E6773204C6F616465640053746F726564207365BA
:200280007474696E67732072657472696576656400205A0020590020204D3938205800482A
:2002A00079737465726573697320286D6D293A002044002049002020204D33303120500050
:2002C0005049442073657474696E67733A00205A0020590020204D323036205800486F6DC2
:2002E00065206F666673657420286D6D293A00204500205A00205800204200205400202000
:200300004D323035205300416476616E636564207661726961626C65733A20533D4D696E89
:2003200020666565647261746520286D6D2F73292C20543D4D696E2074726176656C20663B
:200340006565647261746520286D6D2F73292C20423D6D696E696D756D207365676D656E70
:20036000742074696D6520286D73292C20583D6D6178696D756D205859206A65726B202825
:200380006D6D2F73292C20205A3D6D6178696D756D205A206A65726B20286D6D2F73292C58
:2003A0002020453D6D6178696D756D2045206A65726B20286D6D2F73290020540020204D5E
:2003C000323034205300416363656C65726174696F6E3A20533D616363656C657261746953
:2003E0006F6E2C20543D7265747261637420616363656C65726174696F6E00204500205A65
:200400000020590020204D3230312058004D6178696D756D20416363656C65726174696F71
:200420006E20286D6D2F7332293A00204500205A0020590020204D3230332058004D6178DD
:20044000696D756D2066656564726174657320286D6D2F73293A00204500205A0020590092
:2004600020204D393220580053746570732070657220756E69743A0053657474696E67732B
:200480002053746F7265640020653D00207A3D0020793D00205348494654533A783D00205C
:2004A0004500205A00205900483D58006563686F3A004572726F723A005072696E74657226
:2004C0002073746F707065642064756520746F206572726F72732E204669782074686520E9
:2004E0006572726F7220616E6420757365204D39393920746F20726573746172742E20285C
:2005000054656D70657261747572652069732072657365742E20536574206974206166743C
:2005200065722072657374617274696E6729005072696E7465722068616C7465642E206B29
:20054000696C6C28292063616C6C656421006F6B00526573656E643A20002200556E6B6E10
:200560006F776E20636F6D6D616E643A2022007A5F6D696E3A2000795F6D61783A20007845
:200580005F6D696E3A20005A3A00593A0020436F756E7420583A2000453A005A3A00593A96
:2005A00000583A004D616368696E652D547970653A20506978696520382C204669726D7723
:2005C0006172652D56657273696F6E3A20312E302E3134303731346120202020416C6C206E
:2005E0005269676874732052657365727665642C20506F6C6172203344204C4C430A002024
:20060000423A0020453A00543A0020573A0020453A00543A002042403A0020403A00202F8E
:200620000020423A00202F006F6B20543A002569206D696E2C2025692073656300456E6409
:200640002066696C65206C69737400426567696E2066696C65206C697374000000C8420073
:2006600000B44300001643000020410000000000002041FF00FF000000000000B443000073
:2006800000000000000000000000000000000000C8420000B44300001643256920686F7506
:2006A0007273202569206D696E7574657300446F6E65207072696E74696E672066696C65B1
:2006C000005072696E7465722073746F707065642064756520746F206572726F72732E20AB
:2006E00046697820746865206572726F7220616E6420757365204D39393920746F20726556
:2007000073746172742E202854656D70657261747572652069732072657365742E20536562
:20072000742069742061667465722072657374617274696E6729006F6B004E6F204C696EB0
:2007400065204E756D626572207769746820636865636B73756D2C204C617374204C696E39
:20076000653A20004E6F20436865636B73756D2077697468206C696E65206E756D6265725D
:200780002C204C617374204C696E653A2000636865636B73756D206D69736D617463682C82
:2007A000204C617374204C696E653A20004C696E65204E756D626572206973206E6F7420E5
:2007C0004C617374204C696E65204E756D6265722B312C204C617374204C696E653A200016
:2007E0004D31313000446F6E6520736176696E672066696C652E006F6B004D32390020202C
:20080000506C616E6E657242756666657242797465733A20002046726565204D656D6F728B
:20082000793A2000417567203131203230313400436F6D70696C65643A20007069786965B9
:200840007072696E746572736C6C6300207C20417574686F723A200041756720313120326C
:200860003031342031363A34383A323900204C61737420557064617465643A2000312E308D
:200880002E30004D61726C696E200020536F6674776172652052657365740020576174633A
:2008A00068646F67205265736574002042726F776E206F757420526573657400204578745F
:2008C00065726E616C20526573657400506F7765725570007374617274002200656E717508
:2008E00065696E672022002200656E717565696E672022007C3C3E5E2B3D3F2F5B5D3B2C0A
:200900002A225C0045313A200045303A20005A3A2000593A2000583A20004D53312C4D53DA
:20092000322050696E730A0024F404D9201BC40C5C0E9804C4095F0265077101F405F900BD
:20094000FB04B30048048700C10369005803550003034500BE023A008402310053022A00BA
:200960002902250004022000E4011C00C8011900AF01170098011400840113007101100090
:200980006101100051010E0043010D0036010B002B010B0020010B00150109000C0109005A
:2009A00003010800FB000800F3000800EB000700E4000600DE000600D8000600D2000600B7
:2009C000CC000500C7000500C2000500BD000400B9000400B5000400B1000400AD00040016
:2009E000A9000400A5000300A20003009F0004009B000300980003009500020093000300F4
:200A0000900003008D0002008B000300880002008600020084000300810002007F00020089
:200A20007D0002007B000200790002007700010076000200740002007200010071000200F3
:200A40006F0002006D0001006C0002006A000100690002006700010066000100650001003E
:200A6000640002006200010061000100600001005F0002005D0001005C0001005B00010072
:200A80005A000100590001005800010057000100560001005500010054000100530000009B
:200AA000530001005200010051000100500001004F0001004E0000004E0001004D000100B1
:200AC0004C0001004B0000004B0001004A00010049000100480000004800010047000100C4
:200AE0004600000046000100450000004500010044000100430000004300010042000000D0
:200B0000420001004100000041000100400001003F0000003F0001003E0000003E000100D2
:200B20003D0000003D0001003C0000003C0000003C0001003B0000003B0001003A000000D4
:200B40003A00010039000000390001003800000038000000380001003700000037000100CF
:200B60003600000036000000360001003500000035000000350001003400000034000000CA
:200B80003400010033000000330000003300010032000000320000003200010031000000BE
:200BA00031000000310001003000000030000000300001002F0000002F0000002F000000B4
:200BC0002F0001002E0000002E0000002E0001002D0000002D0000002D0000002D000100A5
:200BE0002C0000002C0000002C0000002C0001002B0000002B0000002B0000002B00010097
:200C00002A0000002A0000002A0000002A0001002900000029000000290000002900000087
:200C2000290001002800000028000000280000002800000028000100270000002700000073
:200C400027000000270000002700010026000000260000002600000026000000260001005F
:200C600025000000250000002500000025000000250000002500010024000000240000004D
:200C8000240000002400000024000100230000002300000023000000230000002300000038
:200CA000230000002300010022000000220000002200000022000000220000002200010020
:200CC00021000000210000002100000021000000210000002100000021000100200000000C
:200CE000200000002000000020000000200000002000000020000000200001001F000000F4
:200D00001F0000001F0000001F0000001F0000001F0000001F0001001E0000001E000000DC
:200D20001E0000001E00000024F4D43050C38E20C2A24017828B7011127A910D816CD90A57
:200D4000A861E108C7586607615143061E4B5D05C145A7041A411104093D9803713931036F
:200D60004036DB0265339102D4305402802E1D02632CEE01752AC501B028A00110278101B9
:200D80008F2564012B244B01E0223401AC211F018D200D01801FFC00841EED00971DDF0003
:200DA000B81CD200E61BC600201BBC00641AB200B219A8000A19A0006A189900D1179100D5
:200DC00040178B00B516840031167E00B31579003A157300C7146F0058146A00EE13660093
:200DE0008813630025135E00C7125B006C12570015125400C111510070114F0021114B006B
:200E0000D61049008D1047004610440002104200C00F4000800F3E00420F3C00060F3B0018
:200E2000CB0E3800930E37005C0E3500270E3400F30D3200C10D3100900D3000600D2E0028
:200E4000320D2D00050D2C00D90C2B00AE0C2900850C29005C0C2700350C27000E0C260004
:200E6000E80B2400C40B2400A00B23007D0B23005A0B2100390B2100180B2000F80A1F00A0
:200E8000D90A1E00BB0A1E009D0A1D00800A1D00630A1C00470A1B002C0A1B00110A1A0088
:200EA000F7091A00DD091900C4091900AB091900920917007B091800630917004C0916002A
:200EC00036091600200916000A091500F5081500E0081400CC081400B8081400A4081400CC
:200EE000900813007D0812006B0813005808120046081200340811002308110012081100A4
:200F000001081100F0071000E0071000D0071000C0071000B0070F00A107100091070E00D7
:200F200083070F0074070F0065070E0057070E0049070E003B070D002E070E0020070D0084
:200F400013070D0006070D00F9060C00ED060D00E0060C00D4060C00C8060C00BC060C00C5
:200F6000B0060C00A4060B0099060C008D060B0082060B0077060B006C060B0061060A00A8
:200F800057060B004C060A0042060A0038060A002E060A0024060A001A060A001006090038
:200FA00007060A00FD050900F4050900EB050900E2050900D9050900D0050900C70509008A
:200FC000BE050900B5050800AD050800A50509009C050800940508008C05080084050800A2
:200FE0007C050800740508006C050700650508005D050700560508004E0507004705070084
:201000004005080038050700310507002A050700230507001C050600160507000F05070039
:201020000805060002050700FB040600F5040700EE040600E8040600E2040700DB040600CE
:20104000D5040600CF040600C9040600C3040600BD040600B7040600B1040500AC04060040
:20106000A6040600A00405009B04060095040500900406008A04050085040500800406008F
:201080007A04050075040500700405006B04050066040500610405005C04050057040500C4
:2010A000520405004D04050048040500430405003E0404003A0405003504050030040400E3
:2010C0002C04050027040400230405001E0404001A04040016040500110404000D040400EB
:2010E000090405000404040000040400FC030400F8030400F4030400F0030400EC030400E3
:20110000E8030400E4030400E0030400DC030400D8030400D4030400D0030400CC030400C7
:20112000C8030300C50303006563686F3A00205A3A0020593A0020583A00656E6473746F97
:201140007073206869743A20004572726F723A0054656D7065726174757265206865617459
:20116000656420626564207377697463686564206F66662E204D415854454D5020747269AC
:20118000676765726564202121003A204578747275646572207377697463686564206F6662
:2011A000662E204D494E54454D50207472696767657265642021003A204578747275646508
:2011C00072207377697463686564206F66662E204D415854454D50207472696767657265E4
:2011E00064202100202D20496E76616C6964206578747275646572206E756D626572202199
:2012000000504944204175746F74756E652066696E6973686564202120506C616365207438
:201220006865204B702C204B6920616E64204B6420636F6E7374616E747320696E207468F4
:201240006520636F6E66696775726174696F6E2E6800504944204175746F74756E65206623
:2012600061696C6564212074696D656F75740020403A006F6B20543A006F6B20423A00503F
:201280004944204175746F74756E65206661696C6564212054656D706572617475726520D8
:2012A000746F206869676800204B643A2000204B693A2000204B703A200020436C617369F3
:2012C000632050494420002054753A2000204B753A2000206D61783A2000206D696E3A2093
:2012E0000020643A200020626961733A200070012C0190012701B0012201C0011D01F001FC
:2013000018011002130130020E016002090190020401C002FF000003FA004003F5008003D1
:20132000F000D003EB002004E6007004E100E004DC004005D700C005D2004006CD00D00644
:20134000C8008007C3003008BE00F008B900C009B400B00AAF00B00BAA00D00CA500000EFA
:20136000A000500F9B00C01096005012910000148C00C0158700B0178200B0197D00D01B04
:201380007800001E730040206E0090226900F024640040275F0090295A00E02B5500102E6C
:2013A000500020304B0010324600E033410090353C001037370070383200A0392D00B03A1D
:2013C0002800A03B2300603C1E00103D1900903D1400103E0F00703E0A00C03E0500003F8F
:2013E00000002000204163743A2000526F643A2000205761726E696E672120496E636F6E8E
:2014000073697374656E7420706172616D657465727321002070756C732000207065726979
:201420006F642028572920002070686173652028502920005A576F62626C6520416D7020CC
:201440002841292000437573746F6D20776F62626C652066756E6374696F6E0001290229E9
:20146000042908291029202940298029012C022C01260226042608261026202640268026F0
:20148000402C802C012302230423082310232023402380230120022004200820102020201E
:2014A00040208020102C202C012F022F042F082F102F202F402F802F7EFE7EFD7EFB7EF748
:2014C0007EEF7EDF7EBF7E7F00010000FC1412000200000E15430003000051150401030903
:2014E00004551518020309046F15160303090487150C0001C10201803601813612010002B7
:2015000002000020C016830400010102030109024300020100C032090400000102020100EE
:20152000052400100105240100010424020605240600010705820308004009040100020AF3
:2015400000000007050302400000070584024000000403090418035400650065006E00733A
:201560000079006400750069006E006F00000016035500530042002000530065007200691D
:201580000061006C0000000C03310032003300340035000000494E46494E4954594E414E29
:2015A000CDCCCC3D0AD7233C17B7D13877CC2B329595E6241FB14F0A000020410000C8420A
:2015C00000401C4620BCBE4CCA1B0E5AAEC59D74B826B72888860C93B22811241FBECFEF9E
:2015E000D0E2DEBFCDBF13E0A0E0B1E0E2EFF1E301E00BBF02C007900D92A234B107D9F766
:201600001BBE10E1A2E4B3E001C01D92A333B107E1F715E1C8EDD5E104C02297FE010E9492
:201620009F98C03DD107C9F70E941D900C94ED980C940000A0E0B0E0E0E2FBE00C94BC9829
:20164000EC015B016115710519F0FB0191838083F9908F2D90E00E94A398892BC9F7FDE254
:20166000FF1621F4F990EE24E39405C02BE2F21609F4F990EE248E0101501040C80165E975
:2016800075E143E050E069D2892BF9F48E010E5F1F4FC80168E975E145E050E05ED2892BB2
:2016A00019F48E01095F1F4FA114B10419F0F50111830083E0FC04C070E090E080E813C09D
:2016C00070E090E080E86FEF07C1C8016DE975E143E050E042D2892B69F4A114B10429F448
:2016E00070E090E080EC6FE7F7C02296F501D183C083F6CF8824992440E050E060E070E05E
:20170000EF2DE053EA30A0F5F2E0EF2A8E2D90E09C0128703070E2FE06C0232B79F50894E2
:20172000811C911C2BC0232B19F0089481089108DB01CA0112E0880F991FAA1FBB1F1A9525
:20174000D1F7480F591F6A1F7B1F440F551F661F771F4E0F511D611D711D483929E952072A
:2017600029E9620729E1720748F084E0E82A06C0EE3F31F4E3FC39C098E0E92AF990C0CF2A
:20178000E53311F0E53189F529912D3219F4E0E1EE2A05C02B3219F081E090E003C0299124
:2017A00082E090E0E22FE053EA3018F0C81BD90B1CC020E030E0FCE020383F075CF4C901AA
:2017C000880F991F880F991F280F391F220F331F2E0F311DE991E053EA3068F3E4FE03C007
:2017E000309521953F4F820E931ECE2CDD24E1FE07C0A114B10421F02197F501D183C0833E
:20180000CB01BA010E9408957B018C01F3E0CF22DD2423E0C216D10421F417FB109517F9A8
:20182000109557016801C801B70120E030E040E050E00E946894882309F44AC097FE0DC0AF
:2018400024EBE22E25E1F22E9094819491089394C0E2D0E000E010E012C09CECE92E95E141
:20186000F92EF6CFF7012591359145915491C601B5010E9448975B016C018C1A9D0A8C1697
:201880009D0684F7D595C7950F5F1F4F0630110529F08CEF9FEFE80EF91EF1CFC501D601B0
:2018A0007C018D018C2D880F8D2D881F8F3F51F0C601B50120E030E040E050E00E946894E2
:2018C000882331F482E290E090933210809331107E2D9F2D802F612F272F392F482F562F3B
:2018E000B901CA01CDB7DEB7ECE00C94D8982F923F925F926F927F928F929F92AF92BF92F5
:20190000CF92DF92EF92FF920F931F93CF93DF938C011B01EA016115710519F0FB01918322
:201920008083209749F0CE010297839728F020E030E040E050E0F6C0F801A1908F018A2D93
:2019400090E00E94A398892BB9F7FDE2AF1631F4F801A1908F015524539407C0FBE2AF168A
:2019600019F4F801A1908F015524209719F0C031D105C1F4F0E3AF1679F4F801808188372D
:2019800011F0883549F4F801A1800E5F1F4FF2E05F2AC0E1D0E006C0209721F480E3A816F8
:2019A000E9F427C0C830D10531F1C930D10524F4C230D10531F50CC0CA30D10589F0C03198
:2019C000D105F9F4C12CD12CE12CB8E0FB2E28C0C12CD12CE12CA0E4FA2E22C0CAE0D0E0C5
:2019E000FCECCF2EFCECDF2EFCECEF2EFCE0FF2E17C0C8E0D0E0C12CD12CE12CE0E1FE2EEC
:201A00000FC09E01442737FD4095542F60E070E080E090E80E944C98C901DA016C017D01E3
:201A200020E030E040E050E060E03E01882477FC8094982C70EDB72EBA0CE9E0EB1570F49B
:201A40008A2D81548A3118F499ECB92E06C08A2D81568A3150F589EAB82EBA0C8B2D90E02C
:201A60008C179D0714F56F3FE1F0C216D306E406F506B0F0CA01B901A40193010E941A984F
:201A80009B01AC012B0D311D411D511D2130F0E03F07F0E04F07F0E85F0710F461E001C0DA
:201AA0006FEFF801A1908F01C5CF2114310481F0662331F001501040F1011183008308C083
:201AC00051FE1AC002501040F1011183008314C067FF12C050FC05C02FEF3FEF4FEF5FE745
:201AE00004C020E030E040E050E882E290E0909332108093311016C050FE08C05095409587
:201B0000309521953F4F4F4F5F4F0CC057FF0AC082E290E090933210809331102FEF3FEFAB
:201B20004FEF5FE7B901CA01DF91CF911F910F91FF90EF90DF90CF90BF90AF909F908F90C4
:201B40007F906F905F903F902F900895FB01DC0105900D920020E1F70895FB01DC01415051
:201B6000504088F08D9181341CF08B350CF4805E659161341CF06B350CF4605E861B6111D8
:201B800071F3990B0895881BFCCFFB0155915523A9F0BF01DC014D9145174111E1F759F4F1
:201BA000CD010590002049F04D9140154111C9F3FB014111EFCF81E090E001970895FB011A
:201BC000DC0104C08D910190801921F441505040C8F7881B990B0895FB01DC0102C0019017
:201BE0000D9241505040D8F70895FB01DC010D900020E9F7119701900D920020E1F70895D6
:201C0000FC018191861721F08823D9F7992708953197CF010895FB01DC0101900D920020D1
:201C2000E1F70895FB01DC014150504030F08D910190801919F40020B9F7881B990B08950C
:201C4000FB01DC014150504048F001900D920020C9F701C01D9241505040E0F70895AEE0AF
:201C6000B0E0E5E3FEE00C94C4980D891E898EE08C831A8309838FEF9FE79E838D839E017B
:201C8000275E3F4FCE0101966F89788DA9010AD02F813885020F131FF80110822E96E4E087
:201CA0000C94E098ABE0B0E0E8E5FEE00C94B6983C012B015A01FC0117821682838181FDE4
:201CC00003C06FEF7FEFB9C19AE0892E1E010894211C311CF3012381F20123FD859123FFA2
:201CE00081912F01882309F4A5C1853239F423FD859123FF81912F01853221F490E0B30126
:201D0000B7D1E8CF982FFF24EE249924FFE1FF15D0F09B3269F09C3228F4903259F0933237
:201D200091F40EC09D3249F0903369F441E024C052E0F52A84E0F82A28C098E0F92A25C0E4
:201D4000E0E1FE2A22C0F7FC29C0892F80538A3070F4F6FE05C0989C902C1124980E15C0DA
:201D6000E89CE02C1124E80EF0E2FF2A0EC09E3229F4F6FC5FC140E4F42A07C09C3619F4F8
:201D800050E8F52A02C0983649F4F20123FD959123FF91912F01992309F0B8CF892F8554A5
:201DA000833018F08052833038F444E050E0A40EB51E5FE359830FC0933631F0933779F0D4
:201DC000933509F052C01FC0F5018081898342E050E0A40EB51E610101E010E011C0F5017D
:201DE000C080D180F6FC03C06FEF7FEF02C0692D70E042E050E0A40EB51EC6012ED18C01FF
:201E00005FE7F52213C0F501C080D180F6FC03C06FEF7FEF02C0692D70E042E050E0A40EDE
:201E2000B51EC6010FD18C0150E8F52AF3FE06C018C080E290E0B3011BD1EA948E2D90E09A
:201E400008171907B0F30DC0F601F7FC8591F7FE81916F0190E0B3010BD1E110EA9401509C
:201E600010400115110581F7E2C0943611F0993661F5F7FE08C0F50120813181428153813F
:201E800084E090E00AC0F501808191819C01442737FD4095542F82E090E0A80EB91E9FE623
:201EA000F92257FF09C050954095309521953F4F4F4F5F4FE0E8FE2ACA01B901A1012AE0B8
:201EC00030E002D1D82ED2183FC0953729F41F2D1F7E2AE030E01DC01F2D197F9F3661F05D
:201EE000903720F4983509F0A5C00FC0903739F0983709F09FC004C028E030E00AC01061DF
:201F000014FD146020E130E004C014FD166020E132E017FF08C0F50160817181828193810F
:201F200044E050E008C0F50180819181BC0180E090E042E050E0A40EB51EA101C5D0D82EDB
:201F4000D2188FE7F82EF122F6FE0BC05EEFF522D91438F4F4FE07C0F2FC05C08FEEF822A9
:201F600002C01D2D01C0192DF4FE0DC0FE01ED0DF11D8081803319F499EEF92208C01F5FDF
:201F8000F2FE05C003C08F2D867809F01F5F0F2DF3FC13C0F0FE0EC01E1510F09D2C0AC018
:201FA0009D2C9E0C911A1E2D05C080E290E0B3015FD01F5F1E15C8F304C01E1510F4E11ADC
:201FC00001C0EE2404FF0EC080E390E0B30150D002FF1BC001FD03C088E790E00EC088E5FF
:201FE00090E00BC0802F867881F001FF02C08BE201C080E2F7FC8DE290E0B30139D005C0E2
:2020000080E390E0B30134D09A94D914C8F3DA94F101ED0DF11D808190E0B30129D0DD20DC
:20202000B1F705C080E290E0B30122D0EA94EE20C9F750CEF30166817781CB012B96E2E12E
:202040000C94D298FC010590615070400110D8F7809590958E0F9F1F0895FC016150704013
:2020600001900110D8F7809590958E0F9F1F08950F931F93CF93DF938C01EB018B8181FF90
:202080001BC082FF0DC02E813F818C819D812817390764F4E881F9810193F983E88306C082
:2020A000E885F985802F0995892B31F48E819F8101969F838E8302C00FEF1FEFC801DF910F
:2020C000CF911F910F910895FA01AA27283051F1203181F1E8946F936E7F6E5F7F4F8F4FA6
:2020E0009F4FAF4FB1E03ED0B4E03CD0670F781F891F9A1FA11D680F791F8A1F911DA11D65
:202100006A0F711D811D911DA11D20D009F468943F912AE0269F11243019305D3193DEF683
:20212000CF010895462F4770405D4193B3E00FD0C9F7F6CF462F4F70405D4A3318F0495DA2
:2021400031FD4052419302D0A9F7EACFB4E0A6959795879577956795BA95C9F70097610595
:20216000710508959B01AC010A2E06945795479537952795BA95C9F7620F731F841F951F78
:20218000A01D0895DF93CF930F92CDB7DEB7FC016983A081B18114962D913C911597BE017B
:2021A0006F5F7F4F41E050E0F90109950F90CF91DF910895FC0111AA14AA27E233E030AB21
:2021C00027A7E05BFF4F1082339610823597318320837F9610823396108235973183208373
:2021E0007F961082339610823597318320837E9689E18083339610827896108239961082DD
:20220000339610823597318320837D96108211821282138238961082118212821382ED5E78
:20222000F0401282138210821182EF50FF4F81E08083E15FF04016A615A60FB6F8948091E6
:202240001F1090912010A0912110B09122100FBEE751FF4F88579C4EAF4FBF4F80839183EA
:20226000A283B3830895FC01128213820895FC018381882311F081E082830895FC018281F3
:20228000811112820895FC0187E293E0918380838581882321F0CF0102960C94F7600895CD
:2022A0000F931F93CF93DF938C010E94616E0E943E6EC80186539F4F0E94F760F801128294
:2022C00083EE90E00E943D468091E006882301F11092E00680919A04C82FD0E0CC0FDD1FAF
:2022E000C05ED14F68817981882777FD8095982F0E940A9520918C0230918D0240918E028D
:2023000050918F020E947696181614F419821882DF91CF911F910F910895EF92FF920F93C1
:202320001F938C013AECE32EF12CE80EF91EC7010E94A960C7010E94F760F80110821182AB
:202340001F910F91FF90EF900895CF92DF92EF92FF920F931F93CF93DF937C016B01DB01B1
:202360000D900020E9F78D0101501040061B170BEAECF0E0EE0EFF1ED7011C92E6E3FFEF52
:20238000EE0EFF1ECB016EE470E03ADCEC01009731F4F8013197EC0DFD1D86010CC060E28E
:2023A00070E02EDC8C010F5F1F4FCE016AE270E027DCFC0131978DE081838AE082831382B2
:2023C000C70188539F4FB8010E94C2688AEC90E0E80EF91ED7018C918823F1F0EDE1F1E0D4
:2023E0006491EF0106C088E290E1CCDE2196FE0164916623C1F7E4E2F1E06491EF0106C07F
:2024000088E290E1BFDE2196FE0164916623C1F788E290E16AE0B6DEDF91CF911F910F917F
:20242000FF90EF90DF90CF900895EF92FF920F93CF93DF937C01FC018381882309F43DC078
:20244000ECE4F1E06491EF0106C088E290E19ADE2196FE0164916623C1F78DEE90E0E80E10
:20246000F91EF701408151816281738183E19FEFE80EF91E88E290E12AE000E00E945E908F
:20248000EAE4F1E06491EF0106C088E290E17ADE2196FE0164916623C1F785EE90E0E80EFA
:2024A000F91EF701408151816281738188E290E12AE000E00E945E900DC0EAE3F1E06491EE
:2024C000EF0106C088E290E15DDE2196FE0164916623C1F788E290E16AE054DEDF91CF911D
:2024E0000F91FF90EF9008952F923F924F925F926F927F928F929F92AF92BF92CF92DF9265
:20250000EF92FF920F931F93DF93CF93CDB7DEB7AB970FB6F894DEBF0FBECDBF5C014B0136
:202520004BA7FC018381882309F4C9C15AEC452E512C4A0C5B1CC2010E94F760F50112822D
:20254000188A1B8A87E293E09F878E874CE4C42ED12CCA0CDB1C2FE230E0A20EB31EF60198
:20256000B182A08221ED3FEFA20EB31EF40180818F3209F083C0C4016FE270E041DB7C0157
:202580000894E11CF11C3E010894611C711C160170C0C7016FE270E033DB6C01009709F4F1
:2025A0007BC0E816F90608F077C08C010E191F09C301B701A80144DB060D171DF8011082C2
:2025C000E0912810F09129100280F381E02D88E290E1B301099588E290E16AE0D3DDF101A1
:2025E000608171816115710519F460E070E002C06E5F7F4FCE014096A30121E00E94C96706
:20260000882361F5E0E0F2E064917F0108C088E290E1B8DD0894E11CF11CF701649166235E
:20262000B1F7E0912810F09129100280F381E02D88E290E1BE016F5F7F4F0995EEEFF1E00A
:2026400064917F0108C088E290E19CDD0894E11CF11CF70164916623B1F72AC12EE030E01C
:202660002C0F3D1FF1013183208376010894E11CF11CE114F10409F08CCF0BC08EE490E072
:20268000A80EB91EF601B182A08222EB3FEFA20EB31E082DD92C02C00E2DDF2CF501E45B2E
:2026A000FF4F3BA5332309F4A9C0608171816115710519F460E070E002C06E5F7F4FC201B4
:2026C000402F5D2D21E00E94C967882309F46BC0A5014B515F4F8BED90E0A80EB91EF50100
:2026E00080819181A281B38125E23FEFA20EB31EFA0180839183A283B383E0EFF1E06491B8
:202700007F0108C088E290E13DDD0894E11CF11CF70164916623B1F7E0912810F091291055
:202720000280F381E02D88E290E1602F7D2D0995E8EEF1E064917F0108C088E290E122DD26
:202740000894E11CF11CF70164916623B1F725EE30E0A20EB31EF5014081518162817381B1
:2027600088E290E12AE000E00E945E9088E290E16AE008DD28E030E0A20EB31EF5011082D9
:20278000118212821382EAEDF1E064917F0108C088E290E1F7DC0894E11CF11CF701649157
:2027A0006623B1F785C0E6ECF1E064917F0108C088E290E1E7DC0894E11CF11CF701649192
:2027C0006623B1F7E0912810F09129100280F381E02D88E290E1602F7D2D0995E4ECF1E00F
:2027E00064917F0108C088E290E1CCDC0894E11CF11CF70164916623B1F75AC06081718168
:202800006115710519F460E070E002C06E5F7F4FC201402F5D2D26E50E94C967882359F540
:20282000E0EBF1E064917F0108C088E290E1AADC0894E11CF11CF70164916623B1F7E09129
:202840002810F09129100280F381E02D88E290E1602F7D2D0995EEEAF1E064917F0108C0EB
:2028600088E290E18FDC0894E11CF11CF70164916623B1F71DC081E0F5018083ECE9F1E071
:2028800064917F0108C088E290E17CDC0894E11CF11CF70164916623B1F7E0912810F091DA
:2028A00029100280F381E02D88E290E1B401099588E290E16AE066DCCE010E96E4DCAB96D3
:2028C0000FB6F894DEBF0FBECDBFCF91DF911F910F91FF90EF90DF90CF90BF90AF909F90F8
:2028E0008F907F906F905F904F903F902F900895FC0181E08183CF0140E0F6CD2F923F920B
:202900004F925F926F927F928F929F92AF92BF92CF92DF92EF92FF920F931F93DF93CF93E3
:20292000CDB7DEB7AA970FB6F894DEBF0FBECDBF5C014B01FC018381882309F426C1C501F7
:2029400086539F4F0E94F760F5011282188A1B8A87E293E09F878E877CE4C72ED12CCA0CA7
:20296000DB1C2FE230E0A20EB31EF601B182A08221ED3FEFA20EB31EF40180818F3209F005
:2029800087C0C4016FE270E03BD97C010894E11CF11C3E010894611C711C260160E1262EB2
:2029A000312C2C0E3D1E6FC0C7016FE270E028D96C01009709F47AC0E816F90608F076C026
:2029C0008C010E191F09C301B701A80139D9060D171DF8011082E0912810F091291002802D
:2029E000F381E02D88E290E1B301099588E290E16AE0C8DBF201608171816115710519F4A2
:202A000060E070E002C06E5F7F4FC101A30121E00E94C967882361F5E8E8F1E064917F0179
:202A200008C088E290E1AEDB0894E11CF11CF70164916623B1F7E0912810F09129100280C1
:202A4000F381E02D88E290E1BE016F5F7F4F0995E6E8F1E064917F0108C088E290E192DBFD
:202A60000894E11CF11CF70164916623B1F786C02EE030E02C0F3D1FF201318320837601D6
:202A80000894E11CF11CE114F10409F08DCF0BC08EE490E0A80EB91EF601B182A08222EBBE
:202AA0003FEFA20EB31ED82C092D02C0DE2C0F2D8CE490E0A80EB91EF5018081918124EBA0
:202AC0003FEFA20EB31E009719F480E090E001C002966D2D702F0E949568882329F1E8E70E
:202AE000F1E064917F0108C088E290E14BDB0894E11CF11CF70164916623B1F7E09128105A
:202B0000F09129100280F381E02D88E290E16D2D702F09952DEE30E0A20EB31EF501108212
:202B20001182128213822EC0E0E6F1E064917F0108C088E290E126DB0894E11CF11CF7019D
:202B400064916623B1F7E0912810F09129100280F381E02D88E290E16D2D702F0995EEE564
:202B6000F1E064917F0108C088E290E10BDB0894E11CF11CF70164916623B1F788E290E1E7
:202B80006AE000DBCE010E967EDBAA960FB6F894DEBF0FBECDBFCF91DF911F910F91FF900E
:202BA000EF90DF90CF90BF90AF909F908F907F906F905F904F903F902F900895EF92FF92D3
:202BC0000F931F93CF93DF937C01FC01138284A9882321F0C701C1960E94F76087010B55D5
:202BE0001F4FC80160E048E00E94C15E8823D9F4EDEEF0E06491EF0106C088E290E1C2DA30
:202C00002196FE0164916623C1F7E2E4F2E06491EF0106C088E290E1B5DA2196FE01649170
:202C20006623C1F76BC0E701C655DF4FCE01B80141E00E945369882311F5CE01B80140E097
:202C40000E9453698823D9F4EDE1F1E06491EF0106C088E290E196DA2196FE0164916623D5
:202C6000C1F7EFE2F2E06491EF0106C088E290E189DA2196FE0164916623C1F73FC0C7015D
:202C8000C196BE010E94CE638823D9F4EDE1F1E06491EF0106C088E290E174DA2196FE01AA
:202CA00064916623C1F7EFE1F2E06491EF0106C088E290E167DA2196FE0164916623C1F789
:202CC0001DC081E0F7018383EDEEF0E06491EF0106C088E290E156DA2196FE016491662323
:202CE000C1F7E4E1F2E06491EF0106C088E290E149DA2196FE0164916623C1F788E290E115
:202D00006AE040DAD701A05BBF4FF701F1968BE101900D928150E1F7C7018F962CE430E09D
:202D2000E20EF31EF70191838083DF91CF911F910F91FF90EF9008952F923F924F925F9254
:202D40006F927F929F92AF92BF92CF92DF92EF92FF920F931F93DF93CF93CDB7DEB7CC5558
:202D6000D0400FB6F894DEBF0FBECDBF8C01662319F50F501F4FD8018C91015F10408823BA
:202D800009F4E6C00FB6F89420911F103091201040912110509122100FBE07511F4FF801CD
:202DA00080819181A281B381095E104082179307A407B50708F4CCC00F501F4FD8011C927C
:202DC000015F1040F8018381882341F4C801F6DED80113968C91882309F4BAC000D000D068
:202DE00000D0EDB7FEB731966E010894C11CD11CADB7BEB71296DC92CE92119784E191E041
:202E000093838283D8019D968D919C919E97958384830E942F0E7601EDB7FEB736960FB6AC
:202E2000F894FEBF0FBEEDBF56010AC0D7018C91992787FD90950E94AB98F70181937F01E0
:202E4000F50101900020E9F73197EA19FB098E2D8C198E175CF3B1E3AB2EB12CA00EB11E01
:202E6000C50140E050E060E070E00E94DF5F9924ADE3CA2ED12CCC0EDD1E2E010894411C8D
:202E8000511CFFE16F2E712C6C0E7D1EEDE02E2EE1E03E2E43C0D7018C9190E00E94AB98F3
:202EA000F70181937F01D6010D900020E9F71197AC19BD098E2D8C198A176CF327968FAD86
:202EC00027978E3759F1C601B20145E050E00E94120E009719F500D000D000D0EDB7FEB726
:202EE0003196ADB7BEB712967C926E92119733822282558244820E942F0EEDB7FEB73696DA
:202F00000FB6F894FEBF0FBEEDBFC3010E94B44689E091E00E943D4699249394C501B6016A
:202F200040E050E00E94ED62181614F47601BBCF992041F48FEF9FEFD8019E969C938E93C2
:202F40009D9706C0F80185A596A5019696A785A7C45ADF4F0FB6F894DEBF0FBECDBFCF9126
:202F6000DF911F910F91FF90EF90DF90CF90BF90AF909F907F906F905F904F903F902F908E
:202F800008952F923F924F925F926F927F928F929F92AF92BF92CF92DF92EF92FF920F93B4
:202FA0001F93DF93CF93CDB7DEB7CB58D0400FB6F894DEBF0FBECDBF7C012B015A0182E092
:202FC00090E0A80EB91EF7017196CB57DF4FF983E883C558D040C7010496CE57DF4F9983C0
:202FE0008883C258D040CC57DF4F1882C458D04092E6C92ED12CCC0EDD1EF6013B96C9575C
:20300000DF4FF983E883C758D04082EF682E712C6E0C7F1C04EF802E912C8E0C9F1C1EE002
:20302000212E312C2C0E3D1E85E490E08C0F9D1F0296C757DF4F99838883C958D040EDEE08
:20304000F0E09491C557DF4F9883CB58D0403EC1F6018385482F50E0BA0168717070603139
:20306000710509F041C1F301208131812130310509F43AC12230310509F436C1F601DE01C7
:2030800011969081903239F08E2F8C19883011F48EE28D939D933196C957DF4F8881998176
:2030A000C758D040E817F90761F71C921E86F2018081882329F4C10160E071E00E94F50D85
:2030C000C101B2010E94F50DC101BE016F5F7F4F0E94F50DC10160E071E00E94F50D1AA65F
:2030E0001DA687E293E099A788A7CE018A96B501AE014F5F5F4F21E00E94C9678823B9F5E6
:20310000F30180819181892B91F5C557DF4F6881CB58D0400DEE10E007C088E290E132D871
:203120000F5F1F4FF80164916623B9F7E0912810F09129100280F381E02D88E290E162E009
:2031400071E0099588E290E16AE01CD8E0912810F09129100280F381E02D88E290E1BE0167
:203160006F5F7F4F099588E290E16AE00BD8C757DF4FA881B981C958D040FE01BA968BE172
:2031800001900D928150E1F787E293E027969FAF8EAF2797C701B101AE014B5B5F4FF1DE28
:2031A000CE018B5B9F4F6FD8CE0188966CD88EC0953E09F48BC09E3209F488C09F3509F4A5
:2031C00085C0F7019189992331F09E3209F47EC09F3509F47BC043FD79C080E060317105C4
:2031E00009F481E0F70184A7882349F4F6018085873409F06BC081858E3709F467C0CE5777
:20320000DF4FA881B981C258D040F6018081803241F08E2F8C19883011F48EE28D93808168
:203220008D933196C957DF4F88819981C758D040E817F90759F71C92F3018081918100976C
:2032400009F5E0912810F09129100280F381E02D88E290E1B2010995E0912810F09129107B
:203260000280F381E02D88E290E1CE57DF4F68817981C258D040099588E290E16AE00E94AB
:20328000C21024C08130910539F4F401808191810196918380831AC00297C1F4CC57DF4FD5
:2032A000F881C458D0402F2F30E0F4018081918128173907F1F0CC57DF4FF881C458D0409D
:2032C000FF5FCC57DF4FF883C458D040C501B601CB57DF4F48815981C558D0400E94ED620A
:2032E00018160CF4B5CE05C0F6019081992309F05FCFC557DF4F0FB6F894DEBF0FBECDBFDC
:20330000CF91DF911F910F91FF90EF90DF90CF90BF90AF909F908F907F906F905F904F90F9
:203320003F902F900895EF92FF920F931F93DF93CF93CDB7DEB76D970FB6F894DEBF0FBE50
:20334000CDBF7C0182EF90E0E80EF91EF701118210828EE09FEFE80EF91E87010F5C1F4FEF
:20336000C80140E050E060E070E00E94DF5FDE011396F8018BE101900D928150E1F787E295
:2033800093E09A838983C70165E171E08E010F5F1F4FA801F6DDC8010E9443116D960FB6C4
:2033A000F894DEBF0FBECDBFCF91DF911F910F91FF90EF9008950F931F93DF93CF93CDB714
:2033C000DEB7E0970FB6F894DEBF0FBECDBFDE011196E7EDF2E080E101900D928150E1F734
:2033E000DE015196E7ECF2E080E101900D928150E1F7DE019196E7EBF2E080E101900D92ED
:203400008150E1F789819A81AB81BC818093840690938506A0938606B093870689899A8966
:20342000AB89BC898093740690937506A0937606B093770689A19AA1ABA1BCA180939406BE
:2034400090939506A0939606B09397068D819E81AF81B8858093880690938906A0938A064F
:20346000B0938B068D899E89AF89B88D8093780690937906A0937A06B0937B068DA19EA1A7
:20348000AFA1B8A58093980690939906A0939A06B0939B0689859A85AB85BC8580938C0612
:2034A00090938D06A0938E06B0938F06898D9A8DAB8DBC8D80937C0690937D06A0937E0607
:2034C000B0937F0689A59AA5ABA5BCA580939C0690939D06A0939E06B0939F068D859E8597
:2034E000AF85B8898093900690939106A0939206B09393068D8D9E8DAF8DB8A180938006DA
:2035000090938106A0938206B09383068DA59EA5AFA5B8A98093A0069093A106A093A206F2
:20352000B093A3060E942B4C80E090E0AAE7B4E48093A8069093A906A093AA06B093AB0623
:2035400080E090E8ABE3B5E48093AC069093AD06A093AE06B093AF0620E030E040E050E092
:203560002093A4063093A5064093A6065093A70680E29EE4A0E0B0E080937006909371065A
:20358000A0937206B09373062093BC063093BD064093BE065093BF0680E090E0A0E2B1E4A3
:2035A0008093B0069093B106A093B206B093B3068DEC9CECACECBEE38093B4069093B5069C
:2035C000A093B606B093B70680E090E0A0EAB0E48093B8069093B906A093BA06B093BB0664
:2035E00020938A0430938B0440938C0450938D042093860430938704409388045093890407
:20360000209382043093830440938404509385048AE999E9A1EBB1E48093990290939A02DD
:20362000A0939B02B0939C0261E77DE38AE89FE30E94B57560939D0270939E0280939F0288
:203640009093A00260E070E084EE92E40E94C1756093A1027093A2028093A3029093A40297
:2036600082E493E060E070E020E030E040E050E00E94962482E493E061E070E020E030E0AB
:2036800040E050E00E94962482E493E062E070E020E030E040E050E00E9496240E948475BC
:2036A00080E090E0A0E8BFE38093A5029093A602A093A702B093A802EFE4F2E064918F0198
:2036C00008C088E290E10E94C2100F5F1F4FF80164916623B1F7E5E5F2E064918F0108C0EF
:2036E00088E290E10E94C2100F5F1F4FF80164916623B1F788E290E16AE00E94C210E09671
:203700000FB6F894DEBF0FBECDBFCF91DF911F910F9108950F931F93CF93DF930FE412E098
:20372000F8016491E80107C088E290E10E94C2102196FE0164916623B9F7E8E6F4E0649121
:20374000EF0107C088E290E10E94C2102196FE0164916623B9F788E290E16AE00E94C210E6
:20376000F8016491CFE4D2E007C088E290E10E94C2102196FE0164916623B9F740918406A1
:2037800050918506609186067091870680E694E00E94582E409188065091890660918A0660
:2037A00070918B068DE594E00E94582E40918C0650918D0660918E0670918F068AE594E094
:2037C0000E94582E4091900650919106609192067091930687E594E00E94582EE09128100E
:2037E000F09129100280F381E02D88E290E166E171E0099588E290E16AE00E94C210F80169
:203800006491CFE4D2E007C088E290E10E94C2102196FE0164916623B9F7EDE3F4E06491BB
:20382000EF0107C088E290E10E94C2102196FE0164916623B9F788E290E16AE00E94C21005
:20384000F8016491CFE4D2E007C088E290E10E94C2102196FE0164916623B9F740917406D0
:2038600050917506609176067091770684E394E00E94582E409178065091790660917A06DE
:2038800070917B0681E394E00E94582E40917C0650917D0660917E0670917F068EE294E010
:2038A0000E94582E409180065091810660918206709183068BE294E00E94582EE09128106C
:2038C000F09129100280F381E02D88E290E166E171E0099588E290E16AE00E94C210F80188
:2038E0006491CFE4D2E007C088E290E10E94C2102196FE0164916623B9F7EDE0F4E06491DE
:20390000EF0107C088E290E10E94C2102196FE0164916623B9F788E290E16AE00E94C21024
:20392000F8016491CFE4D2E007C088E290E10E94C2102196FE0164916623B9F740919406CF
:2039400050919506609196067091970684E094E00E94342E409198065091990660919A0664
:2039600070919B0681E094E00E94342E40919C0650919D0660919E0670919F068EEF93E0AA
:203980000E94342E4091A0065091A1066091A2067091A3068BEF93E00E94342EE091281047
:2039A000F09129100280F381E02D88E290E166E171E0099588E290E16AE00E94C210F801A7
:2039C0006491CFE4D2E007C088E290E10E94C2102196FE0164916623B9F7E6ECF3E06491F9
:2039E000EF0107C088E290E10E94C2102196FE0164916623B9F788E290E16AE00E94C21044
:203A0000F8016491CFE4D2E007C088E290E10E94C2102196FE0164916623B9F74091A806DA
:203A20005091A9066091AA067091AB068DEB93E00E94582E4091AC065091AD066091AE06D4
:203A40007091AF068AEB93E00E94582EE0912810F09129100280F381E02D88E290E166E118
:203A600071E0099588E290E16AE00E94C210F8016491CFE4D2E007C088E290E10E94C21055
:203A80002196FE0164916623B9F7E7E0F3E06491EF0107C088E290E10E94C2102196FE01F7
:203AA00064916623B9F788E290E16AE00E94C210F8016491CFE4D2E007C088E290E10E94A8
:203AC000C2102196FE0164916623B9F74091A4065091A5066091A6067091A7068EEF92E0EF
:203AE0000E94582E4091BC065091BD066091BE067091BF068BEF92E00E94582E4091700691
:203B000050917106609172067091730688EF92E00E94342E4091B0065091B1066091B206B5
:203B20007091B30685EF92E00E94582E4091B4065091B5066091B6067091B70682EF92E048
:203B40000E94582E4091B8065091B9066091BA067091BB068FEE92E00E94582EE0912810DB
:203B6000F09129100280F381E02D88E290E166E171E0099588E290E16AE00E94C210F801E5
:203B80006491CFE4D2E007C088E290E10E94C2102196FE0164916623B9F7EDEDF2E0649130
:203BA000EF0107C088E290E10E94C2102196FE0164916623B9F788E290E16AE00E94C21082
:203BC000F8016491CFE4D2E007C088E290E10E94C2102196FE0164916623B9F74091820441
:203BE00050918304609184047091850484ED92E00E94582E4091860450918704609188040B
:203C00007091890481ED92E00E94582E40918A0450918B0460918C0470918D048EEC92E040
:203C20000E94582EE0912810F09129100280F381E02D88E290E166E171E0099588E290E10A
:203C40006AE00E94C210F8016491CFE4D2E007C088E290E10E94C2102196FE016491662309
:203C6000B9F7E0ECF2E06491EF0107C088E290E10E94C2102196FE0164916623B9F788E2AD
:203C800090E16AE00E94C210F8016491CFE4D2E007C088E290E10E94C2102196FE016491E1
:203CA0006623B9F74091990250919A0260919B0270919C0286EB92E00E94582E60919D021A
:203CC00070919E0280919F029091A0020E94BB75AB01BC0183EB92E00E94582E6091A102F7
:203CE0007091A2028091A3029091A4020E94C775AB01BC0180EB92E00E94582EE0912810AD
:203D0000F09129100280F381E02D88E290E166E171E0099588E290E16AE00E94C210F80143
:203D20006491CFE4D2E007C088E290E10E94C2102196FE0164916623B9F7EFE9F2E0649190
:203D4000EF0107C088E290E10E94C2102196FE0164916623B9F788E290E16AE00E94C210E0
:203D6000F8016491CFE4D2E007C088E290E10E94C2102196FE0164916623B9F782E493E01D
:203D800060E070E0C5D5AB01BC0187E992E00E94582E82E493E061E070E0BAD5AB01BC0124
:203DA00084E992E00E94582E82E493E062E070E0AFD5AB01BC0181E992E00E94582EE0912F
:203DC0002810F09129100280F381E02D88E290E166E171E0099588E290E16AE00E94C21044
:203DE000DF91CF911F910F9108950F931F93DF93CF93CDB7DEB7A0970FB6F894DEBF0FBED3
:203E0000CDBF8091170190911801A0911901B0911A01898B9A8BAB8BBC8BFE013D9604E69A
:203E200010E0F999FECF12BD01BDF89A80B580830F5F1F4F0836110511F03196F2CFCE0154
:203E40004196BE01635F7F4F43E050E00E94120E009709F0C1C1E4E8F6E0F999FECF12BD45
:203E600001BDF89A80B580830F5F1F4F0837110511F03196F2CFE4E7F6E0F999FECF12BD31
:203E800001BDF89A80B580830F5F1F4F0838110511F03196F2CFE4E9F6E0F999FECF12BD0E
:203EA00001BDF89A80B580830F5F1F4F0839110511F03196F2CF0E942B4CE8EAF6E0F9996B
:203EC000FECF12BD01BDF89A80B580830F5F1F4F0C39110511F03196F2CFECEAF6E0F999C0
:203EE000FECF12BD01BDF89A80B580830F5F1F4F003A110511F03196F2CFE4EAF6E0F999B3
:203F0000FECF12BD01BDF89A80B580830F5F1F4F043A110511F03196F2CFECEBF6E0F99985
:203F2000FECF12BD01BDF89A80B580830F5F1F4F083A110511F03196F2CFE0E7F6E0F99971
:203F4000FECF12BD01BDF89A80B580830F5F1F4F0C3A110511F03196F2CFE0EBF6E0F99949
:203F6000FECF12BD01BDF89A80B580830F5F1F4F003B110511F03196F2CFE4EBF6E0F99930
:203F8000FECF12BD01BDF89A80B580830F5F1F4F043B110511F03196F2CFE8EBF6E0F99908
:203FA000FECF12BD01BDF89A80B580830F5F1F4F083B110511F03196F2CFE2E8F4E0F999EF
:203FC000FECF12BD01BDF89A80B580830F5F1F4F043C110511F03196F2CFFE013196F999AA
:203FE000FECF12BD01BDF89A80B580830F5F1F4F063C110599F7FE013396F999FECF12BDE3
:2040000001BDF89A80B580830F5F1F4F083C110511F03196F2CFFE013596F999FECF12BD61
:2040200001BDF89A80B580830F5F1F4F0A3C110511F03196F2CFFE013796F999FECF12BD3D
:2040400001BDF89A80B580830F5F1F4F0C3C110511F03196F2CFFE013996F999FECF12BD19
:2040600001BDF89A80B580830F5F1F4F0E3C110511F03196F2CFFE013B96F999FECF12BDF5
:2040800001BDF89A80B580830F5F1F4F003D110511F03196F2CFE9E9F2E0F999FECF12BD0E
:2040A00001BDF89A80B580830F5F1F4F043D110511F03196F2CFEDE9F2E0F999FECF12BDE6
:2040C00001BDF89A80B580830F5F1F4F083D110511F03196F2CFE1EAF2E0F999FECF12BDCD
:2040E00001BDF89A80B580830F5F1F4F0C3D110511F03196F2CF0E948475FE017596F9993D
:20410000FECF12BD01BDF89A80B580830F5F1F4F003E110511F03196F2CFFE017996F99922
:20412000FECF12BD01BDF89A80B580830F5F1F4F043E110511F03196F2CFFE017D96F999FA
:20414000FECF12BD01BDF89A80B58083073E110521F00F5F1F4F3196F2CF2D893E894F8916
:20416000588D82E493E060E070E0E0D3298D3A8D4B8D5C8D82E493E061E070E0D7D32D8D32
:204180003E8D4F8D58A182E493E062E070E0CED3EFE4F2E064918F0108C088E290E10E9404
:2041A000C2100F5F1F4FF80164916623B1F7E7E7F2E064918F0108C088E290E10E94C210F6
:2041C0000F5F1F4FF80164916623B1F788E290E16AE00E94C21001C0EED89CDAA0960FB653
:2041E000F894DEBF0FBECDBFCF91DF911F910F9108950F931F93DF93CF93CDB7DEB7A09708
:204200000FB6F894DEBF0FBECDBF80911B0190911C01A0911D01B0911E018D879E87AF87CE
:20422000B88BFE013D9604E610E08081F999FECF1FBA12BD01BD80BD0FB6F894FA9AF99A14
:204240000FBE0F5F1F4F0836110511F03196EDCFE4E8F6E08081F999FECF1FBA12BD01BD75
:2042600080BD0FB6F894FA9AF99A0FBE0F5F1F4F0837110511F03196EDCFE4E7F6E0808165
:20428000F999FECF1FBA12BD01BD80BD0FB6F894FA9AF99A0FBE0F5F1F4F0838110511F0A4
:2042A0003196EDCFE4E9F6E08081F999FECF1FBA12BD01BD80BD0FB6F894FA9AF99A0FBE90
:2042C0000F5F1F4F0839110511F03196EDCFE8EAF6E08081F999FECF1FBA12BD01BD80BD7C
:2042E0000FB6F894FA9AF99A0FBE0F5F1F4F0C39110511F03196EDCFECEAF6E08081F9997F
:20430000FECF1FBA12BD01BD80BD0FB6F894FA9AF99A0FBE0F5F1F4F003A110511F03196F4
:20432000EDCFE4EAF6E08081F999FECF1FBA12BD01BD80BD0FB6F894FA9AF99A0FBE0F5F67
:204340001F4F043A110511F03196EDCFECEBF6E08081F999FECF1FBA12BD01BD80BD0FB6A2
:20436000F894FA9AF99A0FBE0F5F1F4F083A110511F03196EDCFE0E7F6E08081F999FECF08
:204380001FBA12BD01BD80BD0FB6F894FA9AF99A0FBE0F5F1F4F0C3A110511F03196EDCF79
:2043A000E0EBF6E08081F999FECF1FBA12BD01BD80BD0FB6F894FA9AF99A0FBE0F5F1F4F38
:2043C000003B110511F03196EDCFE4EBF6E08081F999FECF1FBA12BD01BD80BD0FB6F8940F
:2043E000FA9AF99A0FBE0F5F1F4F043B110511F03196EDCFE8EBF6E08081F999FECF1FBA32
:2044000012BD01BD80BD0FB6F894FA9AF99A0FBE0F5F1F4F083B110511F03196EDCFE2E80A
:20442000F4E08081F999FECF1FBA12BD01BD80BD0FB6F894FA9AF99A0FBE0F5F1F4F043C44
:20444000110511F03196EDCF80EA90E09A83898386E490E09C838B832FEF30E03E832D8319
:204460008EEB90E098878F838AE590E09A8789873C872B87FE0131968081F999FECF1FBA9E
:2044800012BD01BD80BD0FB6F894FA9AF99A0FBE0F5F1F4F063C110571F7FE0133968081A8
:2044A000F999FECF1FBA12BD01BD80BD0FB6F894FA9AF99A0FBE0F5F1F4F083C110511F07E
:2044C0003196EDCFFE0135968081F999FECF1FBA12BD01BD80BD0FB6F894FA9AF99A0FBE47
:2044E0000F5F1F4F0A3C110511F03196EDCFFE0137968081F999FECF1FBA12BD01BD80BD31
:204500000FB6F894FA9AF99A0FBE0F5F1F4F0C3C110511F03196EDCFFE0139968081F99937
:20452000FECF1FBA12BD01BD80BD0FB6F894FA9AF99A0FBE0F5F1F4F0E3C110511F03196C2
:20454000EDCFFE013B968081F999FECF1FBA12BD01BD80BD0FB6F894FA9AF99A0FBE0F5F19
:204560001F4F003D110511F03196EDCFE9E9F2E08081F999FECF1FBA12BD01BD80BD0FB68A
:20458000F894FA9AF99A0FBE0F5F1F4F043D110511F03196EDCFEDE9F2E08081F999FECFDC
:2045A0001FBA12BD01BD80BD0FB6F894FA9AF99A0FBE0F5F1F4F083D110511F03196EDCF58
:2045C000E1EAF2E08081F999FECF1FBA12BD01BD80BD0FB6F894FA9AF99A0FBE0F5F1F4F1A
:2045E0000C3D110511F03196EDCF82E493E060E070E08ED1698B7A8B8B8B9C8B82E493E001
:2046000061E070E085D16D8B7E8B8F8B988F82E493E062E070E07CD1698F7A8F8B8F9C8F73
:20462000FE0171968081F999FECF1FBA12BD01BD80BD0FB6F894FA9AF99A0FBE0F5F1F4F50
:20464000003E110511F03196EDCFFE0175968081F999FECF1FBA12BD01BD80BD0FB6F89424
:20466000FA9AF99A0FBE0F5F1F4F043E110511F03196EDCFFE0179968081F999FECF1FBA47
:2046800012BD01BD80BD0FB6F894FA9AF99A0FBE073E110521F00F5F1F4F3196EDCF80912F
:2046A000170190911801A0911901B0911A018D8F9E8FAF8FB8A3FE017D9684E690E0208192
:2046C000F999FECF1FBA92BD81BD20BD0FB6F894FA9AF99A0FBE8736910519F00196319639
:2046E000EECFEFE4F2E064918F0108C088E290E10E94C2100F5F1F4FF80164916623B1F7C1
:20470000E8E7F4E064918F0108C088E290E10E94C2100F5F1F4FF80164916623B1F788E2F5
:2047200090E16AE00E94C210A0960FB6F894DEBF0FBECDBFCF91DF911F910F9108952F924F
:204740003F924F925F926F927F928F929F92AF92BF92CF92DF92EF92FF920F931F93DF9316
:20476000CF93CDB7DEB73C011A012B01C901B801F30120823182428253820483158326830D
:204780003783C086D186E286F38684869586A686B78620E030E040E050E00E9468948823AA
:2047A00011F410E001C012E0F301608571858285938520E030E040E050E00E9468948823BA
:2047C00011F4EE2402C094E0E92EC501B40120E030E040E050E00E946894882311F4FF2429
:2047E00002C088E0F82E00E0C201B10120E030E040E050E00E946894811101E0102B1E2921
:204800001F29F30111A36081718182819381209184063091850640918606509187060E94CA
:2048200048970E94D794F301608B718B828B938B64817581868197812091880630918906FD
:2048400040918A0650918B060E9448970E94D794F301648B758B868B978B608571858285FF
:20486000938520918C0630918D0640918E0650918F060E9448970E94D794F301608F718F3D
:20488000828F938F6485758586859785209190063091910640919206509193060E944897D8
:2048A0000E94D794F301648F758F868F978FCF91DF911F910F91FF90EF90DF90CF90BF907A
:2048C000AF909F908F907F906F905F904F903F902F9008958F929F92AF92BF92CF92DF928E
:2048E000EF92FF920F931F93DF93CF93CDB7DEB7FC0110A224DFCF91DF911F910F91FF9004
:20490000EF90DF90CF90BF90AF909F908F900895FB01EE0FFF1FEE0FFF1FE80FF91F2081EF
:20492000318142815381B901CA0108950F931F93CF93DF93EC018B01FB01EE0FFF1FEE0F57
:20494000FF1FE80FF91F2083318342835383CA01B90120E030E040E050E00E94689429A1EB
:20496000882309F45EC081E090E002C0880F991F0A95E2F7282B29A3688179818A819B81EE
:20498000209184063091850640918606509187060E9448970E94D794688B798B8A8B9B8B05
:2049A0006C817D818E819F81209188063091890640918A0650918B060E9448970E94D794ED
:2049C0006C8B7D8B8E8B9F8B688579858A859B8520918C0630918D0640918E0650918F0609
:2049E0000E9448970E94D794688F798F8A8F9B8F6C857D858E859F8520919006309191061E
:204A000040919206509193060E9448970E94D7946C8F7D8F8E8F9F8FDF91CF911F910F91B3
:204A2000089581E090E002C0880F991F0A95E2F780952823A0CFCF93DF93EC01FB0160E0B3
:204A4000208131814281538188819981AA81BB81281739074A075B070CF461E02481358114
:204A6000468157818C819D81AE81BF81281739074A075B070CF4626020853185428553850F
:204A800088859985AA85BB85281739074A075B070CF4646024853585468557858C859D8549
:204AA000AE85BF85281739074A075B070CF46860862FDF91CF910895CF93DF93EC01FB01A6
:204AC00060E0208131814281538188819981AA81BB81281739074A075B0709F061E0248111
:204AE0003581468157818C819D81AE81BF81281739074A075B0709F06260208531854285B8
:204B0000538588859985AA85BB85281739074A075B0709F0646024853585468557858C8519
:204B20009D85AE85BF85281739074A075B0709F06860862FDF91CF9108952F923F924F9254
:204B40005F926F927F928F929F92AF92BF92CF92DF92EF92FF920F931F93DF93CF93CDB7DE
:204B6000DEB765970FB6F894DEBF0FBECDBF1C01FB017A01690158018E010F5F1F4F80E13A
:204B8000D8011D928A95E9F760817181828193812091840630918506409186065091870652
:204BA0000E9448970E94D79469837A838B839C83F70160817181828193812091880630916F
:204BC000890640918A0650918B060E9448970E94D7946D837E838F839887D6016D917D91E0
:204BE0008D919C9120918C0630918D0640918E0650918F060E9448970E94D79469877A8779
:204C00008B879C87F5016081718182819381209190063091910640919206509193060E945B
:204C200048970E94D7946D877E878F87988B80ED96E0B80100DF482E80ED96E0B8013CDFAE
:204C4000582ED1019096BC91B98B8B2F84258521282F30E0F10181A190E082239323892B42
:204C600009F465C0E0ED8E2EE6E09E2E74E6A72E73E0B72E3101CC24DD243B8B2A8B842D41
:204C800090E09D8B8C8B8A899B890C2C02C0959587950A94E2F780FF3AC08C899D890C2C8B
:204CA00002C0959587950A94E2F7D3015096ED90FD900D911C91539780FF08C02227332792
:204CC000A9012E193F09400B510B02C0A8019701F40180819181A281B381821B930BA40BA8
:204CE000B50B80839183A283B383CA01B9010E940A959B01AC01D5016D917D918D919C9146
:204D00000E948F93F50160837183828393830894C11CD11C84E090E0880E991EA80EB91ED3
:204D2000680E791E94E0C916D10409F0ACCF852D8095A9898A2354208529F10180A36596F2
:204D40000FB6F894DEBF0FBECDBFCF91DF911F910F91FF90EF90DF90CF90BF90AF909F9053
:204D60008F907F906F905F904F903F902F9008958F929F92AF92BF92CF92DF92EF92FF9245
:204D80000F931F9382E493E040E050E060E070E08A019B016A017B014A015B019BDD1F9129
:204DA0000F91FF90EF90DF90CF90BF90AF909F908F900895CF92DF92EF92FF920F931F93C6
:204DC000DF93CF930F92CDB7DEB77C01E8EAF4E084918F016E010894C11CD11C0CC08983D0
:204DE00088E290E1B60141E050E00E9428920F5F1F4FF8018491882391F7F70140815181CC
:204E00006281738188E290E122E00E94FA90E5EAF4E084918F016E010894C11CD11C0CC0C9
:204E2000898388E290E1B60141E050E00E9428920F5F1F4FF8018491882391F7F70144814D
:204E400055816681778188E290E122E00E94FA90E2EAF4E084918F016E010894C11CD11C7A
:204E60000CC0898388E290E1B60141E050E00E9428920F5F1F4FF8018491882391F7F70106
:204E8000408551856285738588E290E122E00E94FA90EFE9F4E084918F016E010894C11C56
:204EA000D11C0CC0898388E290E1B60141E050E00E9428920F5F1F4FF8018491882391F7D1
:204EC000F701448555856685778588E290E122E00E94FA90E4E9F4E084918F017E010894E6
:204EE000E11CF11C0CC0898388E290E1B70141E050E00E9428920F5F1F4FF80184918823FB
:204F000091F74091640350916503609166037091670388E290E122E00E94FA90E0E9F4E01D
:204F200084918F017E010894E11CF11C0CC0898388E290E1B70141E050E00E9428920F5F21
:204F40001F4FF8018491882391F7409168035091690360916A0370916B0388E290E122E06F
:204F60000E94FA90ECE8F4E084918F017E010894E11CF11C0CC0898388E290E1B70141E007
:204F800050E00E9428920F5F1F4FF8018491882391F740916C0350916D0360916E03709174
:204FA0006F0388E290E122E00E94FA90E8E8F4E084918F017E010894E11CF11C0CC0898330
:204FC00088E290E1B70141E050E00E9428920F5F1F4FF8018491882391F74091700350914F
:204FE0007103609172037091730388E290E122E00E94FA90E0912810F09129100280F381FE
:20500000E02D88E290E16FE171E009958AE0898388E290E1B70141E050E00E9428920F9014
:20502000CF91DF911F910F91FF90EF90DF90CF900895DC01ED91FC910280F381E02D09954E
:205040000895CF93DF930FB6F89480911F1090912010A0912110B09122100FBE8093AF0495
:205060009093B004A093B104B093B204E091D804F091D904E652FB4F8081882399F4EEE440
:20508000F5E06491EF0107C088E290E10E94C2102196FE0164916623B9F788E290E16AE037
:2050A0000E94C210DF91CF91089508958091A50408958130910541F46F5F7F4F09F051C0F9
:2050C00084E793E00C94DA10892B09F04AC06F5F7F4F09F046C087E293E090933D048093C3
:2050E0003C0480914104882321F08EE394E00E94F76087E293E09093FD038093FC0380915E
:205100000104882321F08EEF93E00E94F76087E293E09093E0038093DF038091E40388236B
:2051200021F081EE93E00E94F76087E293E09093C3038093C2038091C703882321F084ECDF
:2051400093E00E94F76087E293E09093A4038093A3038091A803882321F085EA93E00C948A
:20516000F760089580E090E06FEF7FEFA2CF81E090E06FEF7FEF9DCFCF93DF930E94A77593
:205180008091A504882309F034C081E08093A5048091A7049091A804A091A904B091AA044A
:2051A0008093AB049093AC04A093AD04B093AE04E2EBF4E06491EF0107C088E290E10E94B7
:2051C000C2102196FE0164916623B9F7E9EBF4E06491EF0107C088E290E10E94C2102196BF
:2051E000FE0164916623B9F788E290E16AE00E94C210DF91CF910895CF93DF93F8940E947A
:20520000A775779A769A479A439AE2EBF4E06491EF0107C088E290E10E94C2102196FE0141
:2052200064916623B9F7EFE2F5E06491EF0107C088E290E10E94C2102196FE01649166236B
:20524000B9F788E290E16AE00E94C210FFCFEF92FF920F931F930FB6F89480911F1090911F
:205260002010A0912110B09122100FBEE090B304F090B4040091B5041091B6042091AF04F4
:205280003091B0044091B1045091B204821B930BA40BB50BE816F9060A071B0730F4E11489
:2052A000F1040105110509F0A7DFE0907F02F09080020091810210918202E114F104010542
:2052C000110531F10FB6F89480911F1090912010A0912110B09122100FBE2091AF043091ED
:2052E000B0044091B1045091B204821B930BA40BB50BE816F9060A071B0750F49091B10BE2
:205300008091B20B981721F4779A769A479A439A0E94C64B1F910F91FF90EF9008956F926D
:205320007F928F929F92AF92BF92CF92DF92EF92FF920F931F93F82E6091B7047091B804B1
:205340008091B9049091BA042091BB043091BC044091BD045091BE040E9483963B014C0136
:2053600000D000D000D00DB71EB70F5F1F4F60916F0270917002882777FD8095982F0E94D2
:205380000A95209183023091840240918502509186020E94489720E030E040E752E40E94A0
:2053A0006F9420E030E048EC52E40E946F945B016C01F8016082718282829382F482809194
:2053C0009A04858382E794E063EC74E047EB54E020E001E032E0E32E0E942B478091C30451
:2053E0009091C404A091C504B091C6048093720490937304A0937404B09375048091C70459
:205400009091C804A091C904B091CA048093760490937704A0937804B09379048091CB0418
:205420009091CC04A091CD04B091CE0480937A0490937B04A0937C04B0937D048091CF04D8
:205440009091D004A091D104B091D20480937E0490937F04A0938004B09381040FB6F8942F
:2054600080911F1090912010A0912110B09122100FBE8093AF049093B004A093B104B09331
:20548000B2048DB79EB706960FB6F8949EBF0FBE8DBF1F910F91FF90EF90DF90CF90BF90DF
:2054A000AF909F908F907F906F900895CF92DF92EF92FF920F931F930FB6F89480911F10EB
:2054C00090912010A0912110B09122100FBE8093AF049093B004A093B104B093B20460916A
:2054E00072047091730480917404909175042091C3043091C4044091C5045091C6040E94B3
:205500006894882309F07AC0609176047091770480917804909179042091C7043091C80496
:205520004091C9045091CA040E946894882309F065C0609183027091840280918502909101
:20554000860220E030E040E752E40E946F947B018C0183EC94E067EC74E04BEC54E02FEC98
:2055600034E0EAE9CE2EE4E0DE2E0E945A518091C3049091C404A091C504B091C604809352
:20558000720490937304A0937404B09375048091C7049091C804A091C904B091CA048093AB
:2055A000760490937704A0937804B09379048091CB049091CC04A091CD04B091CE0480936B
:2055C0007A0490937B04A0937C04B0937D048091CF049091D004A091D104B091D20480932B
:2055E0007E0490937F04A0938004B09381041F910F91FF90EF90DF90CF90089560916F02D9
:2056000070917002882777FD8095982F0E940A952091830230918402409185025091860299
:205620000E94489720E030E040E752E40E946F9420E030E048EC52E488CFCF93DF9388E2C8
:2056400090E10E941092E1E5F5E06491EF0107C088E290E10E94C2102196FE0164916623CB
:20566000B9F74091A7045091A8046091A9047091AA044F5F5F4F6F4F7F4F88E290E10E94BF
:20568000E99088E290E16AE00E94C210DADCDF91CF9108952F923F924F925F926F927F925F
:2056A0008F929F92AF92BF92CF92DF92EF92FF920F931F93DF93CF9300D000D000D0CDB706
:2056C000DEB72C0163991AC1609172047091730480917404909175040E94D7944B015C0179
:2056E00080915F0290916002A0916102B09162028093830290938402A0938502B0938602B6
:2057000080E090E0A0E0B0E08093720490937304A0937404B093750482E794E066E774E0A1
:205720004AE754E02EE734E00E94734CE7E6F6E0E590F59005911491F3E76F2EF6E07F2EA8
:20574000F301649117FB109517F91095772767FD7095872F972F0E940A959B01AC01C8011E
:20576000B7010E9448976093C3047093C4048093C5049093C6046091830270918402809194
:2057800085029091860220E030E040E752E40E946F947B018C0183EC94E067EC74E04BECFD
:2057A00054E02FEC34E0EAE9CE2EE4E0DE2E0E945A510E94616EB401882777FD8095982F75
:2057C0000E940A95609372047093730480937404909375046093C3047093C4048093C5041D
:2057E0009093C60463998AC060917A0470917B0480917C0490917D040E94D7944B015C019E
:205800008091670290916802A0916902B0916A028093830290938402A0938502B093860274
:2058200080E090E0A0E0B0E080937A0490937B04A0937C04B0937D0482E794E066E774E060
:205840004AE754E02EE734E00E94734CEFE6F6E0E590F59005911491A2E0B0E06A0E7B1E56
:20586000F301649117FB109517F91095772767FD7095872F972F0E940A959B01AC01C801FD
:20588000B7010E9448976093CB047093CC048093CD049093CE046091830270918402809153
:2058A00085029091860220E030E040E752E40E946F947B018C0183EC94E067EC74E04BECDC
:2058C00054E02FEC34E00E945A510E94616EB401882777FD8095982F0E940A9560937A0441
:2058E00070937B0480937C0490937D046093CB047093CC048093CD049093CE0441145104D7
:2059000029F0F2E04F16510409F074C13201660C771C660C771C93012E583B4F3A8329836A
:2059200080E090E0A0E0B0E0F90180839183A283B38382E794E066E774E04AE754E02EE723
:2059400034E00E94734CF301E55AF94F659175918591949123E736E0420E531EF201E490D8
:2059600093012D533B4F3E832D8320E030E040EC5FE30E9448975B016C01FF24E7FCF094C6
:205980000F2D1F2DC801B7010E940A951B012C01C601B501A20191010E944897AD81BE81D4
:2059A0006D937D938D939C931397F301E15AFD4FFC83EB8360817181828193816093830214
:2059C00070938402809385029093860220E030E040E752E40E946F947B018C0183EC94E0FB
:2059E00067EC74E04BEC54E02FEC34E0AAE9CA2EA4E0DA2E0E945A510E94616E80E090E0C1
:205A0000A0E0B0E0E981FA8180839183A283B38382E794E066E774E04AE754E02EE734E013
:205A20000E94734CF301E959F94F85909590A590B490C501B4019058A20191010E944897BB
:205A4000AD81BE816D937D938D939C9313976091830270918402809185029091860220E092
:205A600030E040E752E40E946F947B018C0183EC94E067EC74E04BEC54E02FEC34E00E9445
:205A80005A510E94616EC501B401A50194010E948F93A20191010E944897ED81FE816083EA
:205AA000718382839383AB81BC816D917D918D919C9120E030E040E05FE30E944897609331
:205AC000830270938402809385029093860220E030E040E752E40E946F947B018C0183ECE9
:205AE00094E067EC74E04BEC54E02FEC34E00E945A510E94616E83010E571B4FF301EE57A7
:205B0000F94F6591759185919491FEE8EF2EF4E0FF2EE60CF71CF80120813181428153811A
:205B20000E948F93D7016D937D938D939C931397F301E257F94F6591759185919491E3E74A
:205B4000F2E06E0E7F1ED8012D913D914D915C910E948F93F3016083718382839383F80187
:205B600080819181A281B381E981FA8180839183A283B383ED81FE8180839183A283B38305
:205B800080E090E0A0E0B0E08093830290938402A0938502B09386020E94856D82E794E0EE
:205BA00066E774E04AE754E02EE734E00E94734CAB81BC816D917D918D919C91609383021D
:205BC00070938402809385029093860220E030E040E752E40E946F947B018C0183EC94E0F9
:205BE00067EC74E04BEC54E02FEC34E00E945A510E94616E26960FB6F894DEBF0FBECDBFA3
:205C0000CF91DF911F910F91FF90EF90DF90CF90BF90AF909F908F907F906F905F904F90D0
:205C20003F902F9008954091D8045091D90420E630E0B901469F9001479F300D569F300D33
:205C40001124682F772767FD7095C9018C519B4F0E94000E9C019093E3048093E20480E030
:205C6000232B09F081E00895EF92FF920F931F93CF93DF93EC017A018B01FC01649107C0F8
:205C800088E290E10E94C2102196FE0164916623B9F788E290E1B801A7012AE000E00E9409
:205CA0005E90DF91CF911F910F91FF90EF900895EF92FF920F931F93CF93DF93EC017A0189
:205CC0008B01FC01649107C088E290E10E94C2102196FE0164916623B9F788E290E1B801B8
:205CE000A70122E00E94FA90DF91CF911F910F91FF90EF900895F8946AE070E080E090E00D
:205D00000E94228D81E08093E00080E28093D80064E670E080E090E00E94228D1DBA10925D
:205D200068001CBC10BE1FBA10927A0010926E0010926F0010927000109271001092C900AF
:205D40001092BC0011B814B817B81AB81DB810BA12B815B818B81BB81EB811BA0C9400F89D
:205D6000FFCF8091E2049091E304019660E070E04AE050E00C94770C8091E2049091E304B3
:205D8000019660E070E00C941A0B0F931F93CF93DF938C0180919A048093A60484E543DF6B
:205DA000882309F44EC0E8DF0E94DC946093A604662309F446C0ECEAF4E06491EF0107C0D5
:205DC00088E290E10E94C2102196FE0164916623B9F70936110599F00A36110524F4083606
:205DE0001105E1F407C00D36110571F00A3D1105A9F40FC088E290E160E271E00EC088E2C8
:205E000090E167E371E009C088E290E16EE471E004C088E290E165E671E00BD9E091281067
:205E2000F09129100190F081E02D88E290E16091A604099588E290E16AE00E94C21081E08B
:205E400001C080E0DF91CF911F910F910895AF92BF92CF92DF92EF92FF920F931F93CF9338
:205E6000DF93A2E7EA2EA4E0FA2EC3ECD4E000E010E0F801E951FD4F8081D5DE882331F130
:205E80007BDF5B016C01F801E459FB4F8081882311F061E002C06091D30470E0882777FD74
:205EA0008095982F0E940A95F70120813181428153810E9448979B01AC01C601B5010E94FA
:205EC0008F93688379838A839B8309C0F70180819181A281B38188839983AA83BB830F5F63
:205EE0001F4F84E090E0E80EF91E24960430110509F0BFCF86E497DE8823D9F03DDF7B01DD
:205F00008C016093D4047093D5048093D6049093D70420E030E040E050E00E947696181626
:205F200044F4E0928302F09284020093850210938602DF91CF911F910F91FF90EF90DF9048
:205F4000CF90BF90AF90089582DF89E46CDE882351F012DF6093B7047093B8048093B90485
:205F60009093BA040CC080E090E0A0E0B0E08093B7049093B804A093B904B093BA048AE488
:205F800052DE882351F0F8DE6093BB047093BC048093BD049093BE04089580E090E0A0E0F4
:205FA000B0E08093BB049093BC04A093BD04B093BE0408952F923F924F925F926F927F9290
:205FC0008F929F92AF92BF92CF92DF92EF92FF920F931F93DF93CF93CDB7DEB76E970FB6EE
:205FE000F894DEBF0FBECDBF87E41DDE882309F429C2C2DE0E94D7946430710509F43CC076
:206000006530710554F46230710531F16330710554F57723CCF40C94D43F6A35710509F492
:20602000C0C16B35710534F46C31710511F00C94D43F78C06B35710509F4B7C16C35710500
:2060400011F00C94D43FB6C18091A504882321F4FEDE2CDA0C9407408091A504882319F460
:2060600073DF81E006C08091A504882329F46CDF80E055D90C94074080E5D5DD882321F48E
:20608000AA24BB24650105C077DE0E94DC945B016C0183E5C8DD882359F06EDE20E030E09B
:2060A0004AE754E40E9448970E94DC945B016C010E94616E0FB6F894E0901F10F09020100A
:2060C00000912110109122100FBEEA0CFB1C0C1D1D1D0FB6F89480911F1090912010A091DB
:2060E0002110B09122100FBE8093AF049093B004A093B104B093B20403C00E94FF78A7D856
:206100000FB6F89480911F1090912010A0912110B09122100FBE8E159F05A007B10768F3FA
:206120000C94D43F8091830290918402A0918502B09186028093DE049093DF04A093E004DC
:20614000B093E10480916F0290917002909371048093700484E690E09093700280936F02F0
:206160000FB6F89480911F1090912010A0912110B09122100FBE8093AF049093B004A093CB
:20618000B104B093B20481E00E948C6D8091720490917304A0917404B09175048093C304F9
:2061A0009093C404A093C504B093C6048091760490917704A0917804B09179048093C7047B
:2061C0009093C804A093C904B093CA0480917A0490917B04A0917C04B0917D048093CB043B
:2061E0009093CC04A093CD04B093CE0480917E0490917F04A0918004B09181048093CF04FB
:206200009093D004A093D104B093D20480E090E0A0E0B0E08093830290938402A09385028B
:20622000B093860288E5FFDC882351F489E5FBDC882331F48AE5F7DC882311F481E001C032
:2062400080E080938702882321F488E5ECDC882319F080E090E01EDA80918702882321F477
:2062600089E5E1DC882361F080E090E0A0E0B0E08093760490937704A0937804B09379047D
:2062800080918702882321F48AE5CDDC882319F082E090E0FFD988E5C6DC8823B1F061DD95
:2062A000611571058105910581F08091820490918304A0918404B0918504809372049093F7
:2062C0007304A0937404B093750489E5ACDC882391F047DD611571058105910561F080E0E1
:2062E00090E0A0E0B0E08093760490937704A0937804B09379048AE596DC8823B1F031DD49
:20630000611571058105910581F080918A0490918B04A0918C04B0918D0480937A0490936E
:206320007B04A0937C04B0937D0482E794E066E774E04AE754E02EE734E00E94734C80E09A
:206340000E948C6D8091DE049091DF04A091E004B091E1048093830290938402A093850275
:20636000B093860280917004909171049093700280936F020FB6F89480911F10909120103C
:20638000A0912110B09122100FBE8093AF049093B004A093B104B093B2040E94856D0C94A9
:2063A000D43F1092D3040C94D43F81E08093D3040C94D43F85E437DC882311F40E94616E03
:2063C000B2E7EB2EB4E0FB2EA2E8CA2EA4E0DA2E00E010E0F801E951FD4F808124DC882345
:2063E00021F1033059F4C8DCF70160837183828393838EE794E00E94564C17C0BDDCF601E9
:2064000020813181428153810E948F93F701608371838283938382E794E066E774E04AE735
:2064200054E02EE734E00E94734C0F5F1F4F44E050E0E40EF51EC40ED51E0430110551F613
:206440000C94D43F8DE4EFDB882311F40C940D3F93DC0E94D7946B36710511F40C948C3AB4
:206460006C3671050CF092C06F31710509F48AC3603271050CF042C06731710509F469C21A
:2064800068317105E4F46431710509F428C2653171055CF46131710509F41BC262317105DC
:2064A00011F00C94D43F0C949A3A6531710509F444C26631710511F00C94D43F44C26A3143
:2064C000710509F480C26B31710554F46831710509F45AC26931710511F00C94D43F6DC292
:2064E0006C31710509F492C26C3171050CF488C26E31710511F00C94D43FC4C26036710580
:2065000009F4F8C06136710514F56335710511F40C94963A6435710554F46A32710509F4C7
:20652000DEC36235710511F00C94D43FFCC76535710511F40C94E33A653571050CF4FAC793
:206540006C35710511F00C94D43F0C94F93A6336710509F486C16436710554F461367105E5
:2065600009F4CEC06236710511F00C94D43F73C16936710509F424C46A3671050CF09BC72C
:206580006836710511F00C94D43FEAC36E3C710511F40C94B83D6F3C71050CF04FC0693700
:2065A000710511F40C948D3C6A37710524F56337710511F40C947E3B643771055CF46D3655
:2065C000710509F4CDC46237710511F00C94D43F0C949E3B6737710511F40C94913C683756
:2065E000710514F00C94893C6537710511F00C94D43F0C948E3B693C710511F40C94FA3C97
:206600006A3C710554F46C38710509F4C8C36E3B710511F00C94D43F7CC66C3C710511F43C
:206620000C943A3D6D3C710514F00C945A3D6B3C710511F00C94D43F0C941C3D51E0643F4B
:20664000750711F40C94E33E81E0653F78074CF591E06D32790711F40C94F43DE1E06E326C
:206660007E0764F46C3D710511F40C94D63D6D3D710511F00C94D43F0C94E53DF1E06F325E
:206680007F0711F40C94A03E21E06F32720714F40C949C3E6059714011F00C94D43F0C9496
:2066A000E03E51E0673F750711F40C94EC3E81E0683F78076CF491E0653F790711F40C9479
:2066C000E63E665F714011F00C94D43F0C94E93EF3E0603A7F0709F41AC223E0673E7207B8
:2066E00011F40C94F83E6455734011F00C94D43F0C94EF3E8FE69EE00E94A0860C94D43F64
:2067000081E491DA882339F037DBAB01BC018FE69EE00E942B8687E586DA882339F02CDB6D
:20672000AB01BC018FE69EE00E94038680E57BDA882339F021DBAB01BC018FE69EE00E944A
:2067400082818AE570DA882359F40F2EF0E04F2EF0E05F2EF0E86F2EFFEB7F2EF02D03C0B2
:206760000BDB2B013C0188E45EDA882359F40F2EF0E08F2EF0E09F2EF0E8AF2EFFEBBF2E3B
:20678000F02D03C0F9DA4B015C018CE44CDA882359F40F2EF0E0CF2EF0E0DF2EF0E8EF2E33
:2067A000FFEBFF2EF02D03C0E7DA6B017C01C301B20120E030E040E050E00E947696882308
:2067C00024F1C501B40120E030E040E050E00E947696882344F08FE69EE0B301A20195015C
:2067E00084010E94D088C701B60120E030E040E050E00E947696882344F08FE69EE0B30107
:20680000A201970186010E942B89C701B60120E030E040E050E00E947696181614F00C9401
:20682000D43FC501B40120E030E040E050E00E947696181614F00C94D43FC501B401A701B4
:2068400096010E946F94AB01BC018FE69EE00E94AC7F0C94D43F82E493E00E94DA260C9405
:20686000D43F88E5E0D9882349F086DA9B01AC0182E493E060E070E00E94962489E5D3D973
:20688000882349F079DA9B01AC0182E493E061E070E00E9496248AE5C6D9882349F06CDA7A
:2068A0009B01AC0182E493E062E070E00E94962485E4B9D9882311F40C94D43F5DDA9B0197
:2068C000AC0182E493E063E070E00E9496240C94D43F77987698479843980C94D43FEBE437
:2068E000F6E064918F0108C088E290E10E94C2100F5F1F4FF80164916623B1F788E290E150
:206900006AE00E94C21084E793E00E949319EDE3F6E064918F0108C088E290E10E94C2104B
:206920000F5F1F4FF80164916623B1F788E290E16AE00E94C2100C94D43F84E793E00E9490
:20694000DE150C94D43F84E793E00E9433110C94D43F8091E2049091E30404966AE270E0E5
:206960000E94000EFC01009711F0319710826091E2047091E3046C5F7F4F84E793E041E021
:206980000E9474120C94D43F84E793E00E9437110FB6F89480911F1090912010A091211010
:2069A000B09122100FBE80939D0490939E04A0939F04B093A0040C94D43F84E793E00E942E
:2069C0003E110C94D43F80917703882311F40C94D43F83E528D9882311F40C94D43FC1D961
:2069E000AB01BC01409361045093620480936304709364048EE394E00E94DF5F0C94D43F50
:206A000084E793E00E9415120C94D43F8091E2049091E30404966AE270E00E94000E8C01AA
:206A2000009719F12091D8043091D90480E690E0AC01249FC001259F900D349F900D11247D
:206A40008C519B4F6EE470E00E94000E60E270E00E94000E9C012F5F3F4F3093E3042093C5
:206A6000E20401501040F80110826091E2047091E3046C5F7F4F84E793E040E00E94741286
:206A80000C94D43F80917703882311F40C94D43F84E793E00E948D118091E2049091E30438
:206AA00004966AE270E00E94000E8C01009719F12091D8043091D90480E690E0AC01249F51
:206AC000C001259F900D349F900D11248C519B4F6EE470E00E94000E60E270E00E94000E94
:206AE0009C012F5F3F4F3093E3042093E20401501040F80110826091E2047091E3046C5FE4
:206B00007F4F84E793E00E947E140C94D43F8091E2049091E30405966AE270E00E94000EFC
:206B20008C01009719F12091D8043091D90480E690E0AC01249FC001259F900D349F900D24
:206B400011248C519B4F6EE470E00E94000E60E270E00E94000E9C012F5F3F4F3093E30442
:206B60002093E20401501040F80110826091E2047091E3046B5F7F4F84E793E00E947814ED
:206B80000C94D43F0FB6F89460911F107091201080912110909122100FBE6093A1047093A3
:206BA000A2048093A3049093A40420919D0430919E0440919F045091A004621B730B840B72
:206BC000950B28EE33E040E050E00E944C98F22EE32ED42EC52E4DB75EB7485050400FB6EA
:206BE000F8945EBF0FBE4DBF0DB71EB70F5F1F4FCE010196EDB7FEB7928381838EE296E0E0
:206C0000F801938382836F2D7E2D8D2D9C2D2CE330E040E050E00E944C98F8013583248349
:206C20006F2D7E2D8D2D9C2D2CE330E040E050E00E944C98F801778366830E942F0EECEA04
:206C4000F4E064918F014DB75EB7485F5F4F0FB6F8945EBF0FBE4DBF08C088E290E10E94E1
:206C6000C2100F5F1F4FF80164916623B1F788E290E1BE016F5F7F4F0E94192888E290E153
:206C80006AE00E94C2108091E006882311F40C94D43F1092E00680919A04082F10E0000F6F
:206CA000111F005E114FF80160817181882777FD8095982F0E940A9520918C0230918D024B
:206CC00040918E0250918F020E947696181614F00C94D43FF801118210820C94D43F83E515
:206CE0000E94132E882311F40C94D43F45D80E94D7947B018C016B0180E50E94132E8823BC
:206D000061F0F7FC0AC0FFEFEF16F10409F02CF433D80E94D7947B0103C0EE24EA94FE2C53
:206D2000EBEEF2E0808191818E159F0511F40C94D43F329623E0EB35F207A1F7F7FE02C063
:206D40000C94D43F8E2D0E94988BEE2DF0E00C2C0E94A98B8E2DB6010E94538D0C94D43F60
:206D600088E690E012D8882311F00C94D43F83E50E94132E882379F00E94BC2E2091A604A6
:206D8000022F10E0000F111F005E114F0E94D794F801718360830E94A6750C94D43F83E520
:206DA0000E94132E882311F40C94D43F0E94BC2E0E94D7947093230E6093220E0C94D43FEA
:206DC00089E690E00E94C52E882311F00C94D43FE8E2F6E064918F0108C088E290E10E9476
:206DE000C2100F5F1F4FF80164916623B1F7E091A604F0E0EE0FFF1FEE0FFF1FEA5DF14F1E
:206E0000408151816281738188E290E121E00E94FA90E5E2F6E064918F0108C088E290E13B
:206E20000E94C2100F5F1F4FF80164916623B1F7E091A604F0E0EE0FFF1FE05EF14F60817E
:206E40007181882777FD8095982F0E940A95AB01BC0188E290E121E00E94FA90E1E2F6E0F6
:206E600064918F0108C088E290E10E94C2100F5F1F4FF80164916623B1F740912C0E50918F
:206E80002D0E60912E0E70912F0E88E290E121E00E94FA90EEE1F6E064918F0108C088E2E8
:206EA00090E10E94C2100F5F1F4FF80164916623B1F76091220E7091230E882777FD809567
:206EC000982F0E940A95AB01BC0188E290E121E00E94FA90EAE1F6E064918F0108C088E2E1
:206EE00090E10E94C2100F5F1F4FF80164916623B1F78091A60490E00E949B75AC0166279B
:206F000057FD6095762F88E290E10E94E990E5E1F6E064918F0108C088E290E10E94C21055
:206F20000F5F1F4FF80164916623B1F78FEF9FEF0E949B75AC01662757FD6095762F88E206
:206F400090E10E94E99088E290E16CE771E00E94192888E290E16AE00E94C2100C940740C3
:206F60008DE690E00E94C52E882311F00C94D43F1092E00683E50E94132E882379F00E94B1
:206F8000BC2E2091A604022F10E0000F111F005E114F0E94D794F8017183608383E50E94A7
:206FA000132E882351F00E94BC2E60938C0270938D0280938E0290938F0282E40E94132E65
:206FC000882351F00E94BC2E609388027093890280938A0290938B0286E40E94132E8823E7
:206FE00069F00E94BC2E6093900270939102809392029093930281E08093E0060E94A6751B
:207000000FB6F89480901F1090902010A0902110B09022100FBE2091A604022F10E07724D9
:20702000000F111FF801E05EF14F60817181882777FD8095982F0E940A95000F111F0A5DE1
:20704000114FF80120813181428153810E947696181614F477247394CC24CA94DC2C76019A
:20706000E2E1F6E04490EEE0F6E05490EAE0F6E0649039C1642D02E116E008C088E290E180
:207080000E94C2100F5F1F4FF80164916623B1F7E091A604F0E0EE0FFF1FEE0FFF1FEA5D19
:2070A000F14F408151816281738188E290E121E00E94FA90652D0EE016E008C088E290E105
:2070C0000E94C2100F5F1F4FF80164916623B1F74091A60450E0662757FD6095762F88E2B1
:2070E00090E10E94E990662D0AE016E008C088E290E10E94C2100F5F1F4FF8016491662327
:20710000B1F7F7FC24C00FB6F89420911F103091201040912110509122100FBEC701B6016D
:2071200068577C4E8F4F9F4F621B730B840B950B28EE33E040E050E00E944C9888E290E1F6
:20714000BA01A9012AE000E00E945E9006C088E290E16DE771E00E94192888E290E16AE002
:207160000E94C2100FB6F89480901F1090902010A0902110B09022100FBE0E94FF780E9460
:207180002729FFEFCF16FFEFDF06FFEFEF06FFEFFF0609F050C0E091A604772031F1F0E076
:2071A0008F01000F111F000F111F0A5D114FEE0FFF1FE05EF14F60817181882777FD809556
:2071C000982F0E940A9520E030E040E85FE30E948E939B01AC01F80160817181828193813E
:2071E0000E94769687FF58C062C0F0E08F01000F111F000F111F0A5D114FEE0FFF1FE05E23
:20720000F14F60817181882777FD8095982F0E940A9520E030E040E85FE30E948F939B0141
:20722000AC01F80160817181828193810E946894181694F53CC0F7FC3AC0E091A604F0E095
:207240008F01000F111F000F111F0A5D114FEE0FFF1FE05EF14F60817181882777FD8095B5
:20726000982F0E940A959B01AC01F80160817181828193810E948E930E94D79497FF07C0AD
:2072800090958095709561957F4F8F4F9F4F64307105810591055CF00FB6F894C0901F10DD
:2072A000D0902010E0902110F09022100FBEFFEFCF16FFEFDF06FFEFEF06FFEFFF0699F019
:2072C000F7FC75C60FB6F89480911F1090912010A0912110B09122100FBE8C199D098858D1
:2072E000934108F064C60FB6F89480911F1090912010A0912110B09122100FBE88199909D1
:20730000AA09BB09895E9340A040B04008F0B2CE34CF83E50E94132E882341F00E94BC2E3E
:207320000E94D7947093230E6093220E0FB6F894E0901F10F09020100091211010912210B4
:207340000FBEE7E0F6E09490E3E0F6E0A490EFEFF5E0B49085C00FB6F89480911F109091E4
:207360002010A0912110B09122100FBE8E199F09A00BB10B895E9340A040B04008F46CC0D3
:20738000E0919A04F0E0EE0FFF1FEE0FFF1FEA5DF14FC080D180E280F380692D07E016E078
:2073A00008C088E290E10E94C2100F5F1F4FF80164916623B1F788E290E1B701A60122E07F
:2073C0000E94FA906A2D03E016E008C088E290E10E94C2100F5F1F4FF80164916623B1F7FF
:2073E00040919A0450E0662757FD6095762F88E290E10E94E9906B2D0FEF15E008C088E2C0
:2074000090E10E94C2100F5F1F4FF80164916623B1F740912C0E50912D0E60912E0E709137
:207420002F0E88E290E121E00E94FA9088E290E16CE771E00E94192888E290E16AE00E94DE
:20744000C2100FB6F894E0901F10F090201000912110109122100FBE0E94FF780E9427294D
:207460006091220E7091230E882777FD8095982F0E940A9520912C0E30912D0E40912E0E85
:2074800050912F0E0E94769618160CF464CF0FB6F89480911F1090912010A0912110B0913A
:2074A00022100FBE8093AF049093B004A093B104B093B20479C53C9A449A83E50E94132E12
:2074C000882319F10E94BC2E20E030E040E050E00E94689488231CF460E070E011C00E94AF
:2074E000BC2E20E030E04FE753E40E94769618161CF46FEF70E004C00E94BC2E0E94D7942E
:2075000070939C0460939B044FC58FEF90E090939C0480939B0448C510929C0410929B042F
:207520003C9A449841C510926F043EC581E080936F043AC583E50E94132E882399F00E9474
:20754000BC2E20E030E04AE754E40E9448970E94DC9460937F027093800280938102909383
:20756000820222C588E50E94132E882309F046C589E50E94132E882309F040C58AE50E9496
:20758000132E882309F03AC585E40E94132E882309F034C50E94616E439A0E946D6E04C58A
:2075A000779A89E50E94132E8111769A8AE50E94132E8111479A85E40E94132E882309F40E
:2075C000F3C4439AF1C483E50E94132E0E94BC2E20E030E04AE754E40E9448970E94DC947F
:2075E0006093B3047093B4048093B5049093B604DBC444E8642E46E0742E34E7232E36E0D6
:20760000332E20EC422E26E0522E88249924F401E951FD4F80810E94132E882309F45DC07A
:20762000F3E08F1609F052C00E94BC2E5B016C0120E030E040EA51E40E94689488230CF0BE
:207640003FC0F3016081718182819381A60195010E946F947B018C016091B8067091B906F3
:207660008091BA069091BB06A80197010E9448976093B8067093B9068093BA069093BB066B
:20768000F1016081718182819381A80197010E944897F1016083718382839383F201608194
:2076A0007181828193810E940895A80197010E9448970E94DC94F2016083718382839383C9
:2076C000F301A082B182C282D38207C00E94BC2EF30160837183828393830894811C911CA9
:2076E00044E050E0640E751E240E351E440E551E54E08516910409F08ACF56C4E4EAF5E074
:2077000064918F0108C088E290E10E94C2100F5F1F4FF80164916623B1F746C48091E204D1
:207720009091E30405966AE270E00E94000EFC01009709F439C43197108236C4E1EAF5E0D8
:2077400064918F0108C088E290E10E94C2100F5F1F4FF80164916623B1F74091720450916A
:207760007304609174047091750488E290E122E00E94FA90EEE9F5E064918F0108C088E243
:2077800090E10E94C2100F5F1F4FF80164916623B1F74091760450917704609178047091F4
:2077A000790488E290E122E00E94FA90EBE9F5E064918F0108C088E290E10E94C2100F5F90
:2077C0001F4FF80164916623B1F740917A0450917B0460917C0470917D0488E290E122E09D
:2077E0000E94FA90E8E9F5E064918F0108C088E290E10E94C2100F5F1F4FF80164916623C8
:20780000B1F740917E0450917F04609180047091810488E290E122E00E94FA90EDE8F5E05B
:2078200064918F0108C088E290E10E94C2100F5F1F4FF80164916623B1F780E00E942C6E15
:207840000E940A95209184063091850640918606509187060E946F94AB01BC0188E290E1AC
:2078600022E00E94FA90EAE8F5E064918F0108C088E290E10E94C2100F5F1F4FF8016491CD
:207880006623B1F781E00E942C6E0E940A95209188063091890640918A0650918B060E94D5
:2078A0006F94AB01BC0188E290E122E00E94FA90E7E8F5E064918F0108C088E290E10E94E5
:2078C000C2100F5F1F4FF80164916623B1F782E00E942C6E0E940A9520918C0630918D0665
:2078E00040918E0650918F060E946F94AB01BC0188E290E122E00E94FA9088E290E16CE768
:2079000071E00E94192888E290E16AE00E94C2104BC380E00E948C6D47C381E00E948C6D8B
:2079200043C388E290E16FE771E00E94192888E290E16AE00E94C210EFE7F5E064918F0113
:2079400008C088E290E10E94C2100F5F1F4FF80164916623B1F7639B03C068E971E002C0F0
:207960006DE971E088E290E10E94192888E290E16AE00E94C210E7E7F5E064918F0108C019
:2079800088E290E10E94C2100F5F1F4FF80164916623B1F7639B03C068E971E002C06DE922
:2079A00071E088E290E10E94192888E290E16AE00E94C210EFE6F5E064918F0108C088E2BE
:2079C00090E10E94C2100F5F1F4FF80164916623B1F7639B03C068E971E002C06DE971E0FB
:2079E00088E290E10E94192888E290E16AE00E94C210DAC207EE12E094E9E92E96E0F92E7C
:207A0000F80180810E94132E882349F00E94BC2E0E94DC94F70160837183828393830F5FAF
:207A20001F4F44E050E0E40EF51E52E00B3E150739F70E942B4CB8C207EE12E084E7E82EBD
:207A400086E0F82EF80180810E94132E882339F00E94BC2EF70160837183828393830F5F05
:207A60001F4F44E050E0E40EF51E52E00B3E150749F79AC283E50E94132E882351F00E9433
:207A8000BC2E6093A8067093A9068093AA069093AB0684E50E94132E882309F485C20E9435
:207AA000BC2E6093AC067093AD068093AE069093AF067AC283E50E94132E882351F00E94CD
:207AC000BC2E6093A4067093A5068093A6069093A70684E50E94132E882351F00E94BC2E1E
:207AE0006093BC067093BD068093BE069093BF0682E40E94132E882361F00E94BC2E0E94D9
:207B0000DC946093700670937106809372069093730688E50E94132E882351F00E94BC2E23
:207B20006093B0067093B1068093B2069093B3068AE50E94132E882351F00E94BC2E60937E
:207B4000B4067093B5068093B6069093B70685E40E94132E882309F427C20E94BC2E6093A2
:207B6000B8067093B9068093BA069093BB061CC207EE12E0B2E8EB2EB4E0FB2EF80180819F
:207B80000E94132E882339F00E94BC2EF70160837183828393830F5F1F4F44E050E0E40E96
:207BA000F51E52E00A3E150749F7FEC183E50E94132E882309F4F8C10E94BC2E0E94D794D8
:207BC0007093700260936F02EFC183E50E94132E882309F4E9C10E94BC2E0E94D7947093E3
:207BE000720260937102E0C180E50E94132E882351F00E94BC2E6093990270939A0280930A
:207C00009B0290939C0289E40E94132E882361F00E94BC2E0E94B57560939D0270939E022D
:207C200080939F029093A00284E40E94132E882361F00E94BC2E0E94C1756093A102709387
:207C4000A2028093A3029093A40283E40E94132E882351F00E94BC2E6093A5027093A602F8
:207C60008093A7029093A8020E94847588E290E167EA71E00E94192888E290E16AEA71E000
:207C80000E9419284091990250919A0260919B0270919C0288E290E122E00E94FA9088E278
:207CA00090E16EEA71E00E94192860919D0270919E0280919F029091A0020E94BB75AB01A3
:207CC000BC0188E290E122E00E94FA9088E290E162EB71E00E9419286091A1027091A20249
:207CE0008091A3029091A4020E94C775AB01BC0188E290E122E00E94FA9088E290E166EB8B
:207D000071E00E9419284091A5025091A6026091A7027091A80288E290E122E00E94FA90E0
:207D200088E290E16CE771E00E94192888E290E16AE00E94C21038C181E00E942A4C34C1E1
:207D400085E40E94132E882319F4CC24DD2412C00E94BC2E0E94D7946B0177FF0BC00F2ED9
:207D6000F0E0EF2EF0E0FF2EFCE80F2FF2E41F2FF02D0AC00F2EF0E0EF2EF0E0FF2EF6E1EE
:207D80000F2FF3E41F2FF02D83E50E94132E882321F00E94BC2E7B018C0183E40E94132E7D
:207DA000882319F425E030E005C00E94BC2E0E94D7949B01C801B701A6010E94C47AF4C040
:207DC0000E94616EF1C00E94F920EEC00E94F51EEBC00E94DB19E8C00E948A1BE5C086E424
:207DE0000E94132E882309F4DFC00E947B2EDCC01092A5048091AB049091AC04A091AD04B4
:207E0000B091AE048093A7049093A804A093A904B093AA040E941D2BC7C084E50E94132E54
:207E2000882309F47CC00E94BC2E0E94DC946093A604662369F1ECEAF4E064918F0108C049
:207E400088E290E10E94C2100F5F1F4FF80164916623B1F788E290E16AEB71E00E94192874
:207E6000E0912810F09129100190F081E02D88E290E16091A604099588E290E16CEB71E0F9
:207E80000E94192888E290E16AE00E94C2108CC086E40E94132E8823E1F00E94BC2E7B0149
:207EA0008C016093D4047093D5048093D6049093D70420E030E040E050E00E947696181667
:207EC00044F4E0928302F09284020093850210938602ECEAF4E064918F0108C088E290E154
:207EE0000E94C2100F5F1F4FF80164916623B1F788E290E16DEC71E00E94192840919A043C
:207F000050E0662757FD6095762F88E290E10E94E99088E290E16AE00E94C21045C0ECEA4C
:207F2000F4E064918F0108C088E290E10E94C2100F5F1F4FF80164916623B1F7ECE5F5E030
:207F400064918F0108C088E290E10E94C2100F5F1F4FF80164916623B1F72091D80430913C
:207F6000D90480E690E0289FB001299F700D389F700D11246C517B4F88E290E10E941928C3
:207F8000EAE5F5E064918F0108C088E290E10E94C2100F5F1F4FF80164916623B1F788E23C
:207FA00090E16AE00E94C2100E94212830C00FB6F89480911F1090912010A0912110B09132
:207FC00022100FBE80939D0490939E04A0939F04B093A0040FB6F89480911F10909120108A
:207FE000A0912110B09122100FBE8093AF049093B004A093B104B093B204D6CF0E94616E4B
:208000000895889A0895899A08958A9A08958B9A08958C9A08958D9A08958E9A08958F9A4C
:20802000089558985AC0599874C05A9808955B9808955C9808955D9808955E9808955F98A8
:20804000089570980895719808954098089541980895429808954398089544986CC0459879
:2080600064C046985CC047980895769808957798089528980895299808952A9808952B9832
:2080800008952C9840C02D982CC02E9830C02F9834C01098089511980895129808951398E0
:2080A0000895149808951598089516980895179808957498089575980895889808958998C8
:2080C00008958A9808958B9808958C9808958D9808958E9808958F980895E4B5EF7DE4BDD4
:2080E0000895E0918000EF77E09380000895E0918000EF7DE09380000895E0918000E77FB8
:20810000E09380000895E091B000EF77E093B0000895E091B000EF7DE093B0000895E091CA
:208120009000EF77E09390000895E0919000EF7DE09390000895E0919000E77FE093900032
:208140000895EE3258F4EE0FEE0FFF27EC3718F4EE54FF430994EC54FF430994EE270895D5
:20816000E1E00895E9B1E170D9F70895E9B1E270B9F70895E9B1E47099F70895E9B1E87003
:2081800079F70895E9B1E07159F70895E9B1E07239F70895E9B1E07419F70895E9B1E078B4
:2081A000F9F60895ECB1E170D9F60895ECB1E270B9F60895E6B1E17099F60895E6B1E270A1
:2081C00079F60895E6B1E47059F60895E6B1E87039F60895E6B1E07119F60895E6B1E07284
:2081E000E9F50895E6B1E074C9F50895E6B1E078A9F50895ECB1E07489F50895ECB1E07893
:2082000069F50895E3B1E17049F50895E3B1E27029F50895E3B1E47009F50895E3B1E87093
:20822000E9F40895E3B1E071C9F40895E3B1E072A9F40895E3B1E07489F40895E3B1E07877
:2082400069F40895E0B1E17049F40895E0B1E27029F40895E0B1E47009F40895E1E00895EE
:20826000E0B1E870D9F70895E0B1E071B9F70895E0B1E07299F70895E0B1E07479F7089577
:20828000E0B1E07859F70895ECB1E07139F70895ECB1E07219F70895EFB1E170F9F6089534
:2082A000EFB1E270D9F60895EFB1E470B9F60895EFB1E87099F60895EFB1E07179F60895FF
:2082C000EFB1E07259F60895EFB1E07439F60895EFB1E07819F608951DBA109268001CBCA3
:2082E00010BE1FBA10927A0010926E0010926F0010927000109271001092C9001092BC00AC
:2083000011B814B817B81AB81DB810BA12B815B818B81BB81EB811BA0895F89480E29EE4A0
:208320000197F1F781E08093E00080E28093D80080E69AEE0197F1F7CFDF0C9400FEFFCF94
:20834000F894CADF80E69AEE0197F1F70C940000FFCF8F938FB78F9380915B118D5F8D3755
:20836000D0F480935B11809157118F5F80935711D8F0809158118F4F80935811A8F0809193
:2083800059118F4F8093591178F080915A118F4F80935A1109C08D5780935B118091571133
:2083A0008E5F8093571128F7809153118C5F8093531158F0809154118F4F8093541128F033
:2083C000809155118F4F809355118F918FBF8F9118959B01AC0114D0FB010CC011D06E1B35
:2083E0007F0B685E7340D0F32150304040405040E851FC4F211531054105510579F708952D
:208400000FB6F89466B515B27091531180915411909155110FBE10FE05C06F3F19F07C5F95
:208420008F4F9F4F11240024660F001C660F001C702908951F93CF93DF93182FEB014CDDDD
:20844000103109F44FC0113160F4113009F442C01130A8F01E3009F455C01F3009F05CC05C
:2084600049C01931B9F01A3120F4183109F054C02BC01A31B9F01B3109F04EC01DC0209785
:2084800021F4589884B58F7D03C0C8BD84B5806284BD4AC0D0938900C0938800809180008C
:2084A000806807C0D0938B00C0938A008091800080628093800038C0D0938D00C0938C0075
:2084C000809180008860F5CFC093B3008091B000806805C0C093B4008091B000806280932E
:2084E000B00022C0D0939900C09398008091900080680FC0D0939B00C0939A00809190001F
:20850000806207C0D0939D00C0939C008091900088608093900008C0E12FF0E0C038D10521
:2085200014F41CDD01C014DDDF91CF911F910895F894E1E6F0E020E82083108283E084BD67
:2085400085BDEEE6F0E080818160808391E09093800082E0809381009093B0008093B100AF
:20856000909390008093910086E880937A0020937B0010927E0002D0789408958091D800F7
:2085800087FF02C085FF1BC081E88093D70080EA8093D80086E189BD09B400FEFDCF80E9EF
:2085A0008093D8001092E00010926B1110926C1110925F111092E1008DE08093E20008957D
:2085C0001F920F920FB60F920BB60F9211242F933F934F935F936F937F938F939F93AF933A
:2085E000BF93EF93FF931092E9008091E80083FF57C12091F1009091F1004091F1005091A0
:20860000F1006091F1007091F100A091F100B091F10082EF8093E800963009F044C0E8EE3C
:20862000F9E120E0859195918417950711F0359617C0859195918617970711F0339610C039
:20864000259135914491CD01AF3FB10519F010F08FEF90E0841708F4482FF9015EEF04C047
:208660002F5F2630F9F61CC18091E800282F30E0C90185709070892BB9F322FD14C1242F84
:20868000413208F020E2922F04C085918093F10091509923D1F7421B5093E800442321F7C2
:2086A000203211F300C1953061F48EEF8093E8008091E80080FFFCCF842F80688093E3003D
:2086C000F2C0993009F5222309F0EAC040936B1110925F1110925C118EEF8093E800E2E18E
:2086E000FAE191E09093E90085918093EB00882331F085918093EC0085918093ED009F5F19
:20870000953081F78EE1C7C0983061F4203809F0C7C08091E80080FFFCCF80916B1180934E
:20872000F10096C09132A9F4213A09F0B9C08091E80080FFFCCF20E030E0F901E153FD4FF8
:2087400080818093F1002F5F3F4F27303105A9F77FC0903209F04BC0213209F0A1C0809108
:20876000E80082FFFCCF20E030E0F901E153FD4F8091F10080832F5F3F4F27303105A9F7ED
:208780008BEF8093E8008EEF8093E8008091CF029091D002A091D102B091D20286389105AA
:2087A000A105B10519F48FE080935D118091CF029091D002A091D102B091D202863991051D
:2087C000A105B10509F06FC084E08093E9002FEF06C02093E8008091E80082FDFCCF8091E2
:2087E000EE0090E083709070892B99F7A9DD923251F4213209F054C040935F118091E800B9
:2088000080FFFCCF25C0933241F4213209F048C08091E80080FFFCCF1BC09923E9F4809113
:20882000E80080FFFCCF223811F080E00DC06093E9008091EB0090E025E0969587952A952B
:20884000E1F781701092E9008093F1001092F1008EEF8093E80027C0913011F0933001F553
:208860002230F1F4452BE1F4262F2F77822F81508630B0F48EEF8093E8002093E9009330CE
:2088800079F089E18093EB0081E090E002C0880F991F2A95E2F78093EA001092EA0003C041
:2088A00081E28093EB00FF91EF91BF91AF919F918F917F916F915F914F913F912F910F9058
:2088C0000BBE0F900FBE0F901F9018951F920F920FB60F920BB60F9211242F933F934F93A3
:2088E0005F936F937F938F939F93AF93BF93EF93FF938091E1001092E100982F83FF11C0E7
:208900001092E90081E08093EB001092EC0082E28093ED0088E08093F00010926B11109250
:208920005F1192FF1DC080916B118823C9F080915C11882359F0815080935C11882331F4D5
:2089400084E08093E9008AE38093E80080915D11882331F0815080935D11882309F4DDDC51
:2089600090FF0CC080E18093E20010926B1181E080936C1180EA8093D80019BC80916C117F
:20898000882379F094FF0DC086E189BD09B400FEFDCF80E98093D8008DE08093E2001092D7
:2089A0006C11FF91EF91BF91AF919F918F917F916F915F914F913F912F910F900BBE0F90D3
:2089C0000FBE0F901F901895B3DD0E9480440E94FC43FDCFEF92FF920F931F93CF93DF93F2
:2089E0008C017B01EA010CC0D7016D917D01D801ED91FC910190F081E02DC8010995219751
:208A0000209791F7DF91CF911F910F91FF90EF900895DF93CF9300D0CDB7DEB7DC018DE045
:208A200089838AE08A83ED91FC9111970480F581E02DCD01BE016F5F7F4F42E050E00995E0
:208A40000F900F90CF91DF9108954F925F926F927F928F929F92AF92BF92CF92DF92EF9250
:208A6000FF920F931F93DF93CF93CDB7DEB7A1970FB6F894DEBF0FBECDBF3C016A017B0181
:208A8000222349F4DC01ED91FC910190F081E02D642F099550C0213009F42AE0C114D1041A
:208AA000E104F10421F480E389A310E229C010E2822E9924AA24BB242E010894411C511CBC
:208AC000C701B601A50194010E9482CD6A3010F4605D01C0695CF201E10FF11D6083C7016E
:208AE000B601A50194010E9482CDC901DA016C017D01C114D104E104F10411F01150E0CF6E
:208B0000002331F01150FE01E10FF11D8DE28183812F90E0D301ED91FC91BE016F5F7F4FE6
:208B2000680F791F41E250E0481B590B0480F581E02DC3010995A1960FB6F894DEBF0FBEB1
:208B4000CDBFCF91DF911F910F91FF90EF90DF90CF90BF90AF909F908F907F906F905F90B4
:208B60004F9008950F9377FD02C000E008C070956095509541955F4F6F4F7F4F0DE22AE011
:208B800064DF0F9108954F925F926F927F928F929F92AF92BF92CF92DF92EF92FF920F9307
:208BA0001F93DF93CF93CDB7DEB728970FB6F894DEBF0FBECDBF3C017A018B01522ECB0180
:208BC000BA0120E030E040E050E05FD387FD02C0442406C017FB109517F910954424439429
:208BE00020E030E040E05FE3DD240AC0CA01B9012DEC3CEC4CEC5DE36DD69B01AC01D39407
:208C0000D514A0F3C801B70167D24B015C01B1D36B017C01C301B701A6012AE0042D15DFB6
:208C2000552009F447C0C701B601CFD39B01AC01C501B40150D29B01AC018EE28983D52CEE
:208C400087E0851510F487E0D82EBD2CCC24C3944E010894811C911C1FC0CA01B90120E0D9
:208C600030E040E251E436D67B018C0182D3F401EC0DF11D605D60836053C39470E088277E
:208C800077FD8095982FA3D39B01AC01C801B70122D29B01AC01BA94BB20F9F6D301ED919D
:208CA000FC91D3940480F581E02DC301B4014D2D50E0099528960FB6F894DEBF0FBECDBFF3
:208CC000CF91DF911F910F91FF90EF90DF90CF90BF90AF909F908F907F906F905F904F90E0
:208CE0000895CF93DF93DB010D900020E9F71197A61BB70BEC01E881F9810480F581E02D88
:208D0000AD010995DF91CF910895FC019FB7F89480916B11882311F420E010C083E0809338
:208D2000E9002091F200222349F48091E80082FF05C085FD03C08BE68093E8009FBF8781CF
:208D4000908597FD03C02F3F09F02F5F822F90E00895CF93DF93EC018F81988597FF09C0A7
:208D6000E881F9810084F185E02DCE01099598878F838F819885DF91CF910895FC0127812C
:208D8000308537FD05C08FEF9FEF9087878322C02FB7F89480916B11882369F083E080939D
:208DA000E9009BE68091E80085FD09C082FF03C09093E800F7CF2FBF2FEF3FEF0CC09091C9
:208DC000F1008091E80085FD03C08BE68093E8002FBF292F30E0C9010895FC0180916B11B1
:208DE000882371F09FB7F89483E08093E9002BE602C02093E8008091E80085FDFACF9FBF16
:208E00008FEF9FEF9087878308950F931F93CF93DF93EB0180916B11882309F4D5C03FB7B4
:208E2000F89484E08093E90080915E11882309F4C0C08091E80085FFC6C010925E11B9C011
:208E40009091E400915F8091E80085FD13C03FBF8091E400891721F481E080935E11B4C0D0
:208E600080916B11882309F4AFC03FB7F8940093E900E9CF8091F200212F281B822F90E0E1
:208E80004817590708F4242FE0E4E21BE03428F4EE0FFF27E25BF843099480C089918C9322
:208EA00089918C9389918C9389918C9389918C9389918C9389918C9389918C9389918C93EA
:208EC00089918C9389918C9389918C9389918C9389918C9389918C9389918C9389918C93CA
:208EE00089918C9389918C9389918C9389918C9389918C9389918C9389918C9389918C93AA
:208F000089918C9389918C9389918C9389918C9389918C9389918C9389918C9389918C9389
:208F200089918C9389918C9389918C9389918C9389918C9389918C9389918C9389918C9369
:208F400089918C9389918C9389918C9389918C9389918C9389918C9389918C9389918C9349
:208F600089918C9389918C9389918C9389918C9389918C9389918C9389918C9389918C9329
:208F800089918C9389918C9389918C9389918C9389918C9389918C9389918C938091E80049
:208FA00085FD02C07093E800421B510960935C1106C004E010E4A1EFB0E07AE363E04115B7
:208FC000510509F03DCF3FBFDF91CF911F910F910895E0E6F1E189E0DF011D928A95E9F7EC
:208FE00088EE93E0A0E0B0E08093621190936311A0936411B09365111092661182EA93E002
:2090000090936111809360110895CF93DF93DB010D900020E9F71197A61BB70BEC01E881CC
:20902000F9810480F581E02DAD010995DF91CF9108952FEF3FEFFC01308727839FDA0FB60E
:20904000F8948091571190915811A0915911B0915A110FBEAC0180916B11882329F068EC1B
:2090600070E080E090E0B5C980916C11882309F10FB6F8948091571190915811A091591130
:20908000B0915A110FBE9C0110C00FB6F8948091571190915811A0915911B0915A110FBE82
:2090A000821B930B8B3F9105A8F480916C11882361F70FB6F8948091571190915811A09163
:2090C0005911B0915A110FBE841B950B855C994008F4C1CF08955058BB27AA270ED081C20F
:2090E00041D230F046D220F031F49F3F11F41EF411C20EF4E095E7FBDCC1E92F94D280F341
:20910000BA17620773078407950718F071F49EF5C3C20EF4E0950B2EBA2FA02D0B01B901C3
:2091200090010C01CA01A0011124FF27591B99F0593F50F4503E68F11A16F040A22F232F87
:20914000342F4427585FF3CF469537952795A795F0405395C9F77EF41F16BA0B620B730BFA
:20916000840BBAF09150A1F0FF0FBB1F661F771F881FC2F70EC0BA0F621F731F841F48F458
:20918000879577956795B795F7959E3F08F0B3CF9395880F08F09927EE0F97958795089523
:2091A000E1D158F080E891E009F49EEFE2D128F040E851E059F45EEF09C0ACC16DC2E92F17
:2091C000E07831D268F3092E052AC1F3261737074807590738F00E2E07F8E02569F0E025CF
:2091E000E0640AC0EF6307F8009407FADB01B9019D01DC01CA01AD01EF935DD0F2D10AD0A5
:209200005F91552331F02BED3FE049E450FD49EC63CF0895DF93DD27B92FBF7740E85FE312
:209220001616170648075B0710F4D92FA1D29F938F937F936F9305D4E8E9F0E06ED1D1D1F2
:209240002F913F914F915F9151D3DD2349F09058A2EA2AED3FE049EC5FE3D0785D274DDF38
:20926000DF91BFC102D280F09F3740F491110EF414C260E070E080E89FE3089526F01B16D8
:20928000611D711D811D1BC135C1EFD008F481E0089577D1E395B6C10CD0A3C16AD140F0B7
:2092A00061D130F021F45F3F19F003C15111F5C131C1B9D198F39923C9F35523B1F3951B79
:2092C000550BBB27AA2762177307840738F09F5F5F4F220F331F441FAA1FA9F333D00E2E9F
:2092E0003AF0E0E830D091505040E695001CCAF729D0FE2F27D0660F771F881FBB1F2617CD
:2093000037074807AB07B0E809F0BB0B802DBF01FF2793585F4F2AF09E3F510568F0C9C05D
:20932000BCC15F3FECF3983EDCF3869577956795B795F7959F5FC9F7880F911D9695879549
:2093400097F90895E1E0660F771F881FBB1F621773078407BA0720F0621B730B840BBA0BF5
:20936000EE1F88F7E095089504D06894B11195C1089561D188F09F5790F0B92F9927B751FA
:20938000A0F0D1F0660F771F881F991F1AF0BA95C9F712C0B13081F07FD1B1E008957CC11A
:2093A000672F782F8827B85F39F0B93FCCF3869577956795B395D9F73EF49095809570951E
:2093C00061957F4F8F4F9F4F0895E89409C097FB3EF490958095709561957F4F8F4F9F4F88
:2093E0009923A9F0F92F96E9BB279395F695879577956795B795F111F8CFFAF4BB0F11F4E6
:2094000060FF1BC06F5F7F4F8F4F9F4F16C0882311F096E911C0772321F09EE8872F762F4C
:2094200005C0662371F096E8862F70E060E02AF09A95660F771F881FDAF7880F9695879510
:2094400097F9089512D180F09F3740F491110EF024C160E070E080E89FEB089526F41B1693
:20946000611D711D811D2BC045C0990F0008550FAA0BE0E8FEEF16161706E807F907C0F0EC
:2094800012161306E407F50798F0621B730B840B950B39F40A2661F0232B242B252B21F442
:2094A00008950A2609F4A140A6958FEF811D811D089597F99F6780E870E060E00895882399
:2094C00071F4772321F09850872B762F07C0662311F499270DC09051862B70E060E02AF01F
:2094E0009A95660F771F881FDAF7880F9695879597F908959F3F49F0915028F48695779574
:209500006795B7959F5F80389F4F880F9695879597F908959FEF80EC0895DF93CF931F9337
:209520000F93FF92EF92DF927B018C01689405C0DA2EEF01DBD1FE01E894A591259135916B
:2095400045915591AEF3EF01D8DDFE019701A801DA9479F7DF90EF90FF900F911F91CF91BE
:20956000DF91089500240A941616170618060906089500240A941216130614060506089544
:20958000C9CF59D0E8F3E894EFEFBB273FE048EC5FE76B3D73078407950708F1FF279F57FC
:2095A000B25A6A4D7F40894CF04032F4BE556542704F8643FF4F0894EE1F915030F0BB0FFA
:2095C000661F771F881FFF1FEBCF9EE7882332F0BB0F661F771F881F9A95C1F79395E0958F
:2095E00089CF092E0394000C11F4882352F0BB0F40F4BF2B11F460FF04C06F5F7F4F8F4FBD
:209600009F4F0895EF93E0FF06C0A2EA2AED3FE049EC5FEB72DDE5DF0F90039401FC905829
:20962000E5ECF0E018C257FD9058440F551F59F05F3F71F04795880F97FB991F61F09F3F78
:2096400079F087950895121613061406551FF2CF4695F1DF08C0161617061806991FF1CF06
:2096600086957105610508940895E5DFA0F0BEE7B91788F4BB279F3860F41616B11D672FD8
:20968000782F8827985FF7CF869577956795B11D93959639C8F30895E894BB2766277727EE
:2096A000CB0197F90895E1DE08F48FEF08955ADF19F05FDF09F02ECFFCCEB901CA011ACF2D
:2096C0009F775F77B0DF98F39923B9F35523B9F3FF27951758F4E52FE91BED3070F75E3BA5
:2096E00010F0F1E41CC09034E0F40AC0E92FE51BED3028F79E3B10F0F1E411C0503488F484
:20970000F9EA88232AF09A95660F771F881FDAF744232AF05A95220F331F441FDAF79F1B0E
:209720005F1BFF931F930F93FF92EF9279018A01BB27AB2F9B01AC01DBD09701A801BF936F
:209740007B018C01AA27BA2FB901CA01D1D0AF919701A801EF90FF900F911F91CEDC41DF77
:2097600026D14F9140FF0895552747FD509509C09B01AC0160E070E080E89FE38DCD99CE44
:20978000B9CE59DFE8F39923D9F3940F511DBBF39150504094F059F0882332F0660F771FD2
:2097A000881F91505040C1F79E3F510544F7880F911D9695879597F908955F3FACF0983EA2
:2097C0009CF0BB27869577956795B79508F4B1609395C1F7BB0F58F711F460FFE8CF6F5FBD
:2097E0007F4F8F4F9F4FE3CF58CF0EF083CE92CE68945FCE20DFC8F39923D1F3C6F3DF93B9
:20980000CF931F930F93FF92C92FDD2788232AF02197660F771F881FDAF720E030E040E8CD
:209820005FEB9FE3883920F0803E30F021968F7753DCE3EEF0E003C04FDCE0E1F1E06DDE55
:209840008B01BE01EC01FB2E6F5771097595771F880B990BBCDD28E132E741E35FE346D059
:20986000AF2D9801AE01FF900F911F91CF91DF9144DCB7CEE0DE58F19E5758F19851A0F0B2
:20988000E9F0983020F5092E9927660F771F881F991F0A94D1F712C0062E672F782F882759
:2098A000985F11F4000C07C0993FB4F38695779567959395D9F7611D711D811D3EF490953E
:2098C0008095709561957F4F8F4F9F4F08956894E4CEE2CE0BD085CE45DE28F04ADE18F04A
:2098E000952309F0E6CD16CE1124D7CE9CDEA0F3959FD1F3950F50E0551F629FF001729FF6
:20990000BB27F00DB11D639FAA27F00DB11DAA1F649F6627B00DA11D661F829F2227B00D7C
:20992000A11D621F739FB00DA11D621F839FA00D611D221F749F3327A00D611D231F849F4F
:20994000600D211D822F762F6A2F11249F5750408AF0E1F088234AF0EE0FFF1FBB1F661F08
